:020000040800F2
:1000000000000824692F0008692B00086B2B0008EA
:100010006D2B00086F2B0008712B000800000000FA
:10002000000000000000000000000000732B00082A
:10003000752B000800000000772B0008792B0008C2
:10004000B92F0008B92F0008B92F0008B92F0008F0
:10005000B92F0008B92F0008B92F0008B92F0008E0
:10006000B92F0008B92F0008B92F0008B92F0008D0
:10007000B92F0008B92F0008B92F0008B92F0008C0
:10008000B92F0008B92F0008B92F0008B92F0008B0
:10009000B92F0008B92F0008B92F0008B92F0008A0
:1000A000B92F0008B92F0008B92F0008B92F000890
:1000B000B92F0008B92F0008B92F0008B92F000880
:1000C000B92F0008B92F0008B92F0008B92F000870
:1000D000B92F0008812B0008B92F0008912B0008C8
:1000E000B92F0008B92F000800000000B92F000840
:1000F000B92F0008B92F0008B92F0008B92F000840
:10010000B92F0008B92F0008B92F0008B92F00082F
:10011000B92F0008B92F0008B92F0008B92F00081F
:10012000B92F0008B92F0008B92F0008B92F00080F
:10013000B92F0008B92F0008B92F0008B92F0008FF
:1001400000000000000000000000000000000000AF
:10015000B92F0008B92F0008B92F0008B92F0008DF
:10016000B92F0008B92F0008B92F0008B92F0008CF
:10017000B92F0008B92F0008B92F0008B92F0008BF
:10018000B92F0008B92F0008B92F0008B92F0008AF
:10019000B92F0008B92F0008B92F0008B92F00089F
:1001A000B92F0008B92F0008B92F0008B92F00088F
:1001B000B92F0008B92F0008B92F0008B92F00087F
:1001C000B92F0008B92F0008B92F0008B92F00086F
:1001D000B92F0008B92F0008B92F0008B92F00085F
:1001E000B92F0008B92F0008B92F0008B92F00084F
:1001F000B92F0008B92F0008B92F0008B92F00083F
:10020000B92F0008B92F0008B92F0008B92F00082E
:10021000B92F0008B92F0008B92F0008B92F00081E
:10022000B92F0008B92F0008B92F000800000000FE
:10023000B92F0008B92F000800000000B92F0008EE
:10024000B92F0008B92F0008B92F0008B92F0008EE
:10025000B92F0008B92F0008B92F0008B92F0008DE
:10026000B92F0008B92F0008B92F0008B92F0008CE
:10027000B92F0008B92F0008B92F000800000000AE
:10028000B92F0008B92F0008B92F0008000000009E
:0802900000000000B92F000876
:1002C00010B5054C237833B9044B13B10448AFF390
:1002D00000800123237010BDD40900240000000019
:1002E00044EA000808B5034B1BB103490348AFF3C8
:1002F000008008BD00000000D809002444EA00087E
:1003000081F0004102E000BF83F0004330B54FEAC6
:1003100041044FEA430594EA050F08BF90EA020F33
:100320001FBF54EA000C55EA020C7FEA645C7FEAC6
:10033000655C00F0E2804FEA5454D4EB5555B8BFE9
:100340006D420CDD2C4480EA020281EA030382EA5A
:10035000000083EA010180EA020281EA0303362DEC
:1003600088BF30BD11F0004F4FEA01314FF4801CBF
:100370004CEA113102D0404261EB410113F0004FD1
:100380004FEA03334CEA133302D0524263EB430388
:1003900094EA050F00F0A780A4F10104D5F1200E26
:1003A0000DDB02FA0EFC22FA05F2801841F1000181
:1003B00003FA0EF2801843FA05F359410EE0A5F155
:1003C00020050EF1200E012A03FA0EFC28BF4CF086
:1003D000020C43FA05F3C01851EBE37101F000453C
:1003E00007D54FF0000EDCF1000C7EEB00006EEB49
:1003F0000101B1F5801F1BD3B1F5001F0CD34908D3
:100400005FEA30004FEA3C0C04F101044FEA445229
:1004100012F5800F80F09A80BCF1004F08BF5FEAB0
:10042000500C50F1000041EB045141EA050130BD90
:100430005FEA4C0C404141EB0101013C28BFB1F5A2
:10044000801FE9D291F0000F04BF01460020B1FAED
:1004500081F308BF2033A3F10B03B3F120020CDAC0
:100460000C3208DD02F1140CC2F10C0201FA0CF09E
:1004700021FA02F10CE002F11402D8BFC2F1200C03
:1004800001FA02F120FA0CFCDCBF41EA0C019040B9
:10049000E41AA2BF01EB0451294330BD6FEA040402
:1004A0001F3C1CDA0C340EDC04F11404C4F12002ED
:1004B00020FA04F001FA02F340EA030021FA04F3FF
:1004C00045EA030130BDC4F10C04C4F1200220FA56
:1004D00002F001FA04F340EA0300294630BD21FA94
:1004E00004F0294630BD94F0000F83F4801306BF5A
:1004F00081F480110134013D4EE77FEA645C18BF4E
:100500007FEA655C29D094EA050F08BF90EA020FE4
:1005100005D054EA000C04BF1946104630BD91EADC
:10052000030F1EBF0021002030BD5FEA545C05D1DF
:100530004000494128BF41F0004130BD14F580041E
:100540003CBF01F5801130BD01F0004545F0FE4192
:1005500041F470014FF0000030BD7FEA645C1ABFC7
:10056000194610467FEA655C1CBF0B46024650EAFE
:10057000013406BF52EA033591EA030F41F400212A
:1005800030BD00BF90F0000F04BF0021704730B5B0
:100590004FF4806404F132044FF000054FF0000185
:1005A00050E700BF90F0000F04BF0021704730B546
:1005B0004FF4806404F1320410F0004548BF40421B
:1005C0004FF000013EE700BF42004FEAE2014FEA70
:1005D00031014FEA02701FBF12F07F4393F07F4F4B
:1005E00081F06051704732F07F4208BF704793F04E
:1005F0007F4F04BF41F40021704730B54FF4607461
:1006000001F0004521F000411CE700BF50EA010263
:1006100008BF704730B54FF000050AE050EA01020C
:1006200008BF704730B511F0004502D5404261EB7C
:1006300041014FF4806404F132045FEA915C3FF4BD
:10064000D8AE4FF003025FEADC0C18BF03325FEA5A
:10065000DC0C18BF033202EBDC02C2F1200300FA0B
:1006600003FC20FA02F001FA03FE40EA0E0021FA30
:1006700002F11444BDE600BF4FF0FF3C06E000BFAE
:100680004FF0010C02E000BF4FF0010C4DF804CD1B
:100690004FEA410C7FEA6C5C4FEA430C18BF7FEADB
:1006A0006C5C1BD001B050EA410C0CBF52EA430C09
:1006B00091EA030F02BF90EA020F0020704710F189
:1006C000000F91EA030F58BF994208BF90422CBF18
:1006D000D8176FEAE37040F0010070474FEA410C11
:1006E0007FEA6C5C02D150EA013C07D14FEA430C2F
:1006F0007FEA6C5CD6D152EA033CD3D05DF8040BA0
:10070000704700BF8446104662468C4619466346D1
:1007100000E000BF01B5FFF7B7FF002848BF10F1A8
:10072000000F01BD4DF808EDFFF7F4FF0CBF0120ED
:1007300000205DF808FB00BF4DF808EDFFF7EAFF69
:1007400034BF012000205DF808FB00BF4DF808ED24
:10075000FFF7E0FF94BF012000205DF808FB00BF19
:100760004DF808EDFFF7CEFF94BF012000205DF8A3
:1007700008FB00BF4DF808EDFFF7C4FF34BF0120B0
:1007800000205DF808FB00BF4FEA410C7FEA6C5C7B
:1007900002D150EA013C0AD14FEA430C7FEA6C5C7B
:1007A00002D152EA033C02D14FF0000070474FF0F3
:1007B000010070474FEA410212F5001215D211D51F
:1007C0006FF47873B3EB625212D94FEAC12343F04E
:1007D000004343EA505311F0004F23FA02F018BFD0
:1007E000404270474FF00000704750EA013005D199
:1007F00011F0004008BF6FF0004070474FF000005C
:10080000704700BF80F0004002E000BF81F000416F
:1008100042001FBF5FEA410392EA030F7FEA226CA6
:100820007FEA236C6AD04FEA1262D2EB1363C1BF36
:10083000D218414048404140B8BF5B42192B88BFA5
:10084000704710F0004F40F4000020F07F4018BFC8
:10085000404211F0004F41F4000121F07F4118BFE8
:10086000494292EA030F3FD0A2F1010241FA03FC90
:1008700010EB0C00C3F1200301FA03F100F0004378
:1008800002D5494260EB4000B0F5000F13D3B0F140
:10089000807F06D340084FEA310102F10102FE2AAF
:1008A00051D2B1F1004F40EBC25008BF20F001001F
:1008B00040EA03007047490040EB0000013A28BFBE
:1008C000B0F5000FEDD2B0FA80FCACF1080CB2EB41
:1008D0000C0200FA0CF0AABF00EBC25052421843BF
:1008E000BCBFD0401843704792F0000F81F4000164
:1008F00006BF80F400000132013BB5E74FEA410337
:100900007FEA226C18BF7FEA236C21D092EA030FA2
:1009100004D092F0000F08BF0846704790EA010F1C
:100920001CBF0020704712F07F4F04D1400028BF49
:1009300040F00040704712F100723CBF00F500002B
:10094000704700F0004343F0FE4040F40000704761
:100950007FEA226216BF08467FEA2363014642020D
:1009600006BF5FEA412390EA010F40F48000704720
:100970004FF0000304E000BF10F0004348BF4042C6
:100980005FEA000C08BF704743F0964301464FF002
:1009900000001CE050EA010208BF70474FF000035E
:1009A0000AE000BF50EA010208BF704711F000439F
:1009B00002D5404261EB41015FEA010C02BF84466F
:1009C0000146002043F0B64308BFA3F18053A3F5CE
:1009D0000003BCFA8CF2083AA3EBC25310DB01FA15
:1009E00002FC634400FA02FCC2F12002BCF1004F99
:1009F00020FA02F243EB020008BF20F0010070472A
:100A000002F1200201FA02FCC2F1200250EA4C007D
:100A100021FA02F243EB020008BF20EADC707047C3
:100A20004FF0FF0C1CEAD0521EBF1CEAD15392EAD1
:100A30000C0F93EA0C0F6FD01A4480EA010C4002AD
:100A400018BF5FEA41211ED04FF0006343EA501007
:100A500043EA5111A0FB01310CF00040B1F5000F49
:100A60003EBF490041EAD3715B0040EA010062F1F8
:100A70007F02FD2A1DD8B3F1004F40EBC25008BFE2
:100A800020F00100704790F0000F0CF0004C08BF00
:100A900049024CEA502040EA51207F3AC2BFD2F1CD
:100AA000FF0340EAC250704740F400004FF00003DB
:100AB000013A5DDC12F1190FDCBF00F00040704715
:100AC000C2F10002410021FA02F1C2F1200200FA53
:100AD00002FC5FEA310040F1000053EA4C0308BF1A
:100AE00020EADC70704792F0000F00F0004C02BF6B
:100AF000400010F4000F013AF9D040EA0C0093F0E6
:100B0000000F01F0004C02BF490011F4000F013B3F
:100B1000F9D041EA0C018FE70CEAD15392EA0C0FAD
:100B200018BF93EA0C0F0AD030F0004C18BF31F018
:100B3000004CD8D180EA010000F00040704790F0EE
:100B4000000F17BF90F0004F084691F0000F91F092
:100B5000004F14D092EA0C0F01D142020FD193EA58
:100B60000C0F03D14B0218BF084608D180EA0100E0
:100B700000F0004040F0FE4040F40000704740F0BC
:100B8000FE4040F4400070474FF0FF0C1CEAD0528A
:100B90001EBF1CEAD15392EA0C0F93EA0C0F69D0E6
:100BA000A2EB030280EA010C49024FEA402037D051
:100BB0004FF0805343EA111143EA10130CF0004048
:100BC0008B4238BF5B0042F17D024FF4000C8B4238
:100BD00024BF5B1A40EA0C00B3EB510F24BFA3EB18
:100BE000510340EA5C00B3EB910F24BFA3EB9103E8
:100BF00040EA9C00B3EBD10F24BFA3EBD10340EA42
:100C0000DC001B0118BF5FEA1C1CE0D1FD2A3FF687
:100C100050AF8B4240EBC25008BF20F0010070473C
:100C20000CF0004C4CEA50207F32C2BFD2F1FF03DF
:100C300040EAC250704740F400004FF00003013A10
:100C400037E792F0000F00F0004C02BF400010F4B4
:100C5000000F013AF9D040EA0C0093F0000F01F0C8
:100C6000004C02BF490011F4000F013BF9D041EAEA
:100C70000C0195E70CEAD15392EA0C0F08D142021D
:100C80007FF47DAF93EA0C0F7FF470AF084676E7F0
:100C900093EA0C0F04D14B023FF44CAF08466EE7C9
:100CA00030F0004C18BF31F0004CCAD130F0004297
:100CB0007FF45CAF31F000437FF43CAF5FE700BFEF
:100CC00042000ED2B2F1FE4F0BD34FF09E03B3EBB6
:100CD000126209D44FEA002343F0004323FA02F0E2
:100CE00070474FF00000704712F1610F01D14202CE
:100CF00002D14FF0FF3070474FF00000704700BF47
:100D000053B94AB9002908BF00281CBF4FF0FF3172
:100D10004FF0FF3000F074B9ADF1080C6DE904CE6E
:100D200000F006F8DDF804E0DDE9022304B07047C6
:100D30002DE9F047089E0D4604468846002B4DD10C
:100D40008A42944668D9B2FA82F252B101FA02F3A9
:100D5000C2F1200120FA01F10CFA02FC41EA030879
:100D600094404FEA1C45210CB8FBF5FE1FFA8CF7A6
:100D700005FB1E8341EA03430EFB07F199420BD9A1
:100D80001CEB03030EF1FF3080F01E81994240F20C
:100D90001B81AEF1020E63445B1AA4B2B3FBF5F003
:100DA00005FB103344EA034400FB07F7A7420AD9C6
:100DB0001CEB040400F1FF3380F00881A74240F2ED
:100DC000058164440238E41B40EA0E4000211EB154
:100DD000D4400023C6E90043BDE8F0878B4208D920
:100DE000002E00F0EE800021C6E900050846BDE8AF
:100DF000F087B3FA83F100294AD1AB4202D3824291
:100E000000F2F980841A65EB030301209846002E56
:100E1000E2D0C6E90048DFE702B9FFDEB2FA82F2AB
:100E2000002A40F09180A1EB0C054FEA1C471FFA05
:100E30008CFE0121B5FBF7F307FB1350250C45EAA7
:100E400000450EFB03F0A84208D91CEB050503F191
:100E5000FF3802D2A84200F2CB8043462D1AA4B23A
:100E6000B5FBF7F007FB105544EA05440EFB00FE06
:100E7000A64508D91CEB040400F1FF3502D2A645B3
:100E800000F2BB802846A4EB0E0440EA03409EE734
:100E9000C1F120078B4022FA07FC4CEA030C20FA30
:100EA00007F405FA01F31C43FD404FEA1C4900FA20
:100EB00001F3B5FBF9F8200C1FFA8CFE09FB18555D
:100EC00040EA054508FB0EF0A84202FA01F20BD9F0
:100ED0001CEB050508F1FF3A80F08880A84240F23B
:100EE0008580A8F1020865442D1AA4B2B5FBF9F07B
:100EF00009FB105544EA054500FB0EFEAE4508D936
:100F00001CEB050500F1FF346CD2AE456AD90238FE
:100F1000654440EA0840A0FB0294A5EB0E05A542FB
:100F2000C846A64656D353D05EB1B3EB080265EB74
:100F30000E0505FA07F722FA01F3CD401F43C6E973
:100F400000750021BDE8F087C2F1200320FA03F10B
:100F50000CFA02FC25FA03F395400D434FEA1C47B7
:100F60001FFA8CFEB3FBF7F107FB11302B0C43EAA1
:100F7000004301FB0EF0984204FA02F408D91CEB7E
:100F8000030301F1FF382FD298422DD9023963446F
:100F90001B1AADB2B3FBF7F007FB103345EA03456C
:100FA00000FB0EF3AB4208D91CEB050500F1FF383E
:100FB00016D2AB4214D902386544ED1A40EA014119
:100FC00038E73146304607E78646E5E61846FAE652
:100FD0004B45A9D2B9EB020864EB0C0E0138A3E72C
:100FE0004046EAE7204694E74146D1E7D0467BE712
:100FF000023B654432E7084609E76444023842E7A9
:10100000704700BF844641EA000313F003036DD12B
:10101000403A41D351F8043B40F8043B51F8043BBB
:1010200040F8043B51F8043B40F8043B51F8043BC2
:1010300040F8043B51F8043B40F8043B51F8043BB2
:1010400040F8043B51F8043B40F8043B51F8043BA2
:1010500040F8043B51F8043B40F8043B51F8043B92
:1010600040F8043B51F8043B40F8043B51F8043B82
:1010700040F8043B51F8043B40F8043B51F8043B72
:1010800040F8043B51F8043B40F8043B51F8043B62
:1010900040F8043B403ABDD2303211D351F8043B02
:1010A00040F8043B51F8043B40F8043B51F8043B42
:1010B00040F8043B51F8043B40F8043B103AEDD2B1
:1010C0000C3205D351F8043B40F8043B043AF9D202
:1010D000043208D0D2071CBF11F8013B00F8013BD5
:1010E00001D30B8803806046704700BF082A13D3E2
:1010F0008B078DD010F003038AD0C3F10403D21AFA
:10110000DB071CBF11F8013B00F8013B80D331F82D
:10111000023B20F8023B7BE7043AD9D3013A11F8AD
:10112000013B00F8013BF9D20B7803704B78437018
:101130008B7883706046704700000000000000005C
:10114000A2EB0300704700BF02780B78012A28BF8A
:101150009A42F5D16DE9044540EA0104CDE9026700
:101160006FF0000C4FEA447212B380EA010414F0ED
:10117000070F6AD100F0070420F0070004F0030510
:1011800021F007014FEAC505F0E8042314F0040F2D
:10119000F1E804670CFA05F462EA040266EA040660
:1011A0000AD063EA0403624667EA0407664603E07E
:1011B000F0E80423F1E8046782FA4CF582EA0604B9
:1011C000A4FA8CF46CBB83FA4CF583EA0705A5FA04
:1011D0008CF595B950E9022351E9026782FA4CF582
:1011E00082EA0604A4FA8CF483FA4CF583EA070534
:1011F000A5FA8CF52543DBD09CB92DBAB5FA85F458
:1012000024F0070427FA04F1DDE9026723FA04F366
:1012100003F0FF0001F0FF01FDE80445A0EB010031
:10122000704724BAB4FA84F424F0070426FA04F1CF
:10123000DDE9026722FA04F202F0FF0001F0FF018B
:10124000FDE80445A0EB0100704714F0030F3CD10A
:1012500010F0030428D150F8082B51F8083B82FA0B
:101260004CF582EA0305A5FA8CF55DB950F8042C1B
:1012700051F8043C82FA4CF582EA0305A5FA8CF594
:10128000002DE8D02DBAB5FA85F424F0070423FA2E
:1012900004F122FA04F202F0FF0001F0FF01FDE880
:1012A0000445A0EB010070474FEAC40420F003009E
:1012B00050F8082B21F0030151F8083B0CFA04F414
:1012C00062EA040263EA0403C9E710F003041AD0D7
:1012D000A1EB040120F00300E40750F8042B06D032
:1012E0000FD28B785FFAA2F4E41A06D12BB1CB7837
:1012F0005FFAB2F4E41A00D11BB920465DF8104B36
:10130000704701F1040150F8042BCC0721F00301D0
:1013100051F8043B48D824D222F07F4482FA4CF59D
:1013200094EA1325A5FA8CF50AD165B951F8043B66
:1013300084EA0204B4EB036F0ED150F8042BEBE700
:101340004FEA132355E035F07F454DD10878FDE88D
:101350000445C0F1000070474FEA126203F0FF033A
:1013600047E002EA1C4482FA4CF594EA1345A5FAD8
:101370008CF50AD165B951F8043B84EA0204B4EB58
:10138000034F0CD150F8042BEBE74FEA134330E046
:1013900015EA1C4528D10B884FEA124229E04FEA92
:1013A000124203EA1C4324E002F0FF0482FA4CF5E7
:1013B00094EA1365A5FA8CF50AD165B951F8043B96
:1013C00084EA0204B4EB032F09D150F8042BEBE7B5
:1013D0004FEA13630DE015F0FF0F05D10B684FEADC
:1013E000122223F07F4304E04FF00000FDE80445A3
:1013F000704712BA1BBA82FA4CF482EA0304A4FAC8
:101400008CF5B5FA85F402FA04F203FA04F34FEA14
:101410001260FDE80445A0EB136070470000000077
:1014200000000000000000000000000000000000BC
:1014300000000000000000000000000000000000AC
:1014400090F800F06DE9024520F007016FF0000C04
:1014500010F0070491F820F040F049804FF00004AC
:101460006FF00700D1E9002391F840F000F1080087
:1014700082FA4CF2A4FA8CF283FA4CF3A2FA8CF3BF
:101480004BBBD1E9022382FA4CF200F10800A4FA26
:101490008CF283FA4CF3A2FA8CF3E3B9D1E904237A
:1014A00082FA4CF200F10800A4FA8CF283FA4CF3B1
:1014B000A2FA8CF37BB9D1E9062301F1200182FA6B
:1014C0004CF200F10800A4FA8CF283FA4CF3A2FA71
:1014D0008CF3002BC6D0002A04BF04301A4612BA7F
:1014E000B2FA82F2FDE8024500EBD2007047D1E982
:1014F000002304F00305C4F100004FEAC50514F011
:10150000040F91F840F00CFA05F562EA05021CBFE1
:1015100063EA050362464FF00004A9E700000000FB
:1015200001F0FF01102A2BDB10F0070F08D010F894
:10153000013B013A8B422DD010F0070F42B3F6D198
:10154000F0B441EA012141EA014122F007047FF0B1
:1015500000070023F0E80256083C85EA010586EA08
:10156000010685FA47F5A3FA87F586FA47F6A5FA44
:1015700087F68EB9EED1F0BC01F0FF0102F0070250
:1015800032B110F8013B013A83EA010313B1F8D1FB
:101590000020704701387047002D06BF35460338DC
:1015A000073815F0010F07D1013015F4807F02BF15
:1015B000013015F4C03F0130F0BC0138704700BF66
:1015C00070B54FF0FF0C4CF4E06C1CEA11541DBFD9
:1015D0001CEA135594EA0C0F95EA0C0F00F0DEF8A4
:1015E0002C4481EA030621EA4C5123EA4C5350EA89
:1015F000013518BF52EA033541F4801143F48013DA
:1016000038D0A0FB02CE4FF00005E1FB02E506F06A
:101610000042E0FB03E54FF00006E1FB03569CF0BF
:10162000000F18BF4EF0010EA4F1FF04B6F5007FC5
:1016300064F5407404D25FEA4E0E6D4146EB060637
:1016400042EAC62141EA55514FEAC52040EA5E50C0
:101650004FEACE2EB4F1FD0C88BFBCF5E06F1ED86A
:10166000BEF1004F08BF5FEA500E50F1000041EBA1
:10167000045170BD06F0004646EA010140EA02004E
:1016800081EA0301B4EB5C04C2BFD4EB0C0541EA70
:10169000045170BD41F480114FF0000E013C00F385
:1016A000AB8014F1360FDEBF002001F0004170BDA9
:1016B000C4F10004203C35DA0C341BDC04F11404C2
:1016C000C4F1200500FA05F320FA04F001FA05F24E
:1016D00040EA020001F0004221F0004110EBD3701B
:1016E00021FA04F642EB06015EEA430E08BF20EA47
:1016F000D37070BDC4F10C04C4F1200500FA04F3EA
:1017000020FA05F001FA04F240EA020001F000417B
:1017100010EBD37041F100015EEA430E08BF20EAEE
:10172000D37070BDC4F1200500FA05F24EEA020E36
:1017300020FA04F301FA05F243EA020321FA04F065
:1017400001F0004121FA04F220EA020000EBD3701C
:101750005EEA430E08BF20EAD37070BD94F0000F1C
:101760000FD101F00046400041EB010111F4801F50
:1017700008BF013CF7D041EA060195F0000F18BF01
:10178000704703F00046520043EB030313F4801F3D
:1017900008BF013DF7D043EA0603704794EA0C0FF7
:1017A0000CEA135518BF95EA0C0F0CD050EA41060D
:1017B00018BF52EA4306D1D181EA030101F000418A
:1017C0004FF0000070BD50EA410606BF10461946B2
:1017D00052EA430619D094EA0C0F02D150EA0136BE
:1017E00013D195EA0C0F05D152EA03361CBF1046FF
:1017F00019460AD181EA030101F0004141F0FE419E
:1018000041F470014FF0000070BD41F0FE4141F421
:10181000780170BD70B54FF0FF0C4CF4E06C1CEA21
:1018200011541DBF1CEA135594EA0C0F95EA0C0FD6
:1018300000F0A7F8A4EB050481EA030E52EA033591
:101840004FEA013100F088804FEA03334FF08055B2
:1018500045EA131343EA12634FEA022245EA1115DF
:1018600045EA10654FEA00260EF000419D4208BF90
:10187000964244F1FD0404F5407402D25B084FEA3D
:101880003202B61A65EB03055B084FEA32024FF4E9
:1018900080104FF4002CB6EB020E75EB030E22BF46
:1018A000B61A754640EA0C005B084FEA3202B6EB06
:1018B000020E75EB030E22BFB61A754640EA5C00B5
:1018C0005B084FEA3202B6EB020E75EB030E22BF45
:1018D000B61A754640EA9C005B084FEA3202B6EB46
:1018E000020E75EB030E22BFB61A754640EADC0005
:1018F00055EA060E18D04FEA051545EA16754FEA67
:1019000006164FEAC30343EA52734FEAC2025FEA84
:101910001C1CC0D111F4801F0BD141EA00014FF013
:1019200000004FF0004CB6E711F4801F04BF0143E4
:101930000020B4F1FD0C88BFBCF5E06F3FF6AFAE00
:10194000B5EB030C04BFB6EB020C5FEA500C50F190
:10195000000041EB045170BD0EF0004E4EEA113113
:1019600014EB5C04C2BFD4EB0C0541EA045170BD1A
:1019700041F480114FF0000E013C90E645EA060E5E
:101980008DE60CEA135594EA0C0F08BF95EA0C0F8C
:101990003FF43BAF94EA0C0F0AD150EA01347FF4D4
:1019A00034AF95EA0C0F7FF425AF104619462CE7AB
:1019B00095EA0C0F06D152EA03353FF4FDAE10460E
:1019C000194622E750EA410618BF52EA43067FF45F
:1019D000C5AE50EA41047FF40DAF52EA43057FF4EF
:1019E000EBAE12E74A0011D212F5001211D20DD55A
:1019F0006FF47873B3EB62520ED44FEAC12343F015
:101A0000004343EA505323FA02F070474FF00000BE
:101A1000704750EA013002D14FF0FF3070474FF06D
:101A20000000704738B505460C462846214600227E
:101A30000023FEF781FE28B928462146BDE838403C
:101A400000F00AB8284604F1004100F005F84042D1
:101A500061EB410138BD00BFD0B50C4B00220646FA
:101A60000F46FFF7ADFDFFF7BDFF0446FEF78AFD09
:101A7000074B0022FFF7A4FD02460B4630463946CD
:101A8000FEF742FCFFF7AEFF2146D0BD0000F03D5F
:101A90000000F04100B586464FF0000C604611E0B2
:101AA0000133DBB2072B09D800F001024008002AFD
:101AB000F6D048F20842424090B2F1E70CF1010C36
:101AC0001FFA8CFC8C4504D21EF80C3058400023C1
:101AD000E8E75DF804FB0000F8B5002B18BF00280C
:101AE00024D004461E460378552B21D14378AA2BD7
:101AF00020D1837893421FD1B0F803309D1EADB240
:101B000006392F46A94219DDD91C89B2FFF7C2FF59
:101B10006B1DE35A984214D115B900273846F8BD19
:101B20002A46611D3046FFF76DFAF7E7064FF5E7E5
:101B3000064FF3E7054FF1E7054FEFE76FF0C707F3
:101B4000ECE7044FEAE700BF0CFEFFFFD4FEFFFF07
:101B500070FEFFFFA8FDFFFF08B50146014805F034
:101B600051FC08BD60EA00084FF07E50704700004D
:101B700010B500F03FFE04464368012B11D0A36866
:101B8000012B11D0E368012B11D02369012B11D057
:101B90006369012B11D02368012B11D0207EC8B9B5
:101BA00010BD00F057F8EAE700F062F8EAE700F04D
:101BB0006FF8EAE700F07CF8EAE700F089F8EAE776
:101BC000FFF7D2FFFEF700FD02460B46034805F083
:101BD00019FCE3E7FFF7C0FFE2E700BF6CEA00088B
:101BE000F8B5154B1988B3F90030002B03DB134B04
:101BF00000221A70F8BDCCB2114D00262E551148A6
:101C000005F000FC2946104805F0FCFB0F4F3B4651
:101C1000324621462846FFF75FFF39460C4805F05B
:101C2000F1FB384600F03AFD034B1E80C8223146D6
:101C3000284605F089FBDDE7E00B00240C000024BA
:101C4000180B002480EA000810EB0008F0090024BB
:101C500094EA000808B5044B044A07CA83E8070061
:101C6000184605F031FC08BDD00A0024A4EA00089B
:101C700010B5054C054A234607CA03C31A7020460F
:101C800005F022FC10BD00BFDC0A0024B0EA000809
:101C900010B5054C054A234607CA03C31A702046EF
:101CA00005F012FC10BD00BFC40A0024BCEA000805
:101CB00008B5054B054A92E80300186019711846EB
:101CC00005F002FC08BD00BFBC0A0024C8EA0008F9
:101CD00008B50348034B036005F0F6FB08BD00BFE1
:101CE000B80A002435313200002918BF002826D058
:101CF00000B586468C4688420BD100201DE002F1DB
:101D000020010FE0814217D1DAB10EF1010E0CF182
:101D1000010C9EF800200C4BD35C03F00303012B55
:101D2000EDD011469CF80000074BC35C03F00303A1
:101D3000012BE7D12030E5E7081A5DF804FB01200C
:101D400070470020F9E700BF81EC00082E207047A3
:101D50008446002318460AE0A1F14102D2B2052AC6
:101D600011D808443738022B00D800010133032B67
:101D700011D81CF80310A1F13002D2B2092AEBD815
:101D800008443038EFE7A1F16102D2B2052A03D846
:101D900008445738E7E7704700207047F8B50B1A3A
:101DA000052B60DD06460F4615460230FFF7D0FFD3
:101DB0000446A0F55C43B3F5806F56D3A0F55843B5
:101DC000B3F5806F1CD2B11D7F1A052F4FDDB3799B
:101DD0005C2B4ED1F379752B4DD106F10800FFF73E
:101DE000B7FFA0F55C43B3F5806F46D2254B03EAFD
:101DF0008424C0F30900204300F580340C2000E067
:101E000006207F2C0BD9B4F5006F0DD3B4F5803FBD
:101E10000DD3B4F5881F32D2F027042601E0002745
:101E20000126731EDBB20EE0C0270226F9E7E02789
:101E30000326F6E704F03F012A6841F08001D154FF
:101E4000A409013BDBB2002BF4D1012E06D92B688B
:101E50003C431C702B6833442B6005E02B6804F076
:101E60007F041C70F6E70020F8BD0020FCE700208E
:101E7000FAE70020F8E70020F6E70020F4E700206A
:101E8000F2E700BF00FC0F002DE9F04182B00E46E2
:101E90000F688B685D1C3D440022019207EB030C28
:101EA000FB5C222B40F0858080462C46104600E0EB
:101EB0000134E11B726891420AD22378222B07D0A9
:101EC0005C2BF5D10134E31B934272D20130EFE772
:101ED00091426ED22378222B6BD1A4EB0C0CACEB8D
:101EE0000000336901309847074600285DD0019013
:101EF0002BE0631B002B58DD6B78752B55D85C2BC2
:101F000011D35C3B192B50D8DFE803F0114F4F4F32
:101F10004F4F184F4F4F2B4F4F4F4F4F4F4F324F49
:101F20004F4F394F4047222B01D02F2B3DD1019BE2
:101F30005A1C01926A781A70022305E0019B5A1C10
:101F4000019208221A7002231D44A54239D22B782F
:101F50005C2BCED0019B5A1C019215F8012B1A70F4
:101F6000F3E7019B5A1C01920C221A700223EBE743
:101F7000019B5A1C01920A221A700223E4E7019B7A
:101F80005A1C01920D221A700223DDE7019B5A1C94
:101F9000019209221A700223D6E701AA2146284697
:101FA000FFF7FCFE03460028CED117B1736938460F
:101FB0009847ADB13368ED1AB560002002B0BDE8B6
:101FC000F081019B00221A701023C8F80C30C8F869
:101FD00010703368E41AB4600134B4600120EDE796
:101FE0000020EBE70246D0B110B40468ACB18368BE
:101FF0004068834202D30AE00133936093689842B9
:1020000002D9E15C2029F7D99368984202D01046A2
:1020100010BC7047013B9360F9E72246F7E7704731
:1020200010B5036828209847044618B128220021DB
:1020300005F08AF9204610BD38B5044678B100682D
:1020400078B1A5687DB92B1D6268934207D203223F
:102050000649284405F068FD08B90335A560204607
:1020600038BD0446FBE70024F9E700BFD0EA0008CA
:102070002DE9F04393B005460C4600231193FFF77A
:1020800065FE002C00F099802368002B00F09780FB
:10209000002331E0652A29D048336B44002203F83D
:1020A000442C0DF1040911A9484606F015FD064619
:1020B0000F46DDF84480C84500F08380C5E9066717
:1020C00041A3D3E90023FEF74BFB002864D06FF057
:1020D00000436B610823EB6001ABA8EB0308A36826
:1020E0004344A360012013B0BDE8F08303F148012D
:1020F000694401F8442C01333E2BCDD8A2681A4420
:1021000061688A42C8D221688A5C452AC2D82B2AD3
:10211000C2D3A2F12B011A29BED801A656F821F08C
:10212000ED20000899200008ED2000088D2100080E
:1021300099200008ED200008ED200008ED2000089F
:10214000ED200008ED200008ED200008ED2000083B
:10215000ED200008ED200008ED200008992000087F
:10216000992000089920000899200008992000086B
:10217000992000089920000899200008992000085B
:102180009920000899200008ED20000803F148027A
:102190006A4402F8440CAEE700220D4B3046394643
:1021A000FEF7D4FA18B14FF000436B6192E7304666
:1021B0003946FEF7FFFA68618CE7002093E70020BC
:1021C00091E700208FE700BF0000C0FFFFFFDF4165
:1021D0000000E0C138B5002918BF00281AD00D460C
:1021E00084680AB90AE024687CB1216A69B128468A
:1021F000FEF7AAFF0028F6D107E024682CB1216A77
:102200002846FFF771FD0028F7D12CB1236A2BB1C6
:10221000204638BD0024FBE70024F9E70024F7E757
:1022200038B5044616E0E36813F4807F04D12069D2
:1022300010B10F4B5B689847E36813F4007F04D13B
:10224000206A10B10A4B5B689847094B5B682046CF
:1022500098472C4654B12568E36813F4807FE2D197
:10226000A0680028DFD0FFF7DBFFDCE738BD00BF48
:1022700000000024CB68B3F57A7F80F08B802DE9D5
:10228000F04106460C460133CB60002900F0848003
:102290008B684A68934280F081800A68D25C7B2A0E
:1022A00002D00020BDE8F08101338B600846FFF7C3
:1022B00099FEA3686268934203D22268D35C7D2BA7
:1022C00059D0A3686268934204D2013BA360002501
:1022D0002F4634E0013BA3600020E3E70746A368F4
:1022E0000133A3602046FFF77DFE21462846FFF715
:1022F000CBFD002839D02046FFF774FE2B692B62F6
:1023000000232B61A368626893422ED22268D25CBC
:102310003A2A2AD10133A3602046FFF763FE214603
:10232000284600F03FF800B32046FFF75BFEA368A5
:102330006268934211D22268D35C2C2B0DD1A8463F
:1023400004F11000FFF76CFE054670B1002FC5D0F8
:10235000C8F80000C0F80480C1E7A368626893422F
:1023600003D22268D35C7D2B07D0CFB13846FFF76C
:1023700057FF002096E700252F46E368013BE36006
:1023800007B17D604023F360B760A3680133A360A9
:10239000012087E700207047002083E7002081E7C5
:1023A00000207FE7002975D070B506460C460D6801
:1023B000002D71D08868021D4B689A4206D804220D
:1023C0003749284405F0B0FB00283AD0A068421DE8
:1023D00063689A4206D805223249284405F0A4FBD6
:1023E000002835D0A068021D63689A4206D80422EE
:1023F0002D49284405F098FB00282FD0A368626877
:10240000934202D2EB5C222B30D0A36862689342E5
:1024100007D2EA5CA2F13003DBB22D2A18BF092BE8
:1024200029D9A3686268934202D2EB5C5B2B27D068
:10243000A3686268934231D2EB5C7B2B25D00020ED
:102440002DE00423F360A3680433A360012026E099
:102450000120F060A2680532A26020E00223F36050
:1024600001207061A2680432A26018E02146304663
:10247000FFF70AFD13E021463046FFF7F9FD0EE0B5
:102480002146304600F012F809E021463046FFF7B9
:10249000F1FE04E000207047002000E0002070BD45
:1024A000D4EA0008F4EA0008FCEA0008CB68B3F5B7
:1024B0007A7F6DD22DE9F04106460C460133CB60A0
:1024C0000A688B68D25C5B2A02D00020BDE8F081EC
:1024D00001338B600846FFF785FD3CB1A368626855
:1024E000934203D22268D35C5D2B48D044B1A368E9
:1024F0006268934204D2013BA36000252F461EE090
:10250000A368013BA3600020E0E7C8F80000C0F822
:102510000480A3680133A3602046FFF763FD2146D2
:102520002846FFF73FFF68B32046FFF75BFDA3682F
:10253000626893420ED22268D35C2C2B0AD1A84643
:1025400004F11000FFF76CFD0546D8B1002FDCD177
:102550000746DEE7A3686268934213D22268D35C21
:102560005D2B0FD1E368013BE36007B17D60202361
:10257000F360B760A3680133A3600120A6E70025DC
:102580002F46EFE737B13846FFF74AFE00209DE7B8
:1025900000207047002099E7F0B58BB015461E4625
:1025A00000240394049405940694079408940994D1
:1025B0002B4B1C605C600446002918BF002817D113
:1025C000002C4AD0019400230293059A049B9A425E
:1025D0003ED2029215B1029B23442B60204B01AAEC
:1025E00092E8030083E80300002738460BB0F0BDF3
:1025F000039004911B4B93E807000AAF07E907001B
:102600001846FFF70DFD0746E0B103A8FFF714FDDC
:10261000FFF7E8FC01463846FFF7C4FE90B136B933
:10262000002DE2D0039B059A13442B60DDE703A83D
:10263000FFF7D8FC059B049A934203D2039AD35C1C
:10264000002BEDD0002FBBD03846FFF7E9FDB7E7F0
:10265000002BBFD0013B0293BCE72746C5E700BF74
:10266000E80A00240000002470B5044648B10D4675
:102670001646FEF7E5FE33462A46411C2046FFF784
:102680008BFF70BD08B500221146FFF7EDFF08BDB6
:1026900008B50022FFF79EFD08BD00002DE9F84FA8
:1026A00004460146414804F0ADFE2046FFF7EAFF2C
:1026B000002874D004463E49FFF7EAFF05463D492D
:1026C0002046FFF7E5FF06463B492046FFF7E0FFBF
:1026D00080463A492046FFF7DBFF07463849204647
:1026E000FFF7D6FF824637492046FFF7D1FF8146E4
:1026F00035492046FFF7CCFF8346002D18BF002E3A
:1027000045D03B1E18BF0123B8F1000F3FD0002B6E
:102710003DD0B9F1000318BF0123BAF1000F36D044
:10272000002B34D0002832D06969284804F06AFEB2
:102730007169274804F066FED8F81410254804F0A3
:1027400061FE7969244804F05DFEDAF8141023482C
:1027500004F058FED9F81410214804F053FEDBF8B9
:102760001410204804F04EFED8F814201E4B9A6036
:1027700072695A606A691A607A69DA60DAF8142054
:102780001A61D9F814205A61DBF814201A76174B15
:1027900001221A702046FFF743FDBDE8F88F144868
:1027A00004F092FE114B00221A70F6E704EB0008C9
:1027B00018EB000824EB000828EB00082CEB0008BD
:1027C0003CEB00084CEB000860EB000878EB0008DD
:1027D0008CEB000894EB00089CEB0008B0EB0008C1
:1027E000C4EB0008DCEB0008F00A00240C00002415
:1027F000F8EB000800487047F00A002430B589B0B3
:102800000024039404940594069407941B4BD3F876
:10281000E02042F08002C3F8E020D3F8E02002F08C
:1028200080020092009AD3F8E02042F00102C3F83F
:10283000E020D3F8E02002F001020192019AD3F8DF
:10284000E02042F00202C3F8E020D3F8E03003F0C9
:1028500002030293029B0A4D22460221284601F000
:1028600071F802230393012204920594069303A9AD
:10287000284600F053FF09B030BD00BF00440258A5
:102880000000025872B6FEE700B59FB04C2200214E
:102890000BA804F059FD2022002103A804F054FDE8
:1028A000022001F055F800230093384BDA6A22F039
:1028B0000102DA62DB6A03F001030093344B9A6988
:1028C00042F440429A619B6903F440430093009BA9
:1028D0002F4B9B6913F4005FFAD02E4BD3F8F420F2
:1028E00042F00202C3F8F420D3F8F43003F00203FC
:1028F0000193019B00230293254B9A6942F44042C5
:102900009A619B6903F440430293204BDA6A42F0D8
:102910000102DA62DB6A03F001030293029B1C4BA3
:102920009B6913F4005FFAD001230B934FF48033BB
:102930000C930223149315931693F0221792189375
:1029400019931A9308231B9300231C931D930BA820
:1029500001F028F8B0B93F23039303230493002325
:102960000593082306934023079308934FF480624E
:1029700009920A93042103A801F07AFC20B91FB040
:102980005DF804FBFFF77EFFFFF77CFF00040058B3
:10299000004802580044025808B52F4B5B6913F4F5
:1029A000003F13D1BFF34F8FBFF36F8F2A4B00222D
:1029B000C3F85022BFF34F8FBFF36F8F5A6942F4B1
:1029C00000325A61BFF34F8FBFF36F8F224B5B69A9
:1029D00013F4803F27D1204B0022C3F88420BFF39B
:1029E0004F8FD3F88040C4F34E3000E01846C4F354
:1029F000C90243F6E07303EA401343EA82731649BF
:102A0000C1F860321346013A002BF2D1431E002870
:102A1000ECD1BFF34F8F4B6943F480334B61BFF36D
:102A20004F8FBFF36F8F00F0F1FAFFF72DFFFFF725
:102A3000E5FE00F047F900F081F9084800F012F8CF
:102A4000FFF7CEF8064B1B78002BF9D0FFF790F874
:102A5000034B00221A70F3E700ED00E0780C00242D
:102A60000C00002408B5054B1860054B18680023BE
:102A700002221946806804F039FF08BD0C0B0024BF
:102A800020000024022801D80120704708B504F076
:102A900071F909230360002008BD000010B501385A
:102AA00001280AD814464FF0FF3392B20748006855
:102AB00003F07EFE40B9204610BD04F05BF9092307
:102AC00003604FF0FF30F7E70520F5E70C0B00241B
:102AD000022801D80020704708B504F04BF90923FB
:102AE00003604FF0FF3008BD08B504F043F9092337
:102AF00003604FF0FF3008BD08B548B94FF0FF3311
:102B000001220848006803F0BBFE40B9012008BD5F
:102B100004F030F9092303604FF0FF30F7E7052098
:102B2000F5E700BF0C0B002408B5022804D84FF4C9
:102B300000534B60002008BD04F01CF9092303601A
:102B4000F8E7000082B0074BD3F8F42042F002020D
:102B5000C3F8F420D3F8F43003F002030193019B8F
:102B600002B0704700440258FEE7FEE7FEE7FEE7CA
:102B7000FEE770477047704708B500F075FA08BD6A
:102B800008B5024802F0E8FD08BD00BFE40B0024D0
:102B900008B5024802F0E0FD08BD00BF780C002433
:102BA0000120704708B504F0E5F8162303604FF0E4
:102BB000FF3008BD08B54FF0FF31FFF7F3FFFEE728
:102BC00010B503460C4A0D490D48006840B10C4849
:102BD00000680344521A934206D8094A136010BD94
:102BE0000748084C0460F2E704F0C4F80C230360C3
:102BF0004FF0FF30F3E700BF00000824000400009E
:102C0000100B0024580D0024244B1B6803F00F0305
:102C1000062B06D8214A136823F00F0343F007035D
:102C200013601F4B1A6842F001021A6000221A61F9
:102C300019681C4A0A401A60184B1B6813F0080FE9
:102C400006D0164A136823F00F0343F007031360FE
:102C5000134B00229A61DA611A621349996213498F
:102C6000D962134919635A639963DA6319645A6420
:102C7000196821F4802119601A660E4B1A680E4BF0
:102C80001340B3F1005F03D20C4B0122C3F80821BB
:102C90000B4B43F2D2021A60704700BF0020005273
:102CA000004402587FEDF6EA000202020000FF0134
:102CB000800201010010005C0000FFFF0080005155
:102CC0000040005208B51A481A4B03604FF4E13334
:102CD000436000238360C36003610C22426183610F
:102CE000C36103624362836203F0BAFE98B90021B4
:102CF0000F4803F0F5FF88B900210D4804F015F8DE
:102D000078B90B4803F0CDFF70B901220A49084891
:102D100003F078FF08BDFFF7B5FDE8E7FFF7B2FD68
:102D2000EAE7FFF7AFFDECE7FFF7ACFDEDE700BF2B
:102D3000E40B002400100140140B002408B51A48CD
:102D40001A4B03604FF4E133436000238360C36098
:102D500003610C2242618361C36103624362836247
:102D600003F07EFE98B900210F4803F0B9FF88B93F
:102D700000210D4803F0D9FF78B90B4803F091FF0B
:102D800070B901220A49084803F03CFF08BDFFF76B
:102D900079FDE8E7FFF776FDEAE7FFF773FDECE77B
:102DA000FFF770FDEDE700BF780C002400480040FD
:102DB000140B002410B5BAB00446002135913691A9
:102DC000379138913991C02204A804F0BDFA2368E4
:102DD0003E4A934204D03E4A93423CD03AB010BDA2
:102DE00001220023CDE9042304A801F0DDFC78BB17
:102DF000384BD3F8F02042F01002C3F8F020D3F89B
:102E0000F02002F010020092009AD3F8E02042F085
:102E10000102C3F8E020D3F8E03003F0010301938E
:102E2000019B4FF4C06335930223369300243794FB
:102E300038940723399335A9274800F06FFC2246C0
:102E40002146252000F03AF9252000F06DF9C5E76C
:102E5000FFF718FDCCE702220023CDE9042304A8E4
:102E600001F0A2FC78BB1B4BD3F8E82042F480228F
:102E7000C3F8E820D3F8E82002F480220292029AF4
:102E8000D3F8E02042F00202C3F8E020D3F8E030AB
:102E900003F002030393039B4FF440633593022333
:102EA00036930024379438940723399335A90B4877
:102EB00000F034FC22462146272000F0FFF82720AE
:102EC00000F032F98AE7FFF7DDFCCCE700100140A3
:102ED0000048004000440258000002580004025814
:102EE00008B502681A4B9A4200D008BD194A1388E7
:102EF000B2F90020002A09DB13F4804F11D0164AE2
:102F000012780A2A08D0134B00221A800122124993
:102F1000124803F077FEE8E7114A1A430D4B1A8076
:102F2000F4E70D4A12780D2A0DD0C3F30D010D48B8
:102F3000425401339BB2074A1380C72BE6D913468C
:102F400000221A80E2E743F48043024A1380DDE75F
:102F500000480040E00B0024140B0024780C0024EF
:102F60000080FFFF180B0024DFF834D0FFF74CFE81
:102F70000C480D490D4A002302E0D458C4500433D4
:102F8000C4188C42F9D30A4A0A4C002301E01360AA
:102F90000432A242FBD303F0F3FEFFF7FDFC7047BF
:102FA0000000082400000024D409002488F200084E
:102FB000D4090024580D0024FEE70000104B1B78B4
:102FC0000BB90120704710B504464FF47A70B0FB7E
:102FD000F3F30C4A1068B0FBF3F000F0B3F868B9F3
:102FE0000F2C01D901200AE0002221464FF0FF30CA
:102FF00000F064F8044B1C60002000E0012010BDCC
:1030000018000024100000241C00002410B5032028
:1030100000F042F801F020F80F498B69C3F3032355
:103020000E4AD35C03F01F03D8408B6903F00F03F3
:10303000D35C03F01F0320FA03F3094A1360094B22
:1030400018600F20FFF7BAFF10B10124204610BD11
:103050000446FFF777FDF9E70044025848EC000802
:103060001400002410000024034B1B78034A11684D
:103070000B441360704700BF180000240C0D00249F
:10308000014B1868704700BF0C0D0024014B1868F5
:10309000000C70470010005C0649CB6823F4E06325
:1030A0001B041B0C000200F4E0600343024A1A43B5
:1030B000CA60704700ED00E00000FA0500B5174B4C
:1030C000DB68C3F30223C3F1070CBCF1040F28BF74
:1030D0004FF0040C03F1040EBEF1060F14D9033BAC
:1030E0004FF0FF3E0EFA0CFC21EA0C0199400EFA5B
:1030F00003F322EA03031943002807DB0901C9B2DD
:10310000074B19545DF804FB0023E9E700F00F00BA
:103110000901C9B2034B1954F4E700BF00ED00E008
:1031200000E400E014ED00E0002807DB00F01F02DF
:10313000400901239340024A42F82030704700BF03
:1031400000E100E00138B0F1807F0BD24FF0E023C6
:103150005861054AF02182F8231000209861072267
:103160001A6170470120704700ED00E070B5044619
:10317000FFF786FF002C00F09181054694F835306A
:10318000DBB2022B06D080236365002384F8343041
:10319000012070BD23688C498C4A934218BF8B4232
:1031A00030D0183293422DD0183293422AD01832A0
:1031B000934227D01832934224D01832934221D020
:1031C000183293421ED002F5567293421AD018322A
:1031D000934217D01832934214D01832934211D030
:1031E000183293420ED0183293420BD018329342C9
:1031F00008D01832934205D01A6822F00E021A60E5
:10320000266809E01A6822F01E021A6022685369D3
:1032100023F080035361266823686B496B4A93420D
:1032200018BF8B4242D0183293423FD0183293429B
:103230003CD01832934239D01832934236D01832EB
:10324000934233D01832934230D002F556729342F3
:103250002CD01832934229D01832934226D01832FB
:10326000934223D01832934220D0183293421DD07B
:10327000183293421AD01832934217D0544A9342CC
:1032800014D01432934211D0143293420ED014321F
:1032900093420BD01432934208D01432934205D09B
:1032A0001432934202D01432934204D1226E136836
:1032B00023F48073136023684349444A934218BF40
:1032C0008B422FD0183293422CD01832934229D0FF
:1032D0001832934226D01832934223D018329342A8
:1032E00020D0183293421DD002F55672934219D065
:1032F0001832934216D01832934213D018329342A8
:1033000010D0183293420DD0183293420AD018329E
:10331000934207D01832934204D01A6822F0010277
:103320001A6003E01A6822F001021A60336813F091
:10333000010F0ED0FFF7A4FE431B052BF6D9202367
:103340006365032384F83530002384F8343001208A
:103350001FE723681C491D4A934218BF8B4239D08E
:103360001832934236D01832934233D018329342F7
:1033700030D0183293422DD0183293422AD01832CE
:10338000934227D002F55672934223D018329342CB
:1033900020D0183293421DD0183293421AD01832DE
:1033A000934217D01832934214D01832934211D05E
:1033B000183293420ED0A16DE36D03F01F0201237A
:1033C00093404B600DE000BF100002402800024017
:1033D00008540258A16DE36D03F01F023F23934090
:1033E0008B6023682E492F4A934218BF8B4242D0EC
:1033F000183293423FD0183293423CD01832934255
:1034000039D01832934236D01832934233D0183222
:10341000934230D002F5567293422CD01832934228
:1034200029D01832934226D01832934223D0183232
:10343000934220D0183293421DD0183293421AD0B2
:103440001832934217D0184A934214D01432934240
:1034500011D0143293420ED0143293420BD0143256
:10346000934208D01432934205D01432934202D0D2
:10347000143293420BD1636EA26E5A60E36E33B185
:103480001A6822F480721A60236F626F5A600123F7
:1034900084F83530002084F834007AE6012078E69C
:1034A000100002402800024008540258002800F092
:1034B000298108B5024690F83530DBB2022B03D0E3
:1034C00080234365012008BD0368904890498B42E2
:1034D00018BF83420CBF0121002166D030308342E7
:1034E00063D01830834260D0183083425DD01830EA
:1034F00083425AD01830834257D01830834254D078
:1035000000F55670834250D0183083424DD01830A9
:1035100083424AD01830834247D01830834244D087
:103520001830834241D0183083423ED01830834255
:103530003BD0196821F00E0119601368A0F5956061
:1035400073498B4218BF83426AD072498B4267D05D
:1035500018318B4264D018318B4261D018318B42C4
:103560005ED018318B425BD018318B4258D001F5B8
:1035700056718B4254D018318B4251D018318B4246
:103580004ED018318B424BD018318B4248D0183175
:103590008B4245D018318B4242D018318B423FD0FC
:1035A000196821F0010119603EE0042082F835001D
:1035B00081BB584A93422DD0183293422AD01832F8
:1035C000934227D01832934224D01832934221D00C
:1035D000183293421ED002F5567293421AD0183216
:1035E000934217D01832934214D01832934211D01C
:1035F000183293420ED0183293420BD018329342B5
:1036000008D01832934205D01A6822F001021A60DD
:10361000002058E71A6822F001021A60002052E7E1
:10362000196821F0010119601368384838498B4244
:1036300018BF834242D018318B423FD018318B42A1
:103640003CD018318B4239D018318B4236D01831EA
:103650008B4233D018318B4230D001F556718B42FA
:103660002CD018318B4229D018318B4226D01831FA
:103670008B4223D018318B4220D018318B421DD081
:1036800018318B421AD018318B4217D022498B4205
:1036900014D014318B4211D014318B420ED014311E
:1036A0008B420BD014318B4208D014318B4205D0A1
:1036B00014318B4202D014318B4217D1116E0B683A
:1036C00023F480730B60906DD36D03F01F01012311
:1036D0008B404360536E916E5960D36E33B119685D
:1036E00021F480711960136F516F5960012382F8C2
:1036F0003530002382F83430136D2BB110469847D3
:103700000020E0E6012070470020DCE610000240C7
:1037100028000240400002400854025870B582B0B0
:1037200000236EE085685E000324B44025EA0405AA
:10373000CC68B4402C438460446824EA0C0C4C6888
:10374000C4F300149C4044EA0C0444606CE0DD08BF
:10375000083550F8256003F007044FEA840C0F2465
:1037600004FA0CF426EA040E0C6904FA0CF444EA98
:103770000E0440F825406FE0092400E0002404FA1C
:103780000EF42C430CF1020C6B4D45F82C404FF01D
:10379000B0442568D44325EA0206D1F804C01CF4DD
:1037A000801F01D042EA05064FF0B0452E606D68DB
:1037B00004EA0506D1F804C01CF4001F01D042EA57
:1037C00005064FF0B0456E60D5F8845004EA050652
:1037D000D1F804C01CF4003F01D042EA05064FF0C6
:1037E000B045C5F88460D5F880502C404E6816F47A
:1037F000803F01D042EA05044FF0B042C2F8804059
:1038000001330A6832FA03F400F093804FF0010CA0
:103810000CFA03FC1CEA0202F2D04C6804F0030428
:10382000013C012C7FF67EAF4C6804F00304032CAE
:103830000CD0C4685D004FF0030C0CFA05FC24EAC0
:103840000C0C8C68AC4044EA0C04C4604C6804F076
:103850000304022C3FF47BAF04684FEA430E4FF0A1
:10386000030C0CFA0EFC24EA0C0C4C6804F0030464
:1038700004FA0EF444EA0C0404604C6814F4403F6B
:10388000BED02E4CD4F8F45045F00205C4F8F450E4
:10389000D4F8F44004F002040194019C4FEA930C24
:1038A0000CF10205244C54F8255003F003044FEAB0
:1038B000840E0F2404FA0EF425EA0405204CA042DD
:1038C0003FF45CAF04F58064A04222D004F580642C
:1038D000A04220D004F58064A0421ED004F580648C
:1038E000A0421CD004F58064A0421AD004F5806484
:1038F000A04218D004F58064A04216D004F580647C
:10390000A04214D004F58064A0423FF435AF0A24ED
:1039100035E7012433E7022431E703242FE70424A9
:103920002DE705242BE7062429E7072427E70824A9
:1039300025E702B070BD00BF0004005800440258E3
:10394000000002580AB18161704709048161704723
:10395000134BDB6813F0040F07D1114BDB6803F046
:10396000070383421AD00120704710B50C4AD36870
:1039700023F007031843D060FFF782FB0446084B8F
:103980005B6813F4005F07D1FFF77AFB001BB0F50B
:103990007A7FF4D9012000E0002010BD002070479C
:1039A00000480258002800F0398338B504460368FF
:1039B00013F0010F25D0944A136903F03803926A7B
:1039C000102B15D0182B0FD06368B3F5803F3FD074
:1039D000002B53D18C4B1A6822F480321A601A687B
:1039E00022F480221A6038E002F00302022AEBD1AE
:1039F000854B1B6813F4003F03D06368002B00F075
:103A00000F83236813F0020F00F0A1807E4A136930
:103A1000926A13F038035AD0182B55D0E368002B64
:103A200000F0DE8078490A6822F0190213430B6027
:103A3000FFF726FB0546744B1B6813F0040F40F09C
:103A4000AD80FFF71DFB401B0228F4D90320EEE2F6
:103A50006D4A136843F48033136063682BB3FFF738
:103A60000FFB0546684B1B6813F4003FC9D1FFF7F5
:103A700007FB401B6428F5D90320D8E2B3F5A02F3B
:103A800009D0614B1A6822F480321A601A6822F455
:103A900080221A60E1E75C4B1A6842F480221A60C7
:103AA0001A6842F480321A60D7E7FFF7E9FA054650
:103AB000554B1B6813F4003FA3D0FFF7E1FA401BFE
:103AC0006428F5D90320B2E212F0030FA6D14E4BC1
:103AD0001B6813F0040F03D0E368002B00F0A282F0
:103AE000494A136823F01903E1680B431360FFF799
:103AF000C7FA0546444B1B6813F0040F06D1FFF7C5
:103B0000BFFA401B0228F5D9032090E2FFF7BEFA66
:103B100041F20303984212D82269402A07D03A4959
:103B20004B6823F47C3343EA02334B600FE0364AA0
:103B3000536823F47C3343F40033536007E0324A84
:103B4000536823F0FE43216943EA0163536023680D
:103B500013F0100F00F088802B4A136903F038032C
:103B6000926A082B56D0182B50D0E369002B00F036
:103B7000B880254A136843F080031360FFF780FA8A
:103B80000546214B1B6813F4807F40F08880FFF7C7
:103B900077FA401B0228F4D9032048E2FFF776FAAF
:103BA00041F20303984212D82269402A07D01649ED
:103BB0004B6823F47C3343EA02334B60C7E7124A75
:103BC000536823F47C3343F400335360BFE70E4A59
:103BD000536823F0FE43216943EA01635360B6E76B
:103BE000094A136823F001031360FFF749FA0546F9
:103BF000054B1B6813F0040FA9D0FFF741FA401BD7
:103C00000228F5D9032012E20044025802F0030210
:103C1000012AAAD1A14B1B6813F4807F03D0E3696A
:103C2000802B40F00182FFF731FA41F20303984202
:103C300012D8226A202A07D098494B6823F0F8430B
:103C400043EA82634B600FE0944A536823F0F843E1
:103C500043F08043536007E0904AD36823F07C53DD
:103C6000216A43EA0163D360236813F0080F60D030
:103C70006369002B49D0894A536F43F001035367AE
:103C8000FFF7FEF90546854B5B6F13F0020F50D12D
:103C9000FFF7F6F9401B0228F5D90320C7E1FFF72B
:103CA000F5F941F20303984212D8226A202A07D07C
:103CB0007A494B6823F0F84343EA82634B60D3E7C9
:103CC000764A536823F0F84343F080435360CBE7D0
:103CD000724AD36823F07C53216A43EA0163D360BC
:103CE000C2E76E4A136823F080031360FFF7C8F938
:103CF00005466A4B1B6813F4807FB5D0FFF7C0F907
:103D0000401B0228F5D9032091E1644A536F23F048
:103D100001035367FFF7B4F90546604B5B6F13F07F
:103D2000020F06D0FFF7ACF9401B0228F5D903209B
:103D30007DE1236813F0200F29D0A3699BB1574A76
:103D4000136843F480531360FFF79AF90546534B09
:103D50001B6813F4005F1AD1FFF792F9401B022889
:103D6000F5D9032063E14D4A136823F480531360AF
:103D7000FFF786F90546494B1B6813F4005F06D030
:103D8000FFF77EF9401B0228F5D903204FE1236895
:103D900013F0040F21D1636A002B00F047813F4AE2
:103DA000126902F03802182A00F0EE80022B79D056
:103DB0003A4A136823F080731360FFF761F90446F1
:103DC000364B1B6813F0007F00F0DC80FFF758F9DA
:103DD000001B0228F4D9032029E1314A136843F477
:103DE00080731360FFF74CF905462D4B1B6813F4E5
:103DF000807F06D1FFF744F9401B6428F5D90320E2
:103E000015E1A368012B0AD00BBB244B1A6F22F0DB
:103E100001021A671A6F22F004021A6704E01F4AAF
:103E2000136F43F001031367A36833B3FFF728F957
:103E300005461A4B1B6F13F0020FACD1FFF720F9A8
:103E4000401B41F288339842F3D90320EFE0052B61
:103E500009D0124B1A6F22F001021A671A6F22F072
:103E600004021A67E0E70D4B1A6F42F004021A676A
:103E70001A6F42F001021A67D6E7FFF701F905460B
:103E8000064B1B6F13F0020F85D0FFF7F9F8401BAC
:103E900041F288339842F3D90320C8E00044025825
:103EA00000480258694A136823F080731360FFF7D3
:103EB000E7F80546654B1B6813F0007F06D0FFF757
:103EC000DFF8401B0228F5D90320B0E05F4B996A68
:103ED0005F4A0A40A16AE06A41EA00110A439A6215
:103EE000226B013AC2F30802616B0139490289B2BF
:103EF0000A43A16B0139090401F4FE010A43E16B95
:103F00000139090601F0FE410A431A63DA6A22F018
:103F10000102DA62596B4F4A0A40A16C42EAC102BF
:103F20005A63DA6A22F00C02216C0A43DA62DA6A16
:103F300022F00202616C0A43DA62DA6A42F48032E9
:103F4000DA62DA6A42F40032DA62DA6A42F4802231
:103F5000DA62DA6A42F00102DA621A6842F08072CA
:103F60001A60FFF78DF80446384B1B6813F0007F8A
:103F700006D1FFF785F8001B0228F5D9032056E08B
:103F8000002054E0002052E0304A916A106B012B6F
:103F90004ED001F00303A26A93424BD1C1F3051145
:103FA000E36A994248D1C0F30802236B013B9A426D
:103FB00044D1C0F34622636B013B9A4240D1C0F327
:103FC0000642A36B013B9A423CD1C0F30660E36B0F
:103FD000013B984238D11D4B5B6BC3F3CC03A26C01
:103FE0009A4201D1002022E0184AD36A23F001034B
:103FF000D362FFF745F80546FFF742F8A842FBD029
:10400000124A516B134B0B40A16C43EAC10353633B
:10401000D36A43F00103D362002008E00120704717
:10402000012004E0012002E0012000E0002038BD72
:104030000120FCE70120FAE70120F8E70120F6E77C
:104040000120F4E70120F2E70120F0E700440258E4
:104050000CFCFFFF0700FFFFF8B57E4B1B6903F068
:104060003803102B00F0F280182B10D013B17A4CCB
:104070002046F8BD774B1B6813F0200F00F0E88056
:10408000744B1868C0F3C100744CC440F0E7714B26
:104090009D6A05F003059C6AC4F30514D86A00F014
:1040A00001005B6BC3F3CC0303FB00F0FCF760FC87
:1040B0000646002CDCD0012D76D0022D00F0A48025
:1040C0000DB32046FCF754FC01466548FCF75CFD47
:1040D0000446604B186BC0F30800FCF749FC05462A
:1040E0004FF064513046FCF79BFC01462846FCF734
:1040F0008FFB4FF07E51FCF78BFB01462046FCF70F
:104100008FFC044671E0534B1B6813F0200F29D03D
:10411000504F3B68C3F3C1035048D840FCF728FC1C
:1041200005462046FCF724FC01462846FCF72CFDFA
:104130000446386BC0F30800FCF71AFC05464FF044
:1041400064513046FCF76CFC01462846FCF760FBE6
:104150004FF07E51FCF75CFB01462046FCF760FC0B
:10416000044642E02046FCF703FC01463D48FCF7CC
:104170000BFD0446374B186BC0F30800FCF7F8FB47
:1041800005464FF064513046FCF74AFC014628468C
:10419000FCF73EFB4FF07E51FCF73AFB0146204610
:1041A000FCF73EFC044620E02046FCF7E1FB01461C
:1041B0002B48FCF7E9FC0446264B186BC0F30800BB
:1041C000FCF7D6FB05464FF064513046FCF728FC5F
:1041D00001462846FCF71CFB4FF07E51FCF718FB0C
:1041E00001462046FCF71CFC04461A4B1B6BC3F32C
:1041F0004623581CFCF7BCFB01462046FCF7C4FCD8
:10420000FCF75EFD044633E72046FCF7B1FB0146B0
:104210001548FCF7B9FC04460E4B186BC0F30800B8
:10422000FCF7A6FB05464FF064513046FCF7F8FB5F
:1042300001462846FCF7ECFA4FF07E51FCF7E8FA0D
:1042400001462046FCF7ECFB0446CEE7074C0FE79F
:10425000024C0DE70044025800093D000090D003D5
:104260000024744A0024744C0024F44A00127A009A
:10427000002800F0328170B50D4604469B4B1B6848
:1042800003F00F038B420BD2984A136823F00F03FD
:104290000B431360136803F00F038B4240F01F8140
:1042A000236813F0040F0CD02269914B9B6903F033
:1042B00070039A4205D98E498B6923F070031A4323
:1042C0008A61236813F0080F0CD06269884BDB69A0
:1042D00003F070039A4205D98549CB6923F0700336
:1042E0001A43CA61236813F0100F0CD0A269804BE7
:1042F000DB6903F4E0639A4205D97D49CB6923F475
:10430000E0631A43CA61236813F0200F0CD0E269FE
:10431000774B1B6A03F070039A4205D974490B6A04
:1043200023F070031A430A62236813F0020F0CD0C3
:10433000E2686F4B9B6903F00F039A4205D96C4901
:104340008B6923F00F031A438A61236813F0010F6E
:1043500041D0674A936923F47063A1680B4393616A
:104360006368022B0AD0032B27D0012B2CD0604A84
:10437000126812F0040F06D10120ADE0126812F4A9
:10438000003F00F0AE805A490A6922F00702134349
:104390000B61FEF775FE0646554B1B6903F03803AB
:1043A0006268B3EBC20F16D0FEF76AFE801B41F2C3
:1043B00088339842F0D903208EE04D4A126812F0FB
:1043C000007FE0D1012087E0494A126812F4807F23
:1043D000D9D1012080E0236813F0020F0CD0E268ED
:1043E000434B9B6903F00F039A4205D240498B6906
:1043F00023F00F031A438A613C4B1B6803F00F0341
:10440000AB420AD9394A136823F00F032B431360D8
:10441000136803F00F03AB4265D1236813F0040F58
:104420000CD02269324B9B6903F070039A4205D28B
:104430002F498B6923F070031A438A61236813F0B4
:10444000080F0CD062692A4BDB6903F070039A42B3
:1044500005D22749CB6923F070031A43CA61236848
:1044600013F0100F0CD0A269214BDB6903F4E06359
:104470009A4205D21E49CB6923F4E0631A43CA610C
:10448000236813F0200F0CD0E269194B1B6A03F06C
:1044900070039A4205D216490B6A23F070031A433F
:1044A0000A62FFF7D9FD12498B69C3F30323114A4E
:1044B000D35C03F01F03D8408B6903F00F03D35C78
:1044C00003F01F0320FA03F30B4A13600B4B186031
:1044D0000B4B1868FEF772FD70BD0120704701207C
:1044E000FAE70120F8E70120F6E700BF00200052BC
:1044F0000044025848EC0008140000241000002476
:104500001C00002408B5FFF7A7FD0B4A9369C3F30D
:1045100003230A49CB5C03F01F0320FA03F39269DB
:1045200002F00F02885C00F01F0023FA00F0044A3A
:104530001060044A136008BD0044025848EC0008AB
:10454000140000241000002408B5FFF7DBFF054B22
:10455000DB69C3F30213044AD35C03F01F03D840A2
:1045600008BD00BF0044025848EC000808B5FFF73A
:10457000C9FF054BDB69C3F30223044AD35C03F094
:104580001F03D84008BD00BF0044025848EC000893
:10459000404B9B6A03F00303032B79D070B50546AB
:1045A0000E463C4A136823F080631360FEF768FDF3
:1045B0000446384B1B6813F0006F06D0FEF760FD11
:1045C000031B022BF5D9032070BD324B9A6A22F4EB
:1045D0007C32296842EA01329A626A68013AC2F37F
:1045E0000802A9680139490289B20A43E968013918
:1045F000090401F4FE010A4329690139090601F0A1
:10460000FE410A439A63DA6A22F0C00269690A43EA
:10461000DA62DA6A22F02002A9690A43DA62DA6A07
:1046200022F01002DA62D96B1B4A0A40E96942EAB9
:10463000C102DA63DA6A42F01002DA62C6B91A46D7
:10464000DB6A43F40023D362124A136843F08063A9
:104650001360FEF715FD04460E4B1B6813F0006F48
:1046600014D1FEF70DFD001B0228F5D90320ABE79E
:10467000012E05D0074AD36A43F40013D362E3E75F
:10468000044AD36A43F48013D362DDE700209BE73A
:1046900001207047004402580700FFFF404B9B6A0F
:1046A00003F00303032B79D070B505460E463C4A50
:1046B000136823F080531360FEF7E2FC0446384B86
:1046C0001B6813F0005F06D0FEF7DAFC031B022B19
:1046D000F5D9032070BD324B9A6A22F07C722968AA
:1046E00042EA01529A626A68013AC2F30802A96872
:1046F0000139490289B20A43E9680139090401F420
:10470000FE010A4329690139090601F0FE410A4305
:104710001A64DA6A22F4406269690A43DA62DA6A80
:1047200022F40072A9690A43DA62DA6A22F480721A
:10473000DA62596C1B4A0A40E96942EAC1025A64CA
:10474000DA6A42F48072DA62C6B91A46DB6A43F466
:104750008003D362124A136843F080531360FEF75C
:104760008FFC04460E4B1B6813F0005F14D1FEF75C
:1047700087FC001B0228F5D90320ABE7012E05D0EA
:10478000074AD36A43F08073D362E3E7044AD36AEB
:1047900043F40003D362DDE700209BE7012070476C
:1047A000004402580700FFFFF8B50446036813F001
:1047B000006F30D0836EB3F5001F26D00ED8EBB15A
:1047C000B3F5801F07D102210830FFF7E1FE05464F
:1047D00045B12E4621E0012635461EE0B3F5401FC7
:1047E00009D10025984A136D23F44013A16E0B43A1
:1047F0001365002611E0012635460EE0924AD36A81
:1048000043F40033D3620025ECE702212830FFF7A0
:1048100045FF0546DCE700263546236813F4807F14
:1048200014D0A36D042B32D8DFE803F003232A0849
:104830000800854AD36A43F40033D36255BB824AE9
:10484000136D23F00703A16D0B431365236813F465
:10485000007F31D0E36D802B4CD020D8002B43D08B
:10486000402B19D1002104F10800FFF791FE054605
:104870001AE0002104F10800FFF78AFE0546DDE793
:10488000002104F12800FFF709FF0546D6E70126BD
:104890003546DBE72E46D9E7012635460CE0C02B2E
:1048A00002D0B3F5807F1CD15DBB674A136D23F442
:1048B000E073E16D0B431365236813F4806F46D0FA
:1048C000D4F8A830B3F5800F39D01FD88BB3B3F527
:1048D000001F18D1002104F10800FFF759FE05461A
:1048E0001AE001263546E7E7574AD36A43F4003316
:1048F000D362D9E7002104F12800FFF7CFFE054677
:10490000D2E72E46D8E70126354620E0B3F5C00FA2
:1049100002D0B3F5000F09D1C5B94B4A936D23F40A
:104920006003D4F8A8100B43936510E001263546C8
:104930000DE0454AD36A43F40033D362ECE700212B
:1049400004F12800FFF7AAFE0546E5E72E46236896
:1049500013F4006F24D0D4F8AC30B3F1007F42D010
:104960000ED8002B39D0B3F1807F06D1002104F19D
:104970000800FFF70DFE054608E0012635460FE06A
:10498000B3F1407F02D0B3F1806F23D1002D31D13C
:104990002D4A936D23F0E063D4F8AC100B4393657C
:1049A000236813F0007F2ED0E36C202B40D026D854
:1049B00033B1102B20D1244AD36A43F40033D3629D
:1049C000002D3CD1204AD36C23F03003E16C0B4323
:1049D000D36418E001263546E2E71B4AD36A43F464
:1049E0000033D362D2E7002104F12800FFF756FE1E
:1049F0000546CBE72E46D3E70126354603E0302BAC
:104A0000DED001263546236813F4805F2DD0236E57
:104A1000B3F5005F4FD019D8002B46D0B3F5805FB7
:104A20000FD1002104F10800FFF7B2FD054613E0A5
:104A3000022104F10800FFF7ABFD0546C0E72E4652
:104A4000E1E70126354610E000440258B3F5405F27
:104A500002D0B3F5804F25D1002D33D1774A136DA5
:104A600023F4E043216E0B431365236813F4005FC6
:104A700038D0636EB3F5003F53D028D843B1B3F5B7
:104A8000803F21D1012104F10800FFF781FD054697
:104A9000002D4DD1694A136D23F4E023616E0B4361
:104AA00013651FE001263546DFE7644AD36A43F405
:104AB0000033D362D0E7002104F12800FFF7EEFDB8
:104AC0000546C9E72E46D0E7012635460AE0B3F58C
:104AD000802FDDD0B3F5A02FDAD0B3F5403FD7D08B
:104AE00001263546236813F4804F31D0D4F8B03016
:104AF000B3F1005F45D020D843B1B3F1805F19D145
:104B0000012104F10800FFF743FD0546002D3FD1C8
:104B10004A4A936D23F0E043D4F8B0100B439365F9
:104B200016E0012104F12800FFF7B8FD0546AFE7C4
:104B30002E46D7E7012635460AE0B3F1804FE5D08F
:104B4000B3F1A04FE2D0B3F1405FDFD0012635468C
:104B5000236813F4004F09D0236FB3F1805F19D09D
:104B6000B3F1005F24D0D3B101263546236813F09A
:104B7000807F33D0A36C032B5BD8DFE803F02722C0
:104B80005327012104F12800FFF788FD0546BDE702
:104B90002E46DDE7294AD36A43F40033D36275B960
:104BA000264A136D23F04053216F0B431365DDE755
:104BB000012104F10800FFF7EBFC0546EFE72E4664
:104BC000D4E71E4AD36A43F40033D362A5BB1B4A21
:104BD000D36C23F00303A16C0B43D364236813F459
:104BE000800F2DD1236813F0010F00F0A580E36F33
:104BF000282B00F29F80DFE803F08D9D9D9D9D9DF9
:104C00009D9D879D9D9D9D9D9D9D969D9D9D9D9DF1
:104C10009D9D8D9D9D9D9D9D9D9D8D9D9D9D9D9DE4
:104C20009D9D8D00022104F10800FFF7B1FC0546AF
:104C3000CCE701263546D1E72E46CFE7004402589F
:104C4000914A136843F480731360FEF719FA07461C
:104C50008D4B1B6813F4807F05D1FEF711FAC01B42
:104C60006428F5D90325002D4AD1884B1B6FD4F851
:104C7000B420534013F4407F0CD0844B1A6F22F4BD
:104C80004072196F41F480311967196F21F4803136
:104C900019671A67D4F8B430B3F5807F15D08DBB8F
:104CA000D4F8B43003F44072B2F5407F1ED0774A96
:104CB000136923F47C53136174490B6FD4F8B42047
:104CC000C2F30B0213430B678CE7FEF7D9F90746D3
:104CD0006E4B1B6F13F0020FE1D1FEF7D1F9C01B31
:104CE00041F288339842F3D90325D8E7674802692F
:104CF00022F47C52664901EA131313430361DBE794
:104D00002E466FE72E466DE7012104F10800FFF7FC
:104D10003FFC0546E5B95D4A536D23F03803E16F6A
:104D20000B43536508E0012104F12800FFF7B6FCAE
:104D30000546EFE701263546236813F0020F17D02A
:104D4000A36F052B28D8DFE803F00B05200B0B0B16
:104D50002E46F1E7012104F10800FFF719FC054692
:104D6000EDB94A4A536D23F00703A16F0B43536516
:104D7000236813F0040F23D0D4F89430052B45D8C2
:104D8000DFE803F0150F3D151515012104F128008A
:104D9000FFF784FC0546E3E701263546E8E72E46A3
:104DA000E6E7012104F10800FFF7F2FB054685BBA9
:104DB000364A936D23F00703D4F894100B439365A0
:104DC000236813F0200F34D0D4F89030B3F1005F93
:104DD0004ED023D843B1B3F1805F1CD1002104F140
:104DE0000800FFF7D5FB0546002D48D1274A536D33
:104DF00023F0E043D4F890100B43536519E00121F0
:104E000004F12800FFF74AFC0546D0E701263546A5
:104E1000D6E72E46D4E7012635460AE0B3F1804FA7
:104E2000E2D0B3F1A04FDFD0B3F1405FDCD0012678
:104E30003546236813F0400F37D0D4F89C30B3F5D3
:104E4000006F53D026D843B1B3F5806F19D100213C
:104E500004F10800FFF79CFB0546002D4DD10B4ADD
:104E6000936D23F4E053D4F89C100B4393651CE03E
:104E7000022104F12800FFF711FC0546B4E72E4695
:104E8000D7E70126354610E0004802580044025892
:104E9000CFFFFF00B3F5805FDFD0B3F5A05FDCD0BC
:104EA000B3F5406FD9D001263546236813F0800F43
:104EB00033D0D4F8A030B3F5804F00F0A38021D8D0
:104EC00043B1B3F5005F1AD1002104F10800FFF7E8
:104ED0005FFB0546002D40F09C80814A936D23F4D2
:104EE0006043D4F8A0100B43936516E0022104F14F
:104EF0002800FFF7D3FB0546AFE72E46D5E701268E
:104F000035460AE0B3F5004FE4D0B3F5204FE1D0C9
:104F1000B3F5C04FDED001263546236813F0080FE5
:104F20000CD0D4F88430B3F5805F74D06C4A536DE4
:104F300023F44053D4F884100B435365236813F0D3
:104F4000100F0CD0D4F89830B3F5807F6CD0644A41
:104F5000936D23F44073D4F898100B439365236842
:104F600013F4002F0BD0D4F8A430B3F5803F74D0E5
:104F7000B3F5003F67D0002B5FD00126354623688C
:104F800013F4802F0CD0D4F88830B3F5001F7CD0F8
:104F9000B3F5401F6FD0B3F5801F67D001263546AB
:104FA000236813F4803F08D0236D002B76D0B3F52F
:104FB000803F00F0818001263546236813F0005FB2
:104FC00040F08380236813F4003F00F08E80D4F813
:104FD0008030B3F5807F00F0EC8040F28380B3F541
:104FE000007F03D0B3F5407F40F0E180002D40F01A
:104FF000E6803B4A536D23F44073D4F880100B4392
:10500000536572E0022104F12800FFF747FB0546D3
:1050100060E72E4681E7022104F12800FFF73EFBFE
:10502000002883D0012681E7022104F12800FFF740
:1050300035FB00288BD0012689E7002104F1080008
:10504000FFF7A6FA05467DB9254A936D23F4403350
:10505000D4F8A4100B43936591E7022104F12800D2
:10506000FFF71CFB0546EEE72E4688E71C4AD36A8D
:1050700043F40033D3627DB9194A536D23F44013CE
:10508000D4F888100B4353658AE7012104F1280006
:10509000FFF704FB0546EEE72E4681E7104AD36A88
:1050A00043F40033D36275B90D4AD36C23F48033D3
:1050B000216D0B43D36480E7022104F10800FFF760
:1050C00067FA0546EFE72E4677E7022104F128004C
:1050D000FFF7E4FA00283FF475AF012672E700BF3E
:1050E00000440258002B81D00126236813F4801F4E
:1050F00006D04F4A136D23F00043616F0B431365D5
:10510000236813F0805F07D0494A136923F4804372
:10511000D4F8B8100B431361236813F4001F06D0B2
:10512000434A136D23F08073E16E0B4313652368CC
:1051300013F0804F09D03E4B1A6922F400421A61E5
:105140001A69D4F8BC100A431A612368002B06DAE6
:10515000374AD36C23F04053616D0B43D36423680B
:1051600013F4000F07D0324A536D23F44003D4F8F0
:105170008C100B435365636813F0010F21D16368F2
:1051800013F0020F26D1636813F0040F2BD163686C
:1051900013F0080F30D1636813F0100F35D1636836
:1051A00013F0200F3AD106B101263046F8BD012692
:1051B0009BE71F4AD36A43F40033D36216E72E46B7
:1051C00093E7002104F10800FFF7E2F90028D6D0A8
:1051D0000646D4E7012104F10800FFF7D9F90028B9
:1051E000D1D00646CFE7022104F10800FFF7D0F93D
:1051F0000028CCD00646CAE7002104F12800FFF7BA
:105200004DFA0028C7D00646C5E7012104F1280061
:10521000FFF744FA0028C2D00646C0E7022104F195
:105220002800FFF73BFA0028BDD00646BBE700BFC9
:105230000044025808B5FFF765F9054B1B6AC3F334
:105240000213044AD35C03F01F03D84008BD00BF1B
:105250000044025848EC00082DE9F0410446864B12
:105260009D6A9E6AC6F30536D86AC0F30010DB6BF0
:10527000C3F3CC0303FB00F0FBF77AFB002E00F036
:10528000F58005F003050746012D79D0022D00F0C9
:10529000CB800DB33046FBF76BFB01467748FBF73D
:1052A00073FC0546744B986BC0F30800FBF760FB7A
:1052B00006464FF064513846FBF7B2FB01463046D4
:1052C000FBF7A6FA4FF07E51FBF7A2FA01462846FB
:1052D000FBF7A6FB054674E0674B1B6813F0200F35
:1052E0002CD0DFF89481D8F80030C3F3C1036448B0
:1052F000D840FBF73DFB05463046FBF739FB01463E
:105300002846FBF741FC0546D8F83800C0F30800F2
:10531000FBF72EFB06464FF064513846FBF780FB47
:1053200001463046FBF774FA4FF07E51FBF770FAF6
:1053300001462846FBF774FB054642E03046FBF782
:1053400017FB01464F48FBF71FFC05464A4B986B7D
:10535000C0F30800FBF70CFB06464FF064513846DB
:10536000FBF75EFB01463046FBF752FA4FF07E51E9
:10537000FBF74EFA01462846FBF752FB054620E0B4
:105380003046FBF7F5FA01463C48FBF7FDFB0546C6
:10539000394B986BC0F30800FBF7EAFA06464FF06A
:1053A00064513846FBF73CFB01463046FBF730FAC8
:1053B0004FF07E51FBF72CFA01462846FBF730FBF5
:1053C00005462D4EB06BC0F34620FBF7D1FA4FF0E7
:1053D0007E51FBF71DFA01462846FBF7D5FBFBF78C
:1053E0006FFC2060B06BC0F30640FBF7C1FA4FF0D2
:1053F0007E51FBF70DFA01462846FBF7C5FBFBF78C
:105400005FFC6060B06BC0F30660FBF7B1FA4FF071
:105410007E51FBF7FDF901462846FBF7B5FBFBF78C
:105420004FFCA060BDE8F0813046FBF7A1FA0146D1
:105430001548FBF7A9FB05460F4B986BC0F3080016
:10544000FBF796FA06464FF064513846FBF7E8FA48
:1054500001463046FBF7DCF94FF07E51FBF7D8F9F7
:1054600001462846FBF7DCFA0546AAE7002323603D
:105470006360A360D6E700BF004402580024744A6A
:105480000090D0030024744C0024F44A2DE9F0412C
:105490000446864B9D6A9E6AC6F30556D86AC0F3D9
:1054A00000205B6CC3F3CC0303FB00F0FBF760FA56
:1054B000002E00F0F58005F003050746012D79D098
:1054C000022D00F0CB800DB33046FBF751FA0146B8
:1054D0007748FBF759FB0546744B186CC0F308007E
:1054E000FBF746FA06464FF064513846FBF798FA48
:1054F00001463046FBF78CF94FF07E51FBF788F9F7
:1055000001462846FBF78CFA054674E0674B1B689A
:1055100013F0200F2CD0DFF89481D8F80030C3F3BB
:10552000C1036448D840FBF723FA05463046FBF731
:105530001FFA01462846FBF727FB0546D8F840002E
:10554000C0F30800FBF714FA06464FF064513846E2
:10555000FBF766FA01463046FBF75AF94FF07E51E9
:10556000FBF756F901462846FBF75AFA054642E092
:105570003046FBF7FDF901464F48FBF705FB0546B2
:105580004A4B186CC0F30800FBF7F2F906464FF0DF
:1055900064513846FBF744FA01463046FBF738F9C8
:1055A0004FF07E51FBF734F901462846FBF738FAF5
:1055B000054620E03046FBF7DBF901463C48FBF7A7
:1055C000E3FA0546394B186CC0F30800FBF7D0F935
:1055D00006464FF064513846FBF722FA0146304642
:1055E000FBF716F94FF07E51FBF712F901462846FA
:1055F000FBF716FA05462D4E306CC0F34620FBF73C
:10560000B7F94FF07E51FBF703F901462846FBF747
:10561000BBFAFBF755FB2060306CC0F30640FBF78C
:10562000A7F94FF07E51FBF7F3F801462846FBF748
:10563000ABFAFBF745FB6060306CC0F30660FBF72C
:1056400097F94FF07E51FBF7E3F801462846FBF748
:105650009BFAFBF735FBA060BDE8F0813046FBF715
:1056600087F901461548FBF78FFA05460F4B186C72
:10567000C0F30800FBF77CF906464FF0645138464A
:10568000FBF7CEF901463046FBF7C2F84FF07E51EA
:10569000FBF7BEF801462846FBF7C2F90546AAE724
:1056A000002323606360A360D6E700BF0044025874
:1056B0000024744A0090D0030024744C0024F44A5F
:1056C000026852E8003F23F4907342E80031002959
:1056D000F6D1026802F1080353E8001F0D4B0B409E
:1056E000083242E800310029F3D1C36E012B06D005
:1056F0002023C0F88C300023C366436770470268DC
:1057000052E8003F23F0100342E800310029F6D1AF
:10571000EEE700BFFEFFFFEF704708B5026852E8F2
:10572000003F23F0400342E800310029F6D1202356
:10573000C0F8883000238367FFF7EEFF08BD70478D
:1057400008B5806B0023A0F85E30A0F85630FFF754
:10575000F6FF08BD7047000070B504460168CB69CC
:1057600008688D6840F60F021A4008D113F0200F28
:1057700005D010F0200F34D115F0805F31D12AB15F
:105780008B4A2A4033D18B4E304230D1E26E012A0F
:1057900000F0C68013F4801F03D015F4800F40F092
:1057A0009B8113F0800F07D010F0800F40F09B8199
:1057B00015F4000F40F0978113F0400F03D010F064
:1057C000400F40F0978113F4000F03D010F0804F8A
:1057D00040F0948113F0807F02D00028C0F29281C3
:1057E00070BD636F002BFBD020469847F8E713F09D
:1057F000010F09D010F4807F06D001260E62D4F884
:1058000090103143C4F8901013F0020F0BD015F034
:10581000010F08D0216802260E62D4F8901041F0E2
:105820000401C4F8901013F0040F0BD015F0010F11
:1058300008D0216804260E62D4F8901041F00201CD
:10584000C4F8901013F0080F0BD010F0200F00D107
:105850003AB1226808211162D4F890200A43C4F8B2
:10586000902013F4006F0CD010F0806F09D02268E4
:105870004FF400611162D4F8902042F02002C4F885
:105880009020D4F89020002AAAD013F0200F09D03D
:1058900010F0200F02D115F0805F03D0636F0BB1C1
:1058A00020469847D4F8902023689B6813F0400F57
:1058B00002D112F0280F2CD02046FFF701FF2368F9
:1058C0009B6813F0400F20D0226802F1080353E8D0
:1058D000003F23F04003083242E800310029F3D1B1
:1058E000D4F880306BB1344A1A65D4F88000FDF7E3
:1058F000DDFD00283FF474AFD4F88000036D9847B5
:105900006EE72046FFF71BFF6AE72046FFF717FF09
:1059100066E72046FFF713FF0023C4F890305FE7E7
:1059200013F0100F3FF436AF10F0100F3FF432AF0A
:1059300010230B6223689B6813F0400F00F09280E5
:10594000D4F8802013681D481D498B4218BF83423C
:1059500038D018318B4235D018318B4232D01831C3
:105960008B422FD018318B422CD018318B4229D04A
:1059700018318B4226D001F556718B4222D0183156
:105980008B421FD018318B421CD018318B4219D05A
:1059900018318B4216D018318B4213D018318B42FC
:1059A00010D018318B420DD05B689BB20CE000BF69
:1059B00001000010200100044157000810000240BF
:1059C000280002405B689BB2002B3FF409AFB4F89B
:1059D0005C1099427FF604AFA4F85E30D369B3F54A
:1059E000807F32D0226852E8003F23F4807342E87F
:1059F00000310029F6D1226802F1080353E8003F84
:105A000023F00103083242E800310029F3D1226873
:105A100002F1080353E8003F23F04003083242E854
:105A200000310029F3D12023C4F88C300023E36631
:105A3000226852E8003F23F0100342E800310029B9
:105A4000F6D1D4F88000FDF791FB02232367B4F868
:105A50005C10B4F85E309BB2C91A89B22046FFF7D9
:105A600079FEBDE6B4F85C10B4F85E309BB2C91A9A
:105A700089B2B4F85E309BB2002B3FF4B1AE00297E
:105A80003FF4AEAE226852E8003F23F4907342E840
:105A900000300028F6D1226802F1080353E8000F15
:105AA0001A4B0340083242E800300028F3D120238B
:105AB000C4F88C300023E3666367226852E8003F35
:105AC00023F0100342E800300028F6D102232367B8
:105AD0002046FFF73FFE83E64FF480130B6220461B
:105AE00001F0DCF87CE6A36F002B3FF479AE204692
:105AF000984775E62046FFF710FE71E6204601F054
:105B0000CFF86DE6204601F0CAF869E6FEFFFFEF28
:105B100008B5B0F86030D0F88C20222A05D0026891
:105B2000936943F00803936108BD0268516ADBB2D0
:105B3000826D0B401370836D01338365B0F85E3066
:105B40009BB2013B9BB2A0F85E30B0F85E309BB2D6
:105B5000002BE9D1026852E8003F23F4907342E839
:105B600000310029F6D1026802F1080353E8003F32
:105B700023F00103083242E800310029F3D1202349
:105B8000C0F88C300023436703670368164A9342CA
:105B90000CD05B6813F4000F08D0026852E8003F95
:105BA00023F0806342E800310029F6D1C36E012B57
:105BB00016D10023C366026852E8003F23F01003A9
:105BC00042E800310029F6D10368DA6912F0100FBB
:105BD00001D010221A62B0F85C10FFF7BBFDA3E7FA
:105BE000FDF77EF9A0E700BF000C005808B5B0F83B
:105BF0006020D0F88C30222B05D00268936943F0E6
:105C00000803936108BD03685B6A816D13400B80D4
:105C1000836D02338365B0F85E309BB2013B9BB26B
:105C2000A0F85E30B0F85E309BB2002BEAD102687B
:105C300052E8003F23F4907342E800310029F6D186
:105C4000026802F1080353E8003F23F00103083221
:105C500042E800310029F3D12023C0F88C30002322
:105C6000436703670368164A93420CD05B6813F4DA
:105C7000000F08D0026852E8003F23F0806342E83A
:105C800000310029F6D1C36E012B16D10023C36663
:105C9000026852E8003F23F0100342E80031002977
:105CA000F6D10368DA6912F0100F01D010221A62DF
:105CB000B0F85C10FFF74EFDA4E7FDF711F9A1E77E
:105CC000000C00582DE9F843B0F860600368DD6906
:105CD000D3F80090D3F80880D0F88C20222A05D081
:105CE0009A6942F008029A61BDE8F8830446B0F868
:105CF000687008E0D4F89030002B4CD1B4F85E30D6
:105D00009BB2002B4ED0002F00F0988015F0200F92
:105D100000F094802368596AF3B2A26D0B401370AF
:105D2000A36D0133A365B4F85E309BB2013B9BB217
:105D3000A4F85E302368DD6915F0070FDED015F09A
:105D4000010F09D019F4807F06D001221A62D4F81D
:105D500090301343C4F8903015F0020F0BD018F0B8
:105D6000010F08D0236802221A62D4F8903043F061
:105D70000403C4F8903015F0040FBBD018F0010FE5
:105D8000B8D0236804221A62D4F8903043F002039A
:105D9000C4F89030AEE72046FFF7D1FC0023C4F8EA
:105DA0009030ABE7226852E8003F23F4807342E86A
:105DB00000310029F6D1226802F1080353E8001FE0
:105DC000304B0B40083242E800310029F3D1202348
:105DD000C4F88C3000236367236723682A4A934200
:105DE00003D05B6813F4000F06D1E36E012B0DD0D6
:105DF0002046FDF775F886E7226852E8003F23F059
:105E0000806342E800310029F6D1EEE70023E36623
:105E1000226852E8003F23F0100342E800310029D5
:105E2000F6D12368DA6912F0100F01D010221A623D
:105E3000B4F85C102046FFF78DFC64E7B4F85E30E0
:105E40009BB2002B3FF450AFB4F868209A427FF623
:105E50004BAF226802F1080353E8003F23F0805360
:105E6000083242E800310029F3D1084B6367226809
:105E700052E8003F43F0200342E800310029F6D108
:105E800032E700BFFEFFFFEF000C0058115B000877
:105E90002DE9F843B0F860600368DD69D3F800903D
:105EA000D3F80880D0F88C20222A05D09A6942F0D5
:105EB00008029A61BDE8F8830446B0F8687008E00B
:105EC000D4F89030002B4BD1B4F85E309BB2002B4D
:105ED0004DD0002F00F0978015F0200F00F0938038
:105EE00023685B6AA26D33401380A36D0233A36500
:105EF000B4F85E309BB2013B9BB2A4F85E302368DD
:105F0000DD6915F0070FDFD015F0010F09D019F486
:105F1000807F06D001221A62D4F890301343C4F86F
:105F2000903015F0020F0BD018F0010F08D0236845
:105F300002221A62D4F8903043F00403C4F890307F
:105F400015F0040FBCD018F0010FB9D0236804225B
:105F50001A62D4F8903043F00203C4F89030AFE7EF
:105F60002046FFF7ECFB0023C4F89030ACE7226832
:105F700052E8003F23F4807342E800310029F6D153
:105F8000226802F1080353E8001F304B0B4008322F
:105F900042E800310029F3D12023C4F88C300023DB
:105FA0006367236723682A4A934203D05B6813F42C
:105FB000000F06D1E36E012B0DD02046FCF790FFB9
:105FC00087E7226852E8003F23F0806342E800310F
:105FD0000029F6D1EEE70023E366226852E8003F8D
:105FE00023F0100342E800310029F6D12368DA6972
:105FF00012F0100F01D010221A62B4F85C10204683
:10600000FFF7A8FB65E7B4F85E309BB2002B3FF4C6
:1060100051AFB4F868209A427FF64CAF226802F183
:10602000080353E8003F23F08053083242E8003170
:106030000029F3D1074B6367226852E8003F43F021
:10604000200342E800310029F6D133E7FEFFFFEFDD
:10605000000C0058ED5B000870B586B0044601687E
:1060600083680269134342691343C2691343086892
:10607000884A024013430B602268536823F440535C
:10608000E1680B435360A1692268834B9A4201D0B7
:10609000236A19439068814B03400B439360226845
:1060A000D36A23F00F03616A0B43D36222687C4BEF
:1060B0009A4221D07B4B9A4200F08C807A4B9A42D4
:1060C00000F0A280794B9A4200F0B580784B9A425A
:1060D00000F0C880774B9A4200F0F480764B9A42E9
:1060E00000F01981754B9A4200F02C816A4B9A425C
:1060F00000F03F81802333E0714B5B6D03F0380388
:10610000282B65D8DFE813F02900640064006400E0
:1061100064006400640064004D0164006400640075
:1061200064006400640064002B0064006400640088
:1061300064006400640064005E0064006400640045
:106140006400640064006400600064006400640033
:1061500064006400640064006200012300E008231E
:106160004D498A4200F02F81E069B0F5004F00F000
:10617000AF81202B00F20782202B00F25182DFE852
:1061800013F01E0224024F024F0227024F024F0259
:106190004F022C024F024F024F024F024F024F029A
:1061A0004F0231024F024F024F024F024F024F0285
:1061B0004F024F024F024F024F024F024F024F0257
:1061C0004F023D021023CBE72023C9E74023C7E756
:1061D0008023C5E73A4B5B6D03F00703052B11D80D
:1061E000DFE813F00600E10008000A000C000E00D2
:1061F0000023B5E70823B3E71023B1E72023AFE777
:106200004023ADE78023ABE72D4B5B6D03F0070325
:10621000052B0ED8DFE803F003C90507090B00239F
:106220009EE708239CE710239AE7202398E7402362
:1062300096E7802394E7224B5B6D03F00703052B61
:106240000ED8DFE803F003B40507090B002387E746
:10625000082385E7102383E7202381E740237FE796
:1062600080237DE7164B5B6D03F00703052B0ED8EB
:10627000DFE803F0039F0507090B002370E70823FD
:106280006EE710236CE720236AE7402368E780234A
:1062900066E700BFF369FFCF000C0058FFF4FF1161
:1062A000001001400044004000480040004C004005
:1062B000005000400014014000780040007C004085
:1062C000004402587D4B5B6D03F03803282B20D827
:1062D000DFE803F0151F1F1F1F1F1F1F711F1F1F48
:1062E0001F1F1F1F171F1F1F1F1F1F1F191F1F1FCC
:1062F0001F1F1F1F1B1F1F1F1F1F1F1F1D000123ED
:106300002EE708232CE710232AE7202328E7402341
:1063100026E7802324E7694B5B6D03F00703052B19
:106320000ED8DFE803F0034A0507090B002317E73F
:10633000082315E7102313E7202311E740230FE775
:1063400080230DE75D4B5B6D03F00703052B0ED833
:10635000DFE803F003350507090B002300E70823F6
:10636000FEE61023FCE62023FAE64023F8E680232D
:10637000F6E603F50E339B6D03F00703052B0ED8ED
:10638000DFE803F0031F0507090B0223E8E60823F3
:10639000E6E61023E4E62023E2E64023E0E680235D
:1063A000DEE60423DCE60423DAE60423D8E604234D
:1063B000D6E60423D4E60423D2E60423D0E604235D
:1063C000CEE60423CCE6202B27D8022BC0F01A817E
:1063D000023B1E2B00F21881DFE813F0500016017B
:1063E00056001601160116015B0016011601160172
:1063F000160116011601160160001601160116019C
:1064000016011601160116011601160116011601D4
:1064100016011601160116016C00402B2CD14FF409
:106420000040626A264B33F81220B0FBF2F3656835
:1064300005EB4501994200F2E980B3EB053F00F21C
:10644000E780002633463146FAF75AFC090241EA52
:10645000106100026B08C0182A46334641F1000162
:10646000FAF74EFCA0F54072164B9A4200F2D28029
:106470002368D8603046D4E00120D2E0FEF7DAFE8F
:106480000028CED10020CCE003A8FEF7E5FE04985A
:10649000F6E76846FEF7FAFF0198F1E7074B1B683D
:1064A00013F0200F08D0054B1B68C3F3C103064847
:1064B000D840E5E70548B4E70348B2E7004402588E
:1064C00058EC0008FFFC0F000090D00300093D00CD
:1064D000202B15D8202B00F29F80DFE803F0313706
:1064E0009D9D3A9D9D9D3F9D9D9D9D9D9D9D449DF6
:1064F0009D9D9D9D9D9D9D9D9D9D9D9D9D9D5000B6
:10650000402B1BD1626A4D4B33F81230B0FBF3F0D5
:106510006268530803EB4000B0FBF2F0A0F11002F8
:106520004FF6EF739A4279D883B223F00F03C0F38A
:10653000420018432368D860002072E0012070E018
:10654000FEF702F80028DDD100206AE0FEF70EF821
:10655000F8E703A8FEF780FE0498F3E76846FEF725
:1065600095FF0198EEE7364B1B6813F0200F08D01B
:10657000334B1B68C3F3C1033248D840E2E73248CB
:10658000C0E73048BEE7402B17D14FF40040626AA5
:106590002A4B33F81230B0FBF3F0636800EB530082
:1065A000B0FBF3F0A0F110024FF6EF739A4242D81D
:1065B000236880B2D860002033E0012031E0FDF78D
:1065C000C3FF0028E3D100202BE0FDF7CFFFF8E761
:1065D00003A8FEF741FE0498F3E76846FEF756FF6E
:1065E0000198EEE7164B1B6813F0200F08D0144BF0
:1065F0001B68C3F3C1031348D840E2E71248C6E75B
:106600001048C4E701200CE001200AE0012008E066
:10661000012006E0012004E0012002E0012000E06A
:1066200001200123A4F86A30A4F8683000236367CE
:10663000A36706B070BD0120F3E700BF58EC000867
:10664000004402580090D00300093D00836A13F013
:10665000010F06D00268536823F40033C16A0B436C
:106660005360836A13F0020F06D00268536823F464
:106670008033016B0B435360836A13F0040F06D021
:106680000268536823F48023416B0B435360836A91
:1066900013F0080F06D00268536823F40043816B9F
:1066A0000B435360836A13F0100F06D0026893689F
:1066B00023F48053C16B0B439360836A13F0200F64
:1066C00006D00268936823F40053016C0B43936077
:1066D000836A13F0400F0AD00268536823F48013D2
:1066E000416C0B435360436CB3F5801F0BD0836A3E
:1066F00013F0800F06D00268536823F40023C16CA6
:106700000B43536070470268536823F4C003816CE5
:106710000B435360EBE72DE9F84305460F46164659
:106720009946DDF820802C68E46937EA04030CBF41
:106730004FF0010C4FF0000CB44532D1B8F1FF3FDF
:10674000F1D0FCF79DFCA0EB090040452CD8B8F136
:10675000000F2BD02B681A6812F0040FE3D0DA690F
:1067600012F0080F11D1DA6912F4006FDBD04FF488
:1067700000621A622846FEF7A3FF2023C5F8903076
:10678000002385F8843003200CE008241C6228468E
:10679000FEF796FFC5F89040002385F8843001206D
:1067A00000E00020BDE8F8830320FBE70320F9E7C1
:1067B0002DE9F04182B01E46D0F88830202B5BD105
:1067C00004460D469046002A18BF002901D1012039
:1067D00053E00023C0F890302123C0F88830FCF744
:1067E0004FFC0746A4F85480A4F85680A368B3F57C
:1067F000805F02D04FF0000816E0236943B34FF0EA
:10680000000811E02023C4F88830032035E038F870
:10681000023B2268C3F308039362B4F8562092B295
:10682000013A92B2A4F85620B4F856309BB293B114
:1068300000963B46002280212046FFF76CFF00288F
:10684000E0D1002DE3D015F8012B23689A62E4E72C
:10685000A8460025E8E700963B4600224021204656
:10686000FFF759FF18B92023C4F8883005E020232A
:10687000C4F88830032000E0022002B0BDE8F081B7
:106880002DE9F04383B01E46D0F88C30202B7ED10A
:1068900004460D469046002A18BF002901D1012068
:1068A00076E00023C0F890302222C0F88C20C36626
:1068B000FCF7E6FB0746A4F85C80A4F85E80A368BA
:1068C000B3F5805F06D0A3B9226972B9FF22A4F89C
:1068D000602014E0226922B940F2FF12A4F860207F
:1068E0000DE0FF22A4F8602009E07F22A4F86020D8
:1068F00005E0B3F1805F0AD00022A4F86020B4F86C
:106900006080B3F5805F0CD04FF0000924E022696D
:106910001AB97F22A4F86020F1E73F22A4F8602092
:10692000EDE7236913B14FF0000915E0A9460025F2
:1069300012E02023C4F88C30032029E023685A6A2F
:106940005FFA88F3134005F8013BB4F85E2092B279
:10695000013A92B2A4F85E20B4F85E309BB28BB1DB
:1069600000963B46002220212046FFF7D4FE002857
:10697000DFD1002DE2D123685B6A08EA030329F81E
:10698000023BE2E72023C4F88C30002000E0022024
:1069900003B0BDE8F08330B583B004460023C0F8EF
:1069A0009030FCF76DFB05462268126812F0080F64
:1069B00010D123681B6813F0040F28D12023C4F8DA
:1069C0008830C4F88C300020E066206784F88400AA
:1069D00003B030BD6FF07E430093034600224FF4B6
:1069E00000112046FFF797FE0028E2D0226852E807
:1069F000003F23F0800342E800310029F6D1202334
:106A0000C4F88830002384F884300320E0E76FF076
:106A10007E4300932B4600224FF480012046FFF76F
:106A20007AFE0028CAD0226852E8003F23F490730F
:106A300042E800310029F6D1226802F1080353E848
:106A4000003F23F00103083242E800310029F3D16E
:106A50002023C4F88C30002384F884300320B7E767
:106A600078B310B50446D0F888300BB32423C4F8AB
:106A700088302268136823F0010313602046FFF773
:106A8000EBFA012813D0A36ABBB92268536823F438
:106A9000904353602268936823F02A03936022682E
:106AA000136843F0010313602046FFF774FF10BD25
:106AB00080F88430FCF77EF9D8E72046FFF7C6FD62
:106AC000E3E701207047000010B48165A0F85C2066
:106AD000A0F85E20002343678368B3F5805F06D08B
:106AE000A3B9036973B9FF23A0F8603014E0036908
:106AF00023B940F2FF13A0F860300DE0FF23A0F8A7
:106B0000603009E07F23A0F8603005E0B3F1805FDA
:106B10002DD00023A0F860300023C0F8903022234D
:106B2000C0F88C30016801F1080353E8003F43F0DE
:106B30000103083141E80034002CF3D1436EB3F176
:106B4000005F1ED08368B3F5805F42D0294B436756
:106B50000369002B43D0026852E8003F43F490736E
:106B600042E800310029F6D1002010BC70470369CB
:106B70001BB97F23A0F86030CEE73F23A0F8603038
:106B8000CAE7B0F868309342DCD88368B3F5805F19
:106B900019D0194B4367036943B1026852E8003FBB
:106BA00043F4807342E800310029F6D1026802F113
:106BB000080353E8003F43F08053083242E80031B5
:106BC0000029F3D1D0E70369002BE2D10B4B4367D7
:106BD000E1E70369002BB9D1094B4367B8E70268C5
:106BE00052E8003F43F0200342E800310029F6D18B
:106BF000BAE700BF115B0008C55C0008915E0008A1
:106C0000ED5B000838B5D0F88C30202B19D1002A64
:106C100018BF002917D00023C36603680B4CA3429A
:106C20000CD05B6813F4000F08D0046854E8003FF0
:106C300043F0806344E80035002DF6D1FFF744FFB0
:106C400000E0022038BD0120FCE700BF000C005826
:106C5000436E2BB90123A0F86A30A0F86830704762
:106C600030B403689A68C2F342629968490F094DCB
:106C70006B5C1B01084C615C93FBF1F3A0F86A307C
:106C8000AB5C1B01A25C93FBF2F3A0F8683030BC54
:106C9000704700BF78EC000870EC00087047704740
:106CA000704790F88430012B18D0012380F884308D
:106CB0002423C0F8883003681A68196821F001019C
:106CC000196022F000520023436601680A60202206
:106CD000C0F8882080F8843018467047022070473A
:106CE00038B590F88430012B1DD00446012380F87C
:106CF00084302423C0F8883003681D681A6822F0A5
:106D000001021A600268936823F06043194391609E
:106D1000FFF79EFF23681D602023C4F88830002001
:106D200084F8840038BD0220FCE738B590F8843040
:106D3000012B1DD00446012380F884302423C0F8A1
:106D4000883003681D681A6822F001021A60026820
:106D5000936823F0606319439160FFF779FF23681C
:106D60001D602023C4F88830002084F8840038BDDA
:106D70000220FCE7014B1868704700BF2000002488
:106D800070B50D4E0D4D761BB61006D0002455F88B
:106D9000043B01349847A642F9D1094E094D761BB0
:106DA00007F050FEB61006D0002455F8043B01341D
:106DB0009847A642F9D170BD7CF200087CF2000829
:106DC00084F200087CF20008024B0146186800F0CB
:106DD0000BB800BF20000024024B0146186804F0E5
:106DE00085BE00BF200000242DE9F04F01F10B0605
:106DF000162E83B0044624D8102900F2BA8000F081
:106E0000F5FA102618220220B54F3A44A2F10801E3
:106E100053688B4200F0BA805A68D96822F00302A6
:106E20001A449D68E9608D60516841F00101204677
:106E3000516003F1080500F0DFFA284603B0BDE811
:106E4000F08F36F0070600F19480B14200F2918095
:106E500000F0CCFAB6F5FC7FC0F09A81730A00F01E
:106E60008F80042B00F26F81B30903F1390003F125
:106E7000380CC3009A4F3B44A3F108055B689D4260
:106E800006D10CE0002980F22781DB689D4206D004
:106E90005A6822F00302911B0F29F3DD60463D6919
:106EA000DFF840C265457CD06A6822F00302931B7C
:106EB0000F2B00F37B81002BC7E904CC80F26C819F
:106EC000B2F5007F80F01A81D308796801334FEA68
:106ED000521E012202FA0EF20A4357F833E0C5F8B7
:106EE00008E007EBC3010839E9607A6047F83350DE
:106EF000CEF80C50831001219940914257D811428D
:106F000006D120F003004900114200F10400FAD03C
:106F100007EBC0094D468646D5F80C80454508D19B
:106F20001DE1002B80F22481D8F80C80454500F04B
:106F30001681D8F8042022F00302931B0F2BF0DDFA
:106F40002046D8E9025408EB060146F00106C8F8CD
:106F50000460EC60A56043F00104C7E90411C1E9D5
:106F600002CC4C6048F8023000F046FA08F10805FF
:106F700002E00C2323600025284603B0BDE8F08F13
:106F80004FF4007340204FF03F0C73E7D3689A42F0
:106F900008BF02307FF440AF3D69DFF848C1654566
:106FA00082D17A688310012199409142A7D9BD68A6
:106FB0006B6823F003094E4503D8A9EB06030F2B9A
:106FC0007ADCDFF824B1494BDBF800201B68013282
:106FD000334405EB090A00F0338103F580530F3386
:106FE00023F47F6828F00F084146204600F06CFC2F
:106FF000411C024600F0F380824500F2EE803C4BDB
:10700000196841441960084600F04E81DBF8001011
:10701000019301311BBFA2EB0A0A5044CBF80020B8
:10702000186012F0070B00F01781CBF108010A4439
:10703000CBF5805190440831A1EB0801C1F30B0A54
:1070400051462046009200F03FFC421CDDE900233F
:1070500000F04F81801A00EB0A081968BA6048F006
:1070600001005144BD425060196000F02981B9F11E
:107070000F0F40F227816868A9F10C0C2CF0070C67
:1070800000F0010040EA0C0068604FF0050E05EBCF
:107090000C00BCF10F0FC0E901EE00F23281506824
:1070A0001546144B1A688A4238BF1960124B1A6889
:1070B0008A4238BF196094E0AA1943F0010346F0F0
:1070C00001066E602046BA60536000F095F90835FD
:1070D000284603B0BDE8F08FD9681A44A1E600BF86
:1070E000500400245804002458080024400D0024B3
:1070F000100D0024380D00243C0D0024B2F5206F43
:107100004FEA522363D3142B00F2B78003F15C01E2
:10711000C9005B3307EB010E7958AEF1080E8E45BE
:1071200000F091804B6823F00303934202D98968F1
:107130008E45F7D1D1F80CE07A68C5E9021ECEF889
:107140000850CD60D6E6142B59D9542B00F29D80FF
:10715000330B03F16F0003F16E0CC3008AE60EF1EE
:10716000010E1EF0030F05F108057FF4D5AE51E0C6
:10717000424445465368D8F80C1043F0010353606D
:1071800055F8083F2046D9608B6000F035F9F3E6EA
:10719000F00806F1080237E62A442046536843F017
:1071A00001035360083500F027F9E5E6A9192046E8
:1071B00046F0010643F001046E60C7E90411C1E91D
:1071C00002CC4C60AB5000F017F90835D4E69309B7
:1071D00003F13901C90038339CE7BD425FD0BD6877
:1071E000686820F003084645A8EB060302D80F2B79
:1071F0003FF762AF204600F0FFF80025BCE603F140
:107200005C0003F15B0CC30034E659F808394B45C8
:1072100040F0968010F0030F00F1FF30F5D17B684D
:1072200023EA01037B60490099423FF6C0AE19B9D9
:10723000BDE649000EF1040E1942FAD0704667E629
:1072400003F11008D0E69A104FF001087B6808FAA5
:1072500002F21A437A6070E702EB08014942C1F377
:107260000B0A51462046009200F02EFB431CDDE93C
:1072700000237FF4EFAEDA46EFE6542B25D8130B4C
:1072800003F16F01C9006E3344E7B3F5AA7F25D837
:10729000F30B03F1780003F1770CC300EAE5294B07
:1072A000186840441860B1E6CAF30B0CBCF1000F3B
:1072B0007FF4ACAEBD68C84448F001006860F0E6F9
:1072C0001546EEE60123536094E7B3F5AA7F23D871
:1072D000D30B03F17801C90077331BE740F2545216
:1072E000934223D8B30C03F17D0003F17C0CC3005F
:1072F000C0E5ABF1080BD844A8EB02084FF0000A38
:10730000ABE605F108012046009304F0EFFBBD68F1
:10731000009B68681968C4E640F254518B420BD850
:10732000930C03F17D01C9007C33F3E64FF47E73C7
:107330007F204FF07E0C9DE54FF47E717E23E9E6C1
:107340007B6870E7100D0024830730B548D0541EC9
:10735000002A3FD0CAB2034601E0013C3AD303F809
:10736000012B9D07F9D1032C2DD9CDB245EA052576
:107370000F2C45EA054536D9A4F1100222F00F0C76
:1073800003F1200EE6444FEA121C03F1100242E919
:10739000045542E9025510327245F8D10CF1010250
:1073A00014F00C0F03EB021204F00F0C13D0ACF12D
:1073B000040323F003030433134442F8045B9342B1
:1073C000FBD10CF003042CB1CAB21C4403F8012B0E
:1073D0009C42FBD130BD64461346002CF4D1F9E742
:1073E00003461446BFE71A46A446E0E7014805F005
:1073F00049BA00BF480D0024014805F045BA00BF56
:10740000480D00240FB400B5074983B004AB0868E9
:1074100053F8042B8168019301F06CFB03B05DF815
:1074200004EB04B0704700BF2000002470B505468F
:1074300088B008460C46FAF703F8224EAA6B05906E
:1074400001214318CDE9066104A8022104940393A5
:10745000AC680190029122B3636E13F0010FB4F98E
:107460000C309AB201D1980525D5910406D4626EEC
:1074700043F4005322F40052A3816266284601AA15
:10748000214604F039FC636E002814BF4FF0FF352D
:107490000A25DA0702D4A3899B0506D5284608B039
:1074A00070BD284604F02AFAD6E7A06D05F0ECF985
:1074B000284608B070BDA06D05F0E4F9B4F90C30B1
:1074C0009AB2D2E714EB0008024B01461868FFF7A6
:1074D000ADBF00BF2000002410B4044C03460A4690
:1074E000206810BC194600F003B800BF200000243B
:1074F0002DE9F84F1746002900F0988007F10B0599
:1075000080460C46FFF772FF162D5DD810252A46DF
:10751000AF425ED854F8041C21F003069642A4F151
:10752000080962DABC4BD3F808C009EB06008445B1
:1075300000F09780D0F804C02CF0010303445B688E
:10754000DB0768D42CF0030C06EB0C03934247DAFC
:10755000CB0710D454F8083CA9EB030ADAF804303E
:1075600023F003018C44B444944580F211817318D4
:10757000934280F2E88039464046FFF735FC0746E3
:10758000E0B154F8043C23F001034B44A0F108029D
:10759000934200F0D280321F242A00F2F580132A91
:1075A00000F2AC80034622461168196051685960A8
:1075B00092689A602146404604F098FA4046FFF7E8
:1075C0001BFF3846BDE8F88F25F00705002D2A4639
:1075D0009EDA0C23C8F8003000273846BDE8F88F43
:1075E0001E46D0E90223D3609A60731B0F2B22D86A
:1075F000D9F8043003F0010333434E44C9F8043092
:10760000736843F00103736040462746FFF7F4FEBA
:107610003846BDE8F88FC907ADD454F8083CA9EB4B
:10762000030ADAF8041021F00301A0E7BDE8F84FDF
:107630001146FFF7D9BBD9F8041001F00101294325
:10764000C9F8041009EB05014E4443F001034B60F7
:10765000736843F0010308317360404604F046FA52
:10766000D2E7DCF8040020F0030B06EB0B0C05F16D
:10767000100084454DDAC9073FF57DAF54F8081C6A
:10768000A9EB010ADAF8041021F003018B44B3449A
:1076900058453FF76CAF5746DAF80C1057F8080F0B
:1076A000321F242AC160886000F2DB80132A40F276
:1076B000D6802168CAF808106168CAF80C101B2A25
:1076C00000F2DF8008340AF110022168116061685D
:1076D0005160A16891600AEB0501ABEB050242F035
:1076E000010299604A60DAF8043003F001031D4397
:1076F0004046CAF80450FFF77FFE6EE72368036038
:10770000636843601B2A68D804F1080200F108038B
:107710004AE709EB05029A60ACEB050343F001036D
:10772000536054F8043C03F001031D43404644F801
:10773000045CFFF761FE27464FE750F8043C23F056
:1077400003031E4451E75746DAF80C1057F8080FA8
:10775000321F242AC16088604CD8132A48D9216876
:10776000CAF808106168CAF80C101B2A56D80834E9
:107770000AF110021E462368136063685360A36811
:107780009360D1463C4630E7214605F04BF911E7BE
:10779000D0E902135746CB60996057F8081FDAF812
:1077A0000C30CB60321F242A99602DD8132A29D996
:1077B0002368CAF808306368CAF80C301B2A42D81C
:1077C00008340AF1100322681A6062685A60A268DD
:1077D0009A606646D1463C4607E7A3688360E36843
:1077E000C360242A26D004F1100200F11003DBE666
:1077F0003A46BFE7214638461E46D14605F012F903
:107800003C46F2E63B46DEE7214638466646D14630
:1078100005F008F93C46E8E650040024A168CAF8DF
:107820001010E168CAF81410242A20D010340AF18C
:1078300018029FE7236903616169416104F118023D
:1078400000F11803B0E6A368CAF81030E368CAF87C
:107850001430242A21D010340AF11803B3E73A4631
:1078600033E72146384605F0DDF8164B33E7226949
:10787000CAF818206269CAF81C2018340AF12002DC
:1078800078E7A168CAF81010E168CAF81410242A31
:107890000DD010340AF1180217E72369CAF818301E
:1078A0006369CAF81C3018340AF120038BE7226997
:1078B000CAF818206269CAF81C2018340AF120029C
:1078C00003E700BF5004002438B5074D00220446EA
:1078D00008462A60FBF774F9431C00D038BD2B68BA
:1078E000002BFBD0236038BD540D00242DE9F0435C
:1078F000694CD4F8008083B004460E4617461D46F6
:10790000B8F1000F03D0D8F83830002B77D0022F11
:1079100005D0012F00F2AC80002DC0F2A980636E6B
:10792000DA0752D52146404603F0B4FF216B41B13E
:1079300004F14003994202D0404604F0D7F80023F6
:107940002363B4F90CC000231CF0800FA3616360B3
:1079500064D12CF44A6C2CF0030C022FA4F80CC058
:107960006AD001AB6A462146404605F015F8A38966
:107970001843A081002D2FD0002E2ED0D8F83830FB
:10798000002B38D0009B2660AB42B4F90C301CBFF2
:1079900043F40063A381012F04BF43F00103A381DB
:1079A0009AB213F00803C4E904652CD0D1075DD561
:1079B0006D42A561656E002315F00105A36027D017
:1079C0000025284603B0BDE8F083A3899B05A9D410
:1079D000A06D04F057FFA5E7009D2846FFF7F4F9D6
:1079E0000646002847D0A38943F08003A381D8F836
:1079F0003830002BC6D1404603F080FFC2E7404636
:107A000003F07CFF83E7A360656E15F00105D7D115
:107A1000930524D5284603B0BDE8F083216940468C
:107A200004F064F8B4F90CC02CF44A6C2CF0030C8C
:107A3000022FA4F80CC094D10025002204F14303C6
:107A4000A2600122C4E904322360636E4CF0020C90
:107A5000D807A4F80CC0DDD41CF4007FDAD1A06DE7
:107A600004F012FF284603B0BDE8F083A560CBE721
:107A70004FF0FF35CEE7DDF80090A94504D0484629
:107A8000FFF7A2F9064620B9B4F90CC04FF0FF3554
:107A9000D3E74D46A7E700BF2000002410B50C46F1
:107AA000B1F90E1005F054FD002803DB236D0344EB
:107AB000236510BDA38923F48053A38110BD00BFAB
:107AC0002DE9F0410C46B1F90C101F46CB050546D7
:107AD00016460BD421F48051A1813B46B4F90E1017
:107AE00032462846BDE8F04102F0AEBDB4F90E10B2
:107AF0000223002204F0CAFEB4F90C10EAE700BF2A
:107B000010B50C46B1F90E1004F0C0FEA389421C5A
:107B10000EBF23F4805343F480532065A38110BD2E
:107B2000B1F90E1002F020BEA2B330B540EA010454
:107B3000A40784460B462AD09CF800000C788442A7
:107B40002FD1012A0DD0E64660B11EF8010F11F8C1
:107B5000014F6FEA0E03A042134422D11CEB030332
:107B6000F2D1002030BD0468194653F8045BA4F13B
:107B7000013EAC4284462EEA040E00F104000BD113
:107B8000043A84461946ECD01EF0803FE9D1032A1E
:107B9000E9D8D1E7104670479CF800000C78A04265
:107BA000D1D0001B30BD00BF2DE9F04F1C46984BD3
:107BB0001B68A1B0002581461846884608921C958E
:107BC0000493F9F73DFC002183460020CDE906012E
:107BD000CDF86C804246174612F8013B2D2B2FD86A
:107BE000DFE813F0A1002E002E002E002E002E0044
:107BF0002E002E002E00AF00AF00AF00AF00AF0090
:107C00002E002E002E002E002E002E002E002E0004
:107C10002E002E002E002E002E002E002E002E00F4
:107C20002E002E00AF002E002E002E002E002E0063
:107C30002E002E002E002E002E0006042E00FC0327
:107C400000220A92302B7ED0002209922F2B1C4654
:107C500040F233854FF0000A38465646554612E04A
:107C60000130082D1B90C8BF0AEB8A0A0478C6BFF2
:107C700003EB4A03A3F1300AA2F130062F2C05F1E1
:107C80000105234670DD06EB8602392C03EB420228
:107C9000E6DD04995A46FFF747FF0346002835D131
:107CA0001B9A11465A441B9211F80B40002D40F0CC
:107CB000AC85302C40F06485C2F1010153180132CB
:107CC0001B921478302CF9D0A4F13102082A00F26A
:107CD0003883A4F1300E1B9C03F1010B0023012516
:107CE0002746049306EB86060EEB46060023621C2D
:107CF0001B926478A4F13001092900F2ED8201336E
:107D00008E46002940F0B8841B9CF0E70023652CC8
:107D100004959B469E4601D0452C32D1002D7CD146
:107D2000099A1A4378D1089B13B1089BC3F80080C5
:107D30004FF0000BCDF810B00499584621B0BDE8C3
:107D4000F08F1B9247E77B7803F0DF03582B00F09E
:107D5000748401371B973B78302BFAD0002B00F04E
:107D6000CC800122099271E704995A46FFF7DCFEA4
:107D70000346002800F0D68004954FF0000B5B46C8
:107D8000DE4600220B92002D00F09380049A1346E9
:107D9000002A08BF2B4630460493F8F7F3FB0B4646
:107DA0000246CDE906230B9B102DA3EB0B032C46BB
:107DB000A8BF1024092D0E9313DD164B03EBC4034B
:107DC00053E91223F9F7FCFBCDE906015046F8F719
:107DD000D9FB02460B46DDE90601F8F797FACDE933
:107DE00006010F2D00F3A7800E9B002B00F01884D6
:107DF0000E9B40F39283162B40F3F9840E9AC5F143
:107E00002503934280F20C850E9B2C1B1C4498E0AA
:107E10007CF0000840F100080025DDF86C8008F1D6
:107E200001021B9298F801402B2C00F087822D2C28
:107E300000F0218200220E92A4F13002092A00F201
:107E40001582302C05D11B9A01321B921478302CEC
:107E5000FAD0A4F13102082A93D81B990B914A1C3D
:107E60001B92A4F130004C782F2C09DC00F034BCBC
:107E700001321B929CF801402F2CA1F1300006DD4D
:107E800000EB8001392C944604EB4101F0DD0B99A5
:107E9000521A082A40F3208444F61F620B920E9A6D
:107EA000002A3FF470AF0B9A52420B92002D7FF4E0
:107EB0006DAF099A134320D1BEF1000F7FF433AFA9
:107EC000692C00F03B8400F34183492C00F0368498
:107ED0004E2C7FF428AFAC491BA804F0D5FB00283A
:107EE0003FF421AF1B9B1B78282B00F06D85A74822
:107EF00005F07CFB8346049103E04FF0000BCDF8C6
:107F000010B0089A0AB11B9B13600A9B002B3FF428
:107F100013AF049901F1004304930499584621B02A
:107F2000BDE8F08F1B9A049502EB0B011B9112F830
:107F30000B409B46DEE60E9B2C1B1C44002C40F3A2
:107F40000A8314F00F000AD0914901EBC001DDE96A
:107F50000623D1E90001F9F733FBCDE9060134F03E
:107F60000F0340F08B8200230993049A00962B465E
:107F70003946484604F052FE1390002800F055831D
:107F80000B9BABEB03000E9B002BB4BF0246002201
:107F90000F9223EAE3730022934612939046139CB8
:107FA0004846616804F0BAFD0746002800F04181A8
:107FB00022690232920004F10C010C30F9F722F828
:107FC000DDE9060104910B461EA901911DA90B9044
:107FD00002460091484605F0CDF91C90002800F0BB
:107FE00018810121484604F0C1FE8046002800F0B7
:107FF00020811D9B002BC0F20F810F9A129D9E18AD
:10800000099A1E9C9B1A2344624A013B9342C4F185
:10801000360480F2AE80D21A1F2AA4EB020400F3C9
:108020001D814FF0010A00230AFA02FA0C93099B02
:1080300025443444A6421D443346A8BF2346AB42E0
:10804000A8BF2B46002B02DDE41AED1AF61A0F9B8F
:10805000002B00F3BE80002C00F3D2800E9B002B7F
:1080600000F3DE80002D00F3EF80002E08DD414696
:108070003246484604F0B6FF8046002800F0D9801A
:108080001C993A46484605F045F88346002800F01A
:10809000D0800026C368C6604146109305F01AF8E8
:1080A000B042C0F2638400F0D2834146584605F0E6
:1080B000C3F900224FF0804304460D46F8F746FB13
:1080C00000286FD0109B002B00F0E180079B1193DC
:1080D000314B314C0022CDE90C2335462F4E119AFD
:1080E0002F4B02EA060A9A4500F0FC80099B93B1E7
:1080F000BAF1D46F0FD822A3D3E900232846214632
:10810000F8F724FB002840F087810D9B03F1D6632C
:10811000A3EB0A030D93049E0B98DDE90C23314673
:10812000CDE9042305F09CF802460B46DDE9040185
:10813000F9F746FA33460B9AF8F7E8F8CDE9060165
:108140000E46099B23B9154B33409A4500F0028136
:108150001C99484604F008FD3946484604F004FDE1
:108160004146484604F000FD5946484604F0FCFCF0
:1081700015E700230C934FF0010A58E7AFF3008096
:108180000000C0FFFFFFDF4194ED000888EB00080E
:1081900040F1000802FCFFFF0000F03F0000F07F0C
:1081A0000000E07FAE4B204629460022F9F708FA8E
:1081B000109B024605460C46002B64D101F100439A
:1081C00014901593079B1193DDE91423CDE90C233B
:1081D00084E741461A46484604F0A4FE804640B370
:1081E00001461C9A484604F0EFFD10B310901C990C
:1081F000484604F0B9FC109B1C93002C7FF72EAF6F
:108200001C992246484604F0EDFE1C9000287FF49D
:1082100025AFBA465E460FE0129A0F9ED51AEFE6DA
:108220003946129A484604F07DFE074600287FF43E
:1082300019AFBA465E461C982223C9F80030894B14
:1082400004934FF0000BB4E039462A46484604F048
:10825000C9FE074600287FF408AFEAE7824A4FF0DC
:10826000010AD31A0AFA03F30C93E0E60022CDF8D0
:108270006C800B9287E501220E9208F102021B929C
:1082800098F80240D8E50B46CDE914239AE7DDE9DA
:108290000612002940F0AF80C2F313031192002BA5
:1082A00040F0AF80714B002220462946F8F744FA8F
:1082B000002840F0AE826A4B204629460022F9F79A
:1082C0007FF901F1004305460C4618901993DDE94A
:1082D0001823CDE90C2301E7652C4FF0010E3FF484
:1082E0009CAD19E5A2F154730793DDE90623DDE99E
:1082F0000C01CDE9060110461946CDE90C2304F026
:10830000AFFF02460B46DDE90601F9F759F9DDE951
:108310000C23F7F7FBFF564A0E409642CDE90601C3
:1083200076D9049A534B9A4202D10B9B013380D0E9
:10833000504A4FF0FF33CDE9063209E700220E9292
:108340009BE7652C00F0FB80452C00F0F8804FF097
:10835000010EAEE528462146F9F764FBF8F75EF911
:108360000B46024621462846F7F7CEFF109C069D95
:10837000C6F3130644EA050C5CEA060304460D4600
:1083800000F0C28032A3D3E90023F8F7D5F948B949
:1083900031A3D3E9002320462946F8F7EBF900285A
:1083A0003FF4D6AEDDE906341C9804945E46BA4626
:1083B0009B460146484604F0D7FB5146484604F028
:1083C000D3FB4146484604F0CFFB1399484604F0DE
:1083D000CBFB3146484604F0C7FB92E501230A93E4
:1083E0007A1C1B927B78002B3FF49DAC174629E446
:1083F00000230A93F4E7DDE90612012900F07481F5
:1084000011921D4B194C0022CDE90C23002565E685
:1084100001F15476079694E621462846F9F7E2FAE8
:10842000012838BF0120F8F7ADF8109B0246054639
:108430000C46002B40F0698101F100431690179320
:10844000DDE91623CDE90C235FE600BFAFF3008022
:108450009535A094FFFFDF3F35E5AF350000E03FE5
:108460000000E03F0000F07FE2FBFFFF0000F03F74
:10847000FFFF9F7CFFFFEF7F0000F0BFB3F59A7F07
:1084800000F3D380102B4FEA2314A54B40F3C68290
:10849000DDE906019846099300239A4614F0010F7E
:1084A0000AF1010A4FEA640404D0D8E90023F9F77D
:1084B00087F80123012C08F10808EFD10BB1CDE9B1
:1084C0000601099B03EBCA01079BA3F154730793B1
:1084D000DDE90623D1E90001F9F772F8914BCDE906
:1084E00006010B400A4690498B4200F29E80A1F59E
:1084F00080118B4240F21C828C494FF0FF33CDE952
:1085000006310023099330E583A3D3E90023F8F76C
:1085100013F900283FF41CAE44E71633FFF60BAD09
:108520000B9BABEB0302824B03EBC203DDE90601BD
:10853000D3E90023F9F76EF983460491E1E40022C0
:10854000049293464FF0010EFFF7EABB6E2C3FF406
:10855000C2ACFFF7E8BB3FF406AD644214F00F0273
:108560000AD0734B03EBC203DDE90601D3E9002314
:10857000F9F750F9CDE9060124113FF4F4AC1F2CB2
:1085800035DC14F01003DDE9060118BF6A23DFF8BB
:10859000A48109930023E20704D5D8E90023F9F761
:1085A0000FF80123641008F10808F4D10BB1CDE9EC
:1085B0000601099B93B1DDE90601C1F30A52C2F13C
:1085C0006B03002B0ADD1F2B40F350820020342B5D
:1085D000069040F356824FF05C730793DDE9060185
:1085E00000220023F8F79EF800283FF4BEAC2223B7
:1085F0004FF0000BC9F80030CDF810B081E41E9B9D
:1086000006931D9B03F233421F9B23F4801343EA1E
:1086100002530793200742BF079B43F00043079391
:10862000DDE906349B4604946BE43E4A049222231F
:10863000C9F800304FF0000B63E40A9B01931CABB8
:10864000029400933C4A1DAB1BA9484603F03EFD33
:1086500010F0070504463FF450AC062D40F093801F
:10866000089B0137002B3FF463AB4FF0000B1F60FA
:10867000CDF810B0FFF760BB6A1C012B1B9C9B441C
:10868000104615D02B4403F1FF3C03E0460094450F
:108690000DD001322B46082B154606EB8600F5D986
:1086A000102ADCBF0AEB8A0A4FEA4A0AEFE7981C55
:1086B000082D5BDC0546FFF715BB04995A46384682
:1086C000FFF732FA002800F0888000231D4604934B
:1086D0009A461E46FFF751BB44F61F629042A8BF60
:1086E00010460B90FFF7DBBBDDE906341194002C3C
:1086F0007FF487AEBA465E4622234FF0000B1C98EB
:10870000C9F80030CDF810B053E60B46CDE916237A
:1087100096E600BFAFF300809535A094FFFFCF3FF2
:1087200018F100080000F07F0000A07CFFFFEF7F41
:1087300040F10008C0ED000898ED0008AD491BA805
:1087400003F0A2FF00283FF4EEAA1B9BAA49013BBD
:108750001BA81B9303F098FF10B91B9B01331B93BD
:10876000A64B04934FF0000BFFF7CBBB1028DCBFE8
:108770000AEB8A0A01EB4A0A05460023FFF7B7BA5B
:108780000023FFF7A1BA1C9A3AB135211EA804F0C4
:1087900081FE1C99484604F0E7F9013D042D3FF69F
:1087A00039AF01A353F825F0FF850008D1870008F1
:1087B000CB870008BD870008FF8500084FF0FF3316
:1087C0006FF00045CDE9063524E78C4B079321E790
:1087D0001E9B06931F9B07931CE71B9A13465A4444
:1087E0001B9213F80B4006468246FFF762BA0E98BA
:1087F000834901EBC001DDE90623D1E90001F8F767
:10880000DFFE83460491FFF77CBB04958346FFF7A8
:1088100071BA7C4B7C4C109D0022CDE9182356E5A3
:10882000774CC5F10F0504EBC501DDE90623D1E95D
:108830000001F8F7C5FE0E9B5D1B04EBC504D4E9EF
:108840000023F8F7BDFE83460491FFF75ABB109B47
:108850005E46D446BA46DDE90BB7002B6FD0DDE9A2
:1088600006456A4BC5F3130199422A463CD0002FB6
:1088700000F0A380DDE906231F421C4621D0109B97
:1088800004995846002B00F0CD8004F0E9FC099DC6
:1088900002460B467DB1C4F30A54C4F16B04002CAC
:1088A00009DD240504F17F53002203F54013F8F796
:1088B00087FE02460B4604995846F7F727FD834684
:1088C0000491099B73B10499514B58460022F8F763
:1088D00077FE03460B4308BF22238346049108BF5B
:1088E000C9F800301C9864E5099B0699002B00F03C
:1088F000C580424B2B40B3F1D46F00F2BF801B0DFB
:10890000C3F16B034FF0FF3000FA03F39942AED18D
:10891000404B9A4200F0D880384B134003F5801347
:10892000079300230693DDE906349B460494C8E7C9
:1089300002F15473079300230993FFF716BBDDE997
:108940000612C2F313030B43144690D1099B002B6C
:1089500040F0AF80294B2340A3F580136FEA1353F7
:108960006FEA035307934FF0FF33DBE7DDE90612AD
:10897000109B0B4358465E46BA46DDF82CB0A0D19A
:10898000C2F313031446002B9BD122F000431B0DAE
:108990001B05B3F1D66F94D9436913B90369012B51
:1089A0008FDD31460122484604F01CFB4146064655
:1089B00004F090FB002884DDC8E7DDE906341CEAFA
:1089C000030F3FF47EAF5AE713491BA81EAA03F01A
:1089D00075FE05287FF48BAA1F9B43F0FF4343F4E9
:1089E000E00307931E9B0693DDE906349B4604943F
:1089F000FFF787BA88ED00088CED00080000F07FD3
:108A000040F100080000E0BF0000E03FFFFF0F0062
:108A100000005039FFFFEF7FACED000809934FF0E5
:108A2000000A4EE504F01CFC099D02460B4695B376
:108A3000C4F30A54C4F16B04002C09DD240504F1CD
:108A40007F53109A03F54013F8F7BAFD02460B4620
:108A500004995846F7F758FC0022002383460491F6
:108A6000F7F760FE00283FF42EAF45E64FF0FF32E7
:108A700002FA03F3069A1A400692AFE54FF0FF336D
:108A800044E74FF0FF33C2F14B0203FA02F202EA6D
:108A900001030793A2E504995846F7F735FC002235
:108AA000002383460491F7F73DFE00283FF41AAFF8
:108AB00022E6084B2340B3F1D66F3FF74DAFB3F139
:108AC0005C7F3FF700AF17E601317FF425AFFFF77A
:108AD000B2BB00BF0000F07F10B4044C044B8446CE
:108AE0000A46206810BC6146FFF75EB820000024EB
:108AF000680800242DE9F04FD5B01C460791914637
:108B00000546099003F0B6FE0268179210460E94CF
:108B1000F8F796FC16901DB1AB6B002B00F02A8283
:108B2000079A536EDD0740F13881B2F90C2091B2FB
:108B30008F0409D4079B42F400529A8191B21A46DD
:108B40005B6E23F4005353660E0740F1CB80079B06
:108B50001B69002B00F0C68001F01A030A2B00F0FD
:108B6000CF8000242BAB4D46CDE92944CDE91944F3
:108B7000CDE91B44129428939846189400230B9433
:108B80000024CDE914342B78002B00F09D81AA46F7
:108B900004E01AF8013F002B00F0C780252BF8D124
:108BA000BAEB050640F0C5809AF80030002B00F0C3
:108BB0008B8100234FF0FF329AF801608DF88330EB
:108BC0000A930AF1010A08921F462B244FF020094C
:108BD0000AF1010AA6F120035A2B00F2ED80DFE82A
:108BE00013F0EB02EB00EB00E602EB00EB00EB0016
:108BF0006A00EB00EB005C028002EB0067028A0275
:108C0000EB0085025B005B005B005B005B005B00D0
:108C10005B005B005B00EB00EB00EB00EB00EB00AC
:108C2000EB00EB007A01EB00F801D2017A017A0146
:108C30007A01EB00EB00EB00EB00E102EB00EB0054
:108C40002D02EB00EB00EB000202EB00A402EB00B4
:108C5000EB008307EB00EB00EB00EB00EB00EB001D
:108C6000EB00EB007A01EB00F801D4017A017A0104
:108C70007A01C702D401CD01EB00D402EB006C02F3
:108C80002F02B502CD01EB0002027E008007EB004F
:108C9000EB006107EB007E00A6F1300300221AF81A
:108CA000016B02EB820203EB4202A6F13003092BB7
:108CB000F5D90A928EE7DDF824B0584603F0DAFDC4
:108CC00043681B931846F8F7BBFB1C9006465846B2
:108CD00003F0D0FD83681993002E40F0CD869AF8FA
:108CE000006075E7079D0998294601F0C3FC00283C
:108CF00041F01C83A98901F01A030A2B7FF431AFDC
:108D0000079AB2F90E30002BFFF62BAF536ED8073F
:108D100002D4890541F13B810799099823464A46C7
:108D200055B0BDE8F04F01F04FBCBAEB050600F0BE
:108D3000CB802A9B33442A93299B0133072BC8E914
:108D40000056299305DC08F108080B9B33440B936C
:108D50002AE70799099828AA04F0BCFC80B90DF10C
:108D6000AC08F2E70799099828AA04F0B3FC002898
:108D700000F09B800D9B1BB10998194602F0B6FECE
:108D8000079A536ED90740F1EA8093895B0601F197
:108D9000D9820B9855B0BDE8F08F079BB3F90C2032
:108DA000900591B23FF5C4AE1D46986D03F06AFD83
:108DB000B5F90C2091B2BBE6002E00F085800022B0
:108DC0008DF8EC608DF883200123CDE90C320693F9
:108DD00008920F92139210923BAD17F0020302D04B
:108DE00006990231069117F0840B07D10A9906986B
:108DF000A1EB0009B9F1000F00F370832A9C8AB13E
:108E0000299A0DF1830101320134C8F80010072AB4
:108E10004FF001012A942992C8F8041000F3B68398
:108E200008F1080883B1299B21AA01330234C8F84C
:108E30000020072B4FF002022A942993C8F804203F
:108E400000F3B28308F10808BBF1800F00F06982DB
:108E5000089B0C9AA3EB020BBBF1000F00F3AA8254
:108E6000FB0500F100820C9BC8F804301C44299BD0
:108E7000C8F800500133072B2A94299300F322836A
:108E800008F10808780705D50A9B069A9D1A002D57
:108E900000F39683DDE90A2306998A42ACBF9B184A
:108EA0005B180B93002C7FF45DAF002329930D9B7F
:108EB0001BB10D99099802F019FE0DF1AC08554649
:108EC0002B78002B7FF463AE2A9B002B41F0D381DB
:108ED0000023299354E70E9B073323F00702F2E89F
:108EE0000234CDE91434DDE9143424F000440E9248
:108EF000994618462146B54B4FF0FF32F7F744FC30
:108F0000002840F0EF84B14B484621464FF0FF3235
:108F1000F7F71CFC002840F0E584DDE9140100228D
:108F20000023F7F709FC002840F067879DF88320AD
:108F3000A74DA84B27F080070321472EC8BF1D4629
:108F400000230D9306910C9108930F9313931093A4
:108F5000002A3FF442AF069B013306933DE7079B8F
:108F60009B899A053FF512AF079CA06D03F08CFC1E
:108F7000A3890BE7099802F0C1FCD1E59AF80060DB
:108F800047F0200724E647F01007BA060E9B40F191
:108F90003B84073323F007031A465B6852F8084BFB
:108FA0000E929946002BC0F24C84089B013300F0CE
:108FB000D88254EA090327F0800B40F0D382089B43
:108FC000002B40F0D4825F46002308930C9354ADED
:108FD0001DE10E9B002253F8041B8DF883208DF8B1
:108FE000EC100E93F0E60E9C089B54F8045B4FF0D7
:108FF00000098DF88390002D00F093855A1C00F035
:1090000051861A4649462846F8F78AFA0D900028F4
:1090100001F00E810D9BCDF820905B1B0C930E94FC
:1090200023EAE3739DF883200693CDF83490CDF8BE
:109030003C90CDF84C90CDF8409089E747F0100770
:1090400017F0200900F0D2830E9B073323F00703AB
:10905000D3F8049053F8084B0E9327F4806B002349
:1090600000228DF88320089A511C00F0B88054EA41
:1090700009012BF0800740F0B180002A40F0F6850E
:10908000002BA1D11BF001030C9300F014843023BA
:109090008DF84F310DF24F15B9E00E9B53F8042BAC
:1090A0000A92002A80F2DA830A9A0E9352420A92B6
:1090B0009AF8006047F004078AE5BD0600F1D18404
:1090C000FC0600F1D885780600F1A586B90540F1C7
:1090D000D2850E9B0B9953F8042B0E9311705546B5
:1090E000EEE69AF800608DF8834071E59AF800602A
:1090F00047F080076CE5524612F8016B2A2E01F00A
:109100003F82A6F13003092B924698BF002201F25C
:10911000BC801AF8016B02EB820203EB4202A6F15B
:109120003003092BF5D9089254E547F0100B1BF0DA
:10913000200900F076830E9B073323F00703D3F852
:10914000049053F8084B0E93012389E70E9B53F8C4
:10915000044B0E93302378268DF884301E4B1893E1
:1091600047F0020B8DF885604FF00009022377E786
:109170009AF80060682E03BF9AF8016047F4007700
:109180000AF1010A47F0400722E59AF800606C2EC8
:1091900003BF9AF8016047F020070AF1010A47F07F
:1091A000100715E59AF8006047F0080710E59AF8EF
:1091B000006047F001070BE59DF88330002B7FF43A
:1091C0008EAD9AF800608DF8839001E5FFFFEF7F88
:1091D000E8ED0008ECED0008F8ED0008BB46012BB7
:1091E00000F0C081022B54AD20D1189A04F00F0377
:1091F0002409D35C05F8013D44EA09744FEA1919C2
:1092000054EA0903F2D154AB5B1B5F460C930899F7
:109210000C989DF8832081424FF00003B8BF0146AF
:109220000D9306910F931393109391E604F00703A7
:10923000E40844EA49744FEAD909303354EA090191
:109240002A4605F8013DF1D11BF0010FDBD0302B90
:10925000D9D03023023A05F8013C54AB9B1A5F4643
:109260000C931546D3E7652E40F3E680DDE9140143
:1092700000220023F7F756FA002800F0DC81299B32
:10928000BF4AC8F80020013301340122072B2A9479
:109290002993C8F8042000F3CC8408F10808229B25
:1092A000129A934280F2D682169B179A1C44C8E900
:1092B0000023299B2A940133072B299300F324844C
:1092C00008F10808129B5D1E002D7FF7DBAD102D05
:1092D000299BDFF8B09240F3BD8449462246B94647
:1092E000DDF824B0079C10260F4605E008F10808B9
:1092F000103D102D40F3AA8401331032072BC8E92A
:109300000076CDE92932F1DD28AA2146584604F03D
:10931000E1F900287FF42EADDDE929320DF1AC082A
:10932000E6E70A9B069AA3EB020BBBF1000F7FF75F
:109330008FADBBF1100F299ADFF848922CDD1D96F6
:1093400021464E46079CDDF82490102306E0ABF141
:10935000100BBBF1100F08F108081ADD01321031B3
:10936000072AC8E90063CDE92921F0DD28AA2146B2
:1093700048460DF1AC0804F0ADF900287FF4FAACD2
:10938000ABF1100BBBF1100FDDE929214FF01003F9
:10939000E4DCB1461D9E0C4601325C44072ACDE94F
:1093A0002924C8F80090C8F804B000F3A08308F19D
:1093B00008084DE5BBF1100F299ADFF8C8912DDDA3
:1093C00041462046A8464C46079DDDF824901023D0
:1093D00006E0ABF1100BBBF1100F01F1080119DD34
:1093E00001321030072AC1E90043CDE92920F0DD20
:1093F00028AA2946484604F06DF900287FF4BAAC43
:10940000ABF1100BBBF1100FDDE929202BA94FF0B8
:109410001003E5DC4546A1468846044601325C441B
:10942000072ACDE92924C8F80090C8F804B000F351
:10943000D08108F1080813E5129B012B40F38081CD
:10944000299EC8F80050013601340123072E2A94C2
:109450002996C8F8043000F37C8308F10808169BAD
:10946000179A01361C44072EC8E90023CDE9296468
:1094700000F37C8308F10808DDE9140100220023D1
:10948000F7F750F9002840F07881129B0136013B34
:1094900001351C44072EC8F800502996C8F804303E
:1094A0002A9400F35D8108F108081A9BC8F804307B
:1094B00001361C44072E24ABCDE92964C8F80030DE
:1094C0007FF7DEAC0799099828AA04F003F9002871
:1094D0007FF450AC2A9C0DF1AC08D3E4B9F1100F25
:1094E000DDE929212BDDCDE91D3B1F96DDF824B0F8
:1094F0004E461024A946079D04E0103E102E08F1A8
:10950000080817DD0132204B1031072AC8E9003462
:10951000CDE92921F1DD28AA294658460DF1AC08EC
:1095200004F0D8F800287FF425AC103E102EDDE9B9
:109530002921E7DCDDE91D3B4D46B1461F9EC8F8F9
:109540000490013209EB0104072A0F49C8F8001002
:10955000CDE9292400F351839DF8832008F1080800
:109560004DE4BB460A2C79F1000380F00C833034C3
:1095700001238DF84F415F460C930DF24F1546E6DF
:1095800028EE00083CEE00082CEE00080799099828
:109590001D9328AA04F09EF800287FF4EBAB2A9CC8
:1095A0001D9B0DF1AC083DE40799099828AA04F029
:1095B00091F800287FF4DEAB2A9C0DF1AC0843E45F
:1095C000102D299B21DD099FDDF81C90102604E059
:1095D000103D102D08F1080817DD0133BB4A103487
:1095E000072BC8E90026CDE92934F1DD28AA494630
:1095F00038460DF1AC0804F06DF800287FF4BAABE2
:10960000103D102DDDE92934E7DC0133AF4AC8F8FD
:1096100004502C44072BCDE92934C8F800207FF7EB
:1096200039AC0799099828AA04F054F800287FF467
:10963000A1AB2A9C2EE42299002940F31481DDF885
:109640004090129B9945A8BF9946B9F1000F0BDDD8
:10965000299B01334C44072BC8E900592A942993CC
:1096600000F39A8508F10808109EB9F1000FA8BF11
:10967000A6EB0906002E00F34683DDF840B079051D
:10968000AB4400F1CE84229B129A934202DBFA078C
:1096900040F1B883169A17991444C8E90012299A20
:1096A0002A940132072A299200F3838508F10808D9
:1096B000129AAE18A6EB0B06D51AAE42A8BF2E46DC
:1096C000002E0DDD299BC8F800B001333444072B70
:1096D000C8F804602A94299300F3F18508F108087A
:1096E000002EA8BFAD1B002D7FF7CCAB102D299B02
:1096F000DFF8DC9140F3AE8249462246B946DDF8F8
:1097000024B0079C10260F4605E008F10808103D1C
:10971000102D40F39B8201331032072BC8E90076ED
:10972000CDE92932F1DD28AA2146584603F0D2FFBF
:1097300000287FF41FABDDE929320DF1AC08E6E724
:10974000FE073FF57DAE299EC8F800500136013472
:109750000123072E2A942996C8F804307FF7A3AE78
:109760000799099828AA03F0B5FF00287FF402ABF7
:10977000DDE929640DF1AC0897E6129B5D1E002D12
:109780007FF793AE102DDFF8489140F37F82224699
:109790000897099C079F4FF0100B05E008F1080897
:1097A000103D102D40F3708201361032072EC8E9AB
:1097B000009BCDE92962F1DD28AA3946204603F055
:1097C00089FF00287FF4D6AADDE929620DF1AC08F3
:1097D000E6E70799099828AA03F07CFF00287FF4A0
:1097E000C9AA2A9C0DF1AC08FFF73ABB17F0100389
:1097F00072D117F0400200F0BD820E9A52F8044B6D
:109800000E929946A4B228E453F8044B0E93FB063B
:1098100056D47D0651D544F3C0394B4624B2FFF7E8
:10982000C1BB1BF0100340F036811BF0400200F07A
:1098300092820E9A52F8044B0E929946A4B20123DA
:109840000EE42D2364428DF8833069EB4909BB4651
:10985000012308E4F8077FF515AB25E59AF80060C9
:109860000E93FFF7B5B9299B1A4AC8F800200133B7
:1098700001340122072B2A942993C8F8042000F30D
:10988000708408F10808002940F01E82129A07F03F
:10989000010313433FF4F6AA169B1799E218C8E98F
:1098A0000013299B2A920133072B299300F361832C
:1098B00008F1080819E254ADA9E4B80500F1B48232
:1098C0004FEAE4794B46FFF76DBB00BF2CEE000872
:1098D0003CEE000828EE00080E9B53F8044B0E9354
:1098E000FFF7BBBBDDE9140102460B46F6F74CFF60
:1098F000002840F0A085612E00F05085412E00F038
:109900009982089B013326F02003069300F08F858F
:10991000472B00F07985DDE9141247F480730F932B
:109920001346002BC0F2ED850C9300231D938B464C
:109930000D93069B462B00F04A84452B00F04F8583
:109940000899019126A9049123A9039122A90291C2
:1099500002210C9B099800915A4600F0A9FF069B32
:10996000472B054640F01C8617F0010FB9460F9FA4
:1099700040F0D984269B5B1B1293069B472B00F07B
:109980001883069B462B00F05F84229B1093109B4C
:10999000069A013B412A229300F0AA85F2B20021E7
:1099A000002BB8BF109B8DF89020BABFC3F1010304
:1099B0002D222B22092B8DF8912040F363850DF188
:1099C0009F04BD4F2246104687FB0321DA17C2EBE6
:1099D000A10202EB8201A3EB4101303100F8011C2E
:1099E00019466329134600F1FF32ECDC3033D9B25B
:1099F000831E9C4202F8011C40F2CE8513460DF1F5
:109A0000920201E013F8011B02F8011B9C42F9D1FC
:109A10000DF1A1030DF192021B1A134424AA9B1A03
:109A20001A93129B1A9A012B1A440C9240F37285D6
:109A30000C9B169A13440C930C9A002329F480670C
:109A400022EAE27247F480770F9306921393109301
:109A50001D9B002B40F0DE829DF883200893FFF7CA
:109A600077BA0E9B0B9853F8041B0E93C217C1E9EB
:109A700000025546FFF724BA199B002B3FF42FA98B
:109A8000199B1B78002B3FF42AA99AF8006047F431
:109A90008067FFF79DB80E9B53F8044B0E9301238C
:109AA000FFF7DEBA854B189317F0200949D00E9BBB
:109AB000073323F00703D3F8049053F8084B0E93B1
:109AC000F80709D554EA090306D030238DF88560DC
:109AD00047F002078DF8843027F4806B0223FFF7EC
:109AE000BFBABB46FFF723BB754B1893DCE707995A
:109AF000099828AA03F0EEFD00287FF43BA92A9CD0
:109B00000DF1AC08FFF7A4B90799099828AA03F04A
:109B1000E1FD00287FF42EA92A9C0DF1AC08FFF787
:109B2000D1BB062B294628BF062308950D952A464A
:109B30000693644D0E940C930F9113911091FFF7BF
:109B400007BA17F0100369D00E9B53F8044B0E931D
:109B5000B6E70799099828AA03F0BCFD00287FF40E
:109B600009A9DDE929640DF1AC0878E407990998A1
:109B700028AA03F0AFFD00287FF4FCA8DDE92964E2
:109B80000DF1AC0878E40BF480630022CDE90CA859
:109B90000696DDF8648054AF16469A460CE0002322
:109BA000204649460A22F7F7ABF80A2C79F1000360
:109BB0001BD3044689462F4620460A2200234946E5
:109BC000F7F79EF830327D1E013607F8012CBAF106
:109BD000000FE4D098F800309E42E0D1FF2EDED096
:109BE0000A2C79F1000380F0F480CDF8648012969D
:109BF000DDE90CA8069EFFF706BB079909981D939F
:109C000028AA03F067FD00287FF4B4A89DF88320FC
:109C10002A9C1D9B0DF1AC08FFF7F1B817F040022C
:109C200000F0B6800E9A52F8044B0E929946A4B2F8
:109C300046E70799099828AA03F04CFD00287FF40D
:109C400099A82A9C0DF1AC08FFF729BB14463A46A7
:109C50004F46914601332C44072BC8F80090C8F8B2
:109C60000450CDE929347FF70BA92BE4012BBB4627
:109C70007FF4B8AA7BE40E9B0B9953F8042B55464E
:109C800011600E93FFF71CB9089F144601362C444F
:109C9000072ECDE92964C8F80090C8F804507FF772
:109CA00002AC5DE52846CDF820900E94F7F7C8FB8E
:109CB00003460C90FFF7B4B967666666F8ED0008D6
:109CC0000CEE000820EE0008169B1798E218C8E971
:109CD0000003299B2A920133072B299300F3498122
:109CE00008F108080029C0F2FA821299C8F8005059
:109CF00001338C18072BCDE92934C8F804107FF7FD
:109D0000BFA8FFF7DFBB102E299BDFF8C09252DD02
:109D1000484642462146A846B946099C079D4FF051
:109D2000100B074603E00832103E102E3DDD0133D4
:109D30001031072BC2E9007BCDE92931F3DD28AAD8
:109D40002946204603F0C6FC00287FF413A8DDE96D
:109D500029312BAAE8E70E9B1BF4007914BF53F8B6
:109D6000044B53F8044B0E931CBF9146E4B20123FD
:109D7000FFF776B90E9B17F4007914BF53F8044B24
:109D800053F8044B0E931CBF9146E4B2FFF765B93C
:109D90000E9B17F4007914BF53F8044B53F8044B8F
:109DA0000E931CBF9146E4B28AE6454690463A4679
:109DB0000C464F46914601333444072BCDE92934F4
:109DC000C8F80090C8F8046000F3E68008F10808BD
:109DD00053E41C9B1B99ED1A1A46284603F00CFC11
:109DE00098F801300BB108F10108204649460A22D3
:109DF00000230026F6F784FFDBE62D228DF8832072
:109E0000FFF796B8129AAE18A6EB0B06D51AAE421B
:109E1000A8BF2E4664E40E9B0B9953F8042B0E93B7
:109E200011805546FFF74CB844F3C0194B4664B255
:109E3000FFF7B8B830238DF8843058238DF885307B
:109E4000089B632B47F0020400F39B8200230D93D1
:109E50003BADDDE9141247F481730F931346002BD9
:109E60002746C0F220820C9326F02003069300239D
:109E70008B461D93612E00F0ED82412E7FF459AD8B
:109E800022AA0C99584603F079FB00224FF07F5329
:109E9000F7F796FB02460B46CDE91023002200237C
:109EA000F6F740FC08B101232293494B0C93089B21
:109EB000CDE912A6CDE91E78DDF830A0DDE9106706
:109EC00003F1FF39AB46109506E00022002309F1AB
:109ED000FF39F6F727FCE8B93E4B002230463946F9
:109EE000F7F76EFB0F460646F6F764FC0446F6F7F6
:109EF00059FB0B46024639463046F6F705FA1AF882
:109F00000430B9F1FF3FD8464D460BF8013B0646F9
:109F10000F46DAD1304639462F4BDDF848A0139E64
:109F2000CDF848800022A946DDF87C80109D1E9F58
:109F3000CDE91001F6F71EFC002840F03482DDE97F
:109F40001001254B0022F6F7EDFB10B1E10700F1FF
:109F50002A824B46002B06DB01335B4430220BF890
:109F6000012B5B45FBD1ABEB0503B94612930F9F69
:109F700003E50799099828AA03F0ACFB00287EF4B2
:109F8000F9AEDDE9293222990DF1AC08AAE6906D0F
:109F900002F07AFCFEF7C0BE0799099828AA03F0E0
:109FA00099FB00287EF4E6AE2A9C0DF1AC08FFF781
:109FB00064BB229B1093DA1C02DB089A93420DDDEE
:109FC000023E26F020030693E1E400BF3CEE0008C9
:109FD0000CEE0008000030400000E03F109B129A99
:109FE0009342C0F2568119F0010F00F08782169A51
:109FF00013440C9319F4806F03D0109B002B00F3D3
:10A0000050820C9B23EAE3730693672600230F9389
:10A0100013931DE52D2200238DF883200893FEF76E
:10A020009ABF129BCDF830A04246DDF84C801097C5
:10A03000EB1808935E46199FDDF87090DDF824A0B8
:10A04000DDF81CB00F9B13952146B8F1000F2ED000
:10A05000002B6BD1013F08F1FF381B9BC2E900398F
:10A06000299B01334944072B2A91299362DC08324A
:10A07000089B38789B1B8342A8BF0346002B1C46D5
:10A080000ADD2998013019440728C2E900632A91A2
:10A0900029905ADC38780832002CACBF051B0546E5
:10A0A000002D15DC06440F9BB8F1000FD0D1002B1A
:10A0B0003CD1DDE91235EB189E421997B346DDF825
:10A0C00030A0109F90460C4628BF9B46FFF7DBBA96
:10A0D000102D29981DDD102404E0103D102D02F1F3
:10A0E000080216DD0130AC4B10310728C2E90034FC
:10A0F000CDE92901F1DD28AA5946504603F0EAFAD4
:10A1000000287EF437AE103D102DDDE929012BAA81
:10A11000E8DC0130A04B556029440728CDE929012E
:10A1200013602CDC387808320644BCE70F9B013BF7
:10A130000F9392E728AA5946504603F0CBFA00281D
:10A140007EF418AE2A992BAA92E728AA59465046BF
:10A1500003F0C0FA00287EF40DAE38782A992BAAB5
:10A160009AE70799099828AA03F0B4FA00287EF420
:10A1700001AE22992A9C0DF1AC08FFF784BB28AAF6
:10A180005946504603F0A6FA00287EF4F3AD38781D
:10A190002A992BAA064486E70799099828AA03F06A
:10A1A00099FA00287EF4E6AD2A9C0DF1AC08FFF781
:10A1B0005BBA0799099828AA03F08CFA00287EF464
:10A1C000D9AD229B2A9C0DF1AC08FFF771BA089912
:10A1D000019126A9049123A9039122A902910321A7
:10A1E0000C9B099800915A4600F062FB0378302BD3
:10A1F000054600F09581229B089AB94613440F9FAB
:10A20000EC180C99584600220023F6F78BFA10B18F
:10A210002346FFF7B0BB269BA342BFF4ACAB302173
:10A220005A1C26921970269B9C42F9D8FFF7A3BBB3
:10A23000089B9DF883200E9406930C9308900F9032
:10A2400013901090FEF784BE229A1092002A40F3D9
:10A250008181089909F001030B4340F05581109B5F
:10A260000C93662619F4806F40F01C810C9B23EA46
:10A27000E3730693CAE60799099828AA03F02AFA15
:10A2800000283EF425AEFEF77BBD00230893FEF7C1
:10A29000A1BC129B169A9A18109B0C92002B40F3AB
:10A2A0004D816726DEE726F020030693DDE91434AE
:10A2B0009B4604F100430C932D231D93DAE5079987
:10A2C000099828AA03F006FA00287EF453AD229DCF
:10A2D000129B2A9C5D1B0DF1AC08FFF701BA4E42A0
:10A2E0001031DFF8B49034DA4146DDF824B0A846E6
:10A2F0001024079D03E00831103E102E27DD0133A6
:10A300001032072BC1E90094CDE92932F3DD28AAE8
:10A310002946584603F0DEF900287EF42BADDDE92E
:10A3200029322BA9E8E7089BEC186AE7079B5B6ECC
:10A33000DD0707D4079B9B899C0503D4079B986D79
:10A3400002F0A2FA4FF0FF330B93FEF722BD454611
:10A35000884601333244072BCDE92932C8F80090F2
:10A36000C8F804607FF7A4AA0799099828AA03F0FF
:10A37000B1F900287EF4FEACDDE929320DF1AC081C
:10A38000B3E40998591CFCF72FFD0546002800F09E
:10A390000D810D905DE500BF3CEE000830238DF887
:10A3A000843078234AE5129B26930C9B1BF8012CE2
:10A3B000D97B8A425B4609D1302003F8010C269BE9
:10A3C0005A1E269213F8012C9142F6D0392A0BBF5F
:10A3D0000C9A0132927AD2B203F8012CC3E50899A3
:10A3E0000C9B09984C1C26A9049123A9039122A92E
:10A3F000029102215A460194009100F059FA054653
:10A40000B9462C440F9FFCE6089B002B08BF012394
:10A41000089347F480730F93159B002BC0F2AE8016
:10A42000DDF850B01D900C930D90FFF789BA06230C
:10A430000893FFF770BA159B604D002BB4BF2D2217
:10A440009DF883205E4BB8BF8DF8832027F08007EE
:10A45000FEF772BD22AA0C99584603F08FF800222D
:10A460004FF07F53F7F7ACF802460B46CDE91023C7
:10A4700000220023F6F756F908B101232293514B2D
:10A480000C9314E5002962D130228DF892200DF151
:10A490009302303302F8013B24ABD31A1A93FFF72F
:10A4A000C0BA672619990B78FF2B7BD00024109A2D
:10A4B000204603E001300131FF2B08D0934206DA39
:10A4C000D21A4B78002BF5D10B780134F4E71991AF
:10A4D000109213900F940F9A139B1C9913440C9A8B
:10A4E00001FB03230C9323EAE3730693FFF7B0BA4F
:10A4F00006F10F02D2B20121FFF752BA109B0C9362
:10A5000078E500230D93D1E6169BD31819440C91DE
:10A510006626A7E619F0010F3FF48EAAFFF788BA66
:10A520000C99584600220023F6F7FCF800287FF427
:10A5300062AE089BC3F1010322935DE6C3F1010300
:10A540001A4422EAE2730C92069367265EE50DF147
:10A5500092029EE7089A09F0010959EA020304D120
:10A560000123069366260C9350E5169B01331A448B
:10A5700022EAE2730C920693662647E50D9095E673
:10A580000E9B9AF80160924653F8042B0E9342EA10
:10A59000E2720892FEF71CBB02231A93FFF741BA3E
:10A5A000089C2DE700230F93139394E7079A938950
:10A5B00043F040039381FEF7E3BB00BFF0ED0008DA
:10A5C000F4ED0008F8ED0008F0B51F468B89ADF2F8
:10A5D0006C4D23F00203ADF80C304B6E1993CB8910
:10A5E000ADF80E30CB6907934B6A09931AAB009311
:10A5F00004934FF48063154606460293059316A80C
:10A6000000230C46069302F039F92A463B46694678
:10A610003046FEF76FFA051E07DB6946304601F04B
:10A6200039F9002818BF4FF0FF35BDF80C305B0634
:10A6300003D5A38943F04003A381169802F020F9C3
:10A6400028460DF26C4DF0BD38B50C46084D8446D9
:10A65000114620461A4600232B606446F8F71EFA7E
:10A66000431C00D038BD2B68002BFBD0236038BDC5
:10A67000540D002438B5334B1B6805460C460BB10E
:10A680009A6B12B3B4F90C3018079AB225D5216928
:10A6900000292DD012F0010007D00020A0606069D1
:10A6A0004042A06139B1002038BD950758BF6069AC
:10A6B000A0600029F7D1120658BF0846F4D543F030
:10A6C0004003A3814FF0FF3038BD184601F016F962
:10A6D000B4F90C3018079AB2D9D4D1062AD552074A
:10A6E00014D4216943F00803A3819AB20029D1D17F
:10A6F00002F42070B0F5007FCCD02146284602F04D
:10A70000DBF8B4F90C3021699AB2C3E7216B51B17F
:10A7100004F14002914204D0284601F0E7F9B4F96F
:10A720000C300022226321690022C4E9001223F0C8
:10A730002403D7E7092243F040032A604FF0FF309B
:10A74000A38138BD20000024024B13B1024800F061
:10A7500005B870470000000021BA00080023014638
:10A760001A46184603F0DEBE38B5074D00220446EF
:10A7700008462A60F8F7ACF9431C00D038BD2B68B6
:10A78000002BFBD0236038BD540D00242DE9F04F81
:10A7900003690C69A34283B0C0F28680013C01F1D9
:10A7A0001405A30000F11408009355F8243058F85C
:10A7B000242001338A469A4208EB8401814605EB46
:10A7C00084070191B2FBF3F638D30023AE4640462E
:10A7D0009B465EF8041B02681FFA81FC06FB0C33E3
:10A7E000090C4FEA134C06FB01CC99B2ABEB01010B
:10A7F0001FFA8CF311FA82F1C3EB124202EB2142F1
:10A8000089B241EA0241774540F8041B4FEA1C43F4
:10A810004FEA224BDDD2009B58F8033073B9019BFD
:10A82000043B984504D307E0984504F1FF3403D274
:10A8300053F80429002AF7D0C9F810405146484679
:10A8400002F048FC00282BDB01364046002355F877
:10A85000041BD0F800C08AB29A1A0B0C12FA8CF2C0
:10A86000C3EB1C4303EB224392B242EA0342AF42E2
:10A8700040F8042B4FEA2343E9D258F8242008EB90
:10A8800084036AB9043B984504D307E0984504F172
:10A89000FF3403D253F80429002AF7D0C9F8104036
:10A8A000304603B0BDE8F08F002003B0BDE8F08F64
:10A8B0002DE9F04F016C99B090469946CDE9048995
:10A8C000259D044641B1426C4A60012393408B6050
:10A8D00002F04AF900232364B9F1000AB4BF01234E
:10A8E00000232B60764BBCBF2AF0004ACDF814A0A1
:10A8F00033EA0A0300F0AA80DDE904231046194672
:10A9000000220023CDE90A01F5F70CFF074670B1DC
:10A91000249A01231360269B002B00F0E4826948EF
:10A920001860431E0393039819B0BDE8F08F16AB6F
:10A93000019317AB00932046DDE90A2302F01AFDCC
:10A940005FEA1A56054640F09780DDE916763E44E8
:10A9500006F23240202840F3B583C0F140000AFAE5
:10A9600000FA06F2124028FA00F04AEA0000F5F771
:10A9700009FE0123013EA1F1F8710F93524B002211
:10A98000F5F7C2FC48A3D3E90023F6F719FE48A364
:10A99000D3E90023F5F7BAFC804630468946F5F73F
:10A9A00001FE45A3D3E90023F6F70AFE02460B4653
:10A9B00040464946F5F7AAFC80468946F5F7FAFE77
:10A9C00000228346002340464946F5F7B5FE00289D
:10A9D00040F07C82BBF1160F00F26B823B4B03EB25
:10A9E000CB03D3E90023DDE90A01F5F7A5FE002832
:10A9F00072D00023BE1B0E93731E0BF1FF3B069318
:10AA000000F15E8200230993BBF1000F6BDA099B12
:10AA1000CDF81CB0A3EB0B030993CBF100030D930E
:10AA2000229B092B4FF0000B66D8052B40F348837F
:10AA3000043B22930026229B023B032B00F26886F4
:10AA4000DFE813F05C04590450043304249A42F202
:10AA50000F73CAF3130A13605AEA08031AD1269B2C
:10AA6000002B00F064861A4B03930833269A039850
:10AA7000136019B0BDE8F08FDDE90A12C2F31303C9
:10AA8000084643F07F510F97A6F2FF36169F41F418
:10AA9000401173E7269B002B40F0EA830D4B039394
:10AAA00041E700BFAFF3008061436F63A787D23FE8
:10AAB000B3C8608B288AC63FFB799F501344D33FAD
:10AAC0000000F07F29EE00080000F83F40F1000888
:10AAD00050EE00084CEE0008BE1B731E069300F1FA
:10AAE00085840E900990069B5B44CDE9063B0023CC
:10AAF0000D93229B092B98D90023CDE922330126FF
:10AB00004FF0FF330C960893089B12930021616469
:10AB1000204602F003F80390002800F00186039B12
:10AB20002364089B0E2B00F21381002E00F010818D
:10AB30000799002940F35C84AE4B01F00F0203EB50
:10AB4000C2034FEA2118C905D3E9006740F1148414
:10AB5000A94BDDE90A01D3E90823F6F75BFECDE94D
:10AB6000100108F00F084FF0030AB8F1000F13D0DE
:10AB7000DFF8849218F0010F09D030463946D9E940
:10AB80000023F6F71DFD0AF1010A06460F465FEAAB
:10AB9000680809F10809EDD1DDE9100132463B46AC
:10ABA000F6F738FE804689460E9B43B1934B002250
:10ABB00040464946F5F7C0FD002840F03085504634
:10ABC000F5F7F0FC42464B46F6F7FAFC8C4B0022B8
:10ABD000F5F79CFBA1F15073CDE910011193089B8F
:10ABE000002B00F09780079B1493089B13930C9BFA
:10ABF000002B00F0A584139A7E4B8249039E03EB41
:10AC0000C20353E902230020F6F704FEDDE9102316
:10AC1000F5F77AFBCDE9100149464046F5F7CAFD44
:10AC20000746F5F7BFFC02460B4640464946F5F796
:10AC30006BFB3037DDE9102306F8017B804689463F
:10AC4000F5F77AFD002840F02985CDF854B00027AB
:10AC5000DDE910AB1095139D13942AE00137AF4244
:10AC600080F22C85684B504659460022F6F7A8FC26
:10AC7000654B002282468B4640464946F6F7A0FCCB
:10AC800089468046F5F796FD0446F5F78BFC0246AB
:10AC90000B4640464946F5F737FB303406F8014B82
:10ACA00052465B4680468946F5F746FD002840F04F
:10ACB000F38442464B4651490020F5F725FB5246A6
:10ACC0005B46F5F739FD0028C8D0DDE91343109D38
:10ACD000039A079302E0964200F0C884B24616F841
:10ACE000013D392BF7D00133DBB23370079B0133C1
:10ACF0000793C8E15046F5F755FC42464B46F6F738
:10AD00005FFC3F4B0022F5F701FBA1F15073CDE949
:10AD1000100111933D4B404649460022F5F7F4FAE5
:10AD2000DDE910894B46424606460F46F5F722FDFF
:10AD30008146002840F0AA84DDE91001024601F1B5
:10AD4000004330463946F5F7F7FC002840F04583CC
:10AD5000179B002BC0F28C80079A0E2A00F3888084
:10AD6000244B03EBC203D3E900AB239B002B1BDA7C
:10AD7000089B002B18DC40F02E83244B0022504609
:10AD80005946F6F71DFC02460B46DDE90A01F5F7C8
:10AD9000DDFCDDF820904E46002800F0C782239BA2
:10ADA000DDF80C80DF43C9E2DDE90A7852465B46F4
:10ADB00038464146F6F72EFDF5F7FCFC8146099032
:10ADC000F5F7F0FB52465B46F6F7FAFB039E0B469F
:10ADD000024641463846F5F797FA09F1300306F87E
:10ADE000013B089B012B00F05C830694012704952E
:10ADF0001C462AE040F1000818F100080000F03F6E
:10AE000000001C400000E03F00002440000014400F
:10AE100052465B4640464946F6F7FCFCF5F7CAFC4D
:10AE20000546F5F7BFFB52465B46F6F7C9FB01370F
:10AE30000B46024649464046F5F766FA05F13003EF
:10AE4000A74206F8013B00F02983AC4B0022F6F73D
:10AE5000B7FB0022002380468946F5F763FC0028F3
:10AE6000D6D0049D069C079B01330793B2460AE1A6
:10AE70000C9A002A3DD0229A012A40F39C82089B1A
:10AE800003F1FF380D9B4345C0F26D82A3EB080828
:10AE9000089B002BC0F23C83069A1A440692099A3A
:10AEA00017461A4409920121204601F05FFF064629
:10AEB00023E00123BE1B0E93731E06937FF5A2AD04
:10AEC000C6F101030993002306939DE55846F5F763
:10AED00069FB42464B46F5F725FC00287FF47AAD26
:10AEE0000BF1FF3B76E5864B0393039819B0BDE861
:10AEF000F08FDDF83480099F0C9E002F0CDD069941
:10AF000000290B4608DD099AB942A8BF3B46D21A70
:10AF1000FF1ACB1A099206930D9BDBB10C9B002BF9
:10AF200000F05D82B8F1000F0FDD31464246204649
:10AF300001F0F8FF2A4601460646204601F044FF8C
:10AF400029460546204601F00FFE0D9BB3EB080293
:10AF500040F0D8820121204601F008FFBBF1000F2C
:10AF6000814600F3B480229B012B40F386814FF091
:10AF7000000A0120BBF1000F40F0B580069A104492
:10AF800010F01F0000F09380C0F12003042B40F369
:10AF9000D283099BC0F11C00034402440993074477
:10AFA0000692099B002B05DD29461A46204602F031
:10AFB00019F80546069B002B05DD49461A46204632
:10AFC00002F010F881460E9B002B40F03681089B62
:10AFD000002B40F31D810C9B002B40F0A080079BB1
:10AFE00001330793DDF80C80DDF820A0012707E08E
:10AFF000294600230A22204601F0C0FD01370546FC
:10B0000049462846FFF7C2FB574500F1300308F8D0
:10B01000013BEDDB089A002AC8BF9346039AD8BFCC
:10B020004FF0010B93440027294601222046049348
:10B0300001F0D8FF4946054602F04CF8002840F3DD
:10B04000A8811BF8013C039A0BF1FF3B04E05A4531
:10B0500000F0AA811BF8013D392B0BF1010AF6D053
:10B0600001338BF800304946204601F07DFD56B192
:10B070002FB1B74203D03946204601F075FD314665
:10B08000204601F071FD2946204601F06DFD0023A8
:10B090008AF80030249B079A1A60269B002B3FF405
:10B0A00042AC0398C3F800A019B0BDE8F08F1C2093
:10B0B000099B03440993069B03440744069370E7E6
:10B0C0000126B8E4C0F1200008FA00F04FE4014680
:10B0D0005A46204601F026FF229B012B814640F371
:10B0E000B3814FF0000AD9F8103009EB83031869D7
:10B0F00001F0EEFDC0F1200040E700BF0000244059
:10B1000028EE0008314600230A22204601F036FDD1
:10B11000129B002B064640F3E782CDE90783002F00
:10B1200000F31A81BAF1000F40F0D581B046049BBC
:10B13000039F089903F001027B1E1944229B0C9285
:10B14000134309910A9349462846FFF71FFB3146EE
:10B150008346284601F0BEFF4246494682462046C5
:10B1600001F0D8FFC26801460BF13003002A42D13A
:10B1700006902846089301F0ADFF069904902046FA
:10B1800001F0F2FC049A089B1AB90A99002900F010
:10B190009B82BAF1000FC0F2638122994AEA010A48
:10B1A0000C9951EA0A0100F05B81002A00F3B48196
:10B1B000099A3B7007F1010A9742D34600F0B28129
:10B1C000294600230A22204601F0D8FC46450546C0
:10B1D00031464FF000034FF00A02204612D001F032
:10B1E000CDFC4146064600230A22204601F0C6FC5B
:10B1F00057468046A7E72046049301F0B5FC049B20
:10B200000122C6E701F0BAFC5746064680469AE797
:10B21000229B022B79DC0C9B002B80D1079B49469B
:10B22000013328460793FFF7B1FADDF80CB000F1BF
:10B2300030030BF8013B0027F6E64946284601F0AB
:10B2400049FF0028BFF6C3AE294600230A22204644
:10B2500001F094FC079B03F1FF380C9B0546002B83
:10B260007FF450AF129B002B40F335820893B9E670
:10B27000AF4B03930333FFF7F9BBDDE90412002959
:10B280007FF475AEC2F31303002B7FF470AEA94BAD
:10B290001340002B00F0FE81099B01330993069BAC
:10B2A000013306934FF0010A63E601230C93239BBD
:10B2B000079A134412930133012B1F460893B8BF1A
:10B2C00001270021172F61647FF722AC012204239C
:10B2D0005B0003F11400B842114602F10102F7D9F4
:10B2E000616415E401230C93239B002B4CDD129326
:10B2F00008931F46E5E700230C93D8E700230C933F
:10B30000F2E7129BCDF81C800893089B002B7FF47A
:10B3100046AD49460522204601F030FC01468146F3
:10B32000284601F0D7FE00287FF739AD0398079F24
:10B330003123804600F8013B0137039049462046FF
:10B3400001F012FC7B1CDDF80CA00793CDF80C80FB
:10B35000002E7FF494AE96E631463A46204601F040
:10B3600041FE0646DEE60D9BCDF83480A8EB0303D4
:10B370009B444FF000088BE5DDE90A234FF0020AF9
:10B38000CDE91023FFF7F1BB012323930893FFF7C7
:10B39000BBBB03D1049BDB073FF553AEDA461BF87A
:10B3A000013D302BFAD05EE6079B039A01330793E9
:10B3B0003123137057E60F9A002A00F0268103F21A
:10B3C0003343069ADDF834801A440692099A1746E8
:10B3D0001A44099267E54FF000094E46DFE429461A
:10B3E0000D9A204601F09EFD0546B3E50E9067E5F7
:10B3F00000F00F81079A504B564206F00F0203EB04
:10B40000C203D3E90023DDE90A01F6F7D9F83611C2
:10B410008046894600F07181484F00234FF0020AB0
:10B42000F20706D5D7E90023F6F7CAF80AF1010AB0
:10B430000123761007F10807F2D1002B3FF4B4ABDB
:10B4400080468946FFF7B0BB049B002B7FF449AED2
:10B45000DDE90412C2F31303002B3FF418AF40E6FA
:10B46000002A12DD294601222046049301F0BAFD8C
:10B470004946054601F02EFE0028049B40F3188142
:10B48000392B00F0F9800BF13103BA460AF8013B81
:10B49000079B0133374607934646E4E50995069C2A
:10B4A000049D02460B46F4F731FF52465B46804648
:10B4B0008946F5F75FF960B952465B464046494612
:10B4C000F5F730F900283FF4CEAC099BD9077FF59A
:10B4D000CAAC039A02E47168204601F01FFB0746DC
:10B4E000002800F00E81336902339A0006F10C0146
:10B4F0000C30F5F787FD39460122204601F072FD38
:10B50000804614E62946204601F00CFD054621E55B
:10B51000DDE908239F1AC6E4392B00F0AD80BA4656
:10B520000133B3E7079A01323746079246467BE577
:10B530004CEE00080000F07F40F1000818F1000810
:10B54000DDF84CA0844901EBCA01DDE9102351E983
:10B550000201F6F735F8CDE9100149464046F5F706
:10B5600029F90646F5F71EF80B46024649464046BD
:10B57000F4F7CAFE039F53463036012B07F8016BE0
:10B580008046894600F0AE80139E039B1E44734B99
:10B59000002240464946F6F713F889468046F5F7FB
:10B5A00009F98246F4F7FEFF0AF1300A02460B461B
:10B5B00040464946F4F7A8FE07F801ABB74280467B
:10B5C0008946E4D1664B0022DDE91001F4F79EFEC6
:10B5D00042464B46F5F7B0F8002864D1DDE9102368
:10B5E0005F490020F4F790FE42464B46F5F7C2F85B
:10B5F00000283FF4ADABB246013E1AF8013C302BB7
:10B60000F9D0149B013307933DE5169BC3F1360334
:10B61000D7E6DDE90A894FF0020AFFF7C5BA089BB1
:10B62000002B3FF467AB129B002B7FF791AB079A7F
:10B63000013ACDE913324046484B00224946F5F71E
:10B64000BFFF804689460AF10100F4F7ABFF42468E
:10B650004B46F5F7B5FF434B0022F4F757FEA1F137
:10B660005073CDE910011193FFF7C1BA079B013365
:10B6700007933123FFF739BB079BBB460133079381
:10B68000392337460BF8013B4646DCE44FF000090E
:10B690004E464BE69A466CE4109D139C149B013376
:10B6A0000793B246EFE4149B039A0793FFF716BB88
:10B6B0007FF4EBAEDA077FF5E8AEE1E6DDF854B0F3
:10B6C000109D139CFFF744BB392BD5D0BAF1000F66
:10B6D0003FF7D9AED9E6229B022B3FF712AECDF849
:10B6E0001C809BE53E466DE7229B022B3FF709AE8F
:10B6F000129BCDF81C80089311E54FF0020AFFF76A
:10B7000053BA194B19483A4640F2EA2102F050FF69
:10B71000002666643146204601F000FA039078B9AD
:10B72000114B124800224FF4D57102F041FF104B2B
:10B730000393FFF7F8B83FF434ACC0F13C00B7E432
:10B74000039B236401224FF0FF33239612930C9244
:10B750000893FFF7FDBA00BF40F100080000244045
:10B760000000E03F00001C405CEE000870EE0008A6
:10B7700050EE0008B1F90C20F8B50C461107074649
:10B7800042D4636842F40062002BA28159DDA56AAD
:10B79000002D54D000233E683B6093B212F48052D7
:10B7A00053D1E16901233846A847421C63D0A389DD
:10B7B000A56A5B0705D56368C01A236B0BB1E36B01
:10B7C000C01AE169024600233846A847411C3ED111
:10B7D0003B68002B3BD01D2B01D0162B52D1A389E7
:10B7E0002269226023F4006300216160A381216B40
:10B7F0003E6021B304F14003994202D0384600F084
:10B8000075F900202063F8BD2669C6B193B225689A
:10B8100026609A070CBF63690023AD1BA3600CE090
:10B82000D4F824C0E1692B4632463846E047B0F1EF
:10B83000000CA5EB0C05664416DD002DF0DC0020A5
:10B84000F8BDE36B002BA2DCF9E7206DB1E7B4F99A
:10B850000C302269226023F40063A3810022DB0400
:10B860006260C4D52065C2E7A38943F040034FF06E
:10B87000FF30A381F8BD3B68002B98D01D2B06D06C
:10B88000162B04D0A38943F04003A381F8BD3E608A
:10B89000D5E700BF38B50C46054608B1836BA3B1A8
:10B8A000B4F90C00B8B1636EDB0701D4810515D57E
:10B8B00028462146FFF75EFF636EDA07054602D48D
:10B8C000A3899B050ED5284638BD00F017F8B4F9BA
:10B8D0000C000028E7D10546284638BDA06D00F0D1
:10B8E000D1FFE5E7A06D00F0CFFF284638BD00BFCF
:10B8F000014900F075BB00BF69E600082DE9F0477B
:10B900008246394800F0BEFFDAF83840002C66D194
:10B91000DAF80450354ACAF83C200323CAE9B84390
:10B92000DFF8CC90DFF8CC80334F344E04230AF597
:10B930003B72CAF8E8222146C5E90243C5E9004442
:10B94000C5E904446C660822AC6105F15C00FBF7B4
:10B95000FBFCC5E90759C5E90987EE6205F1580006
:10B9600000F08CFFDAF80850254BEB602146C5E962
:10B970000044C5E904446C66AC60AC61082205F182
:10B980005C00FBF7E1FCC5E90759C5E90987EE62F0
:10B9900005F1580000F072FFDAF80C50194BEB601B
:10B9A0002146C5E90044C5E904446C66AC60AC615D
:10B9B000082205F15C00FBF7C7FC05F15800C5E95A
:10B9C0000759C5E90A76C5F8248000F057FF01231E
:10B9D000CAF838300448BDE8F04700F055BFBDE86C
:10B9E000F047014800F050BF500D0024F1B80008A6
:10B9F0009D7A0008C17A0008017B0008217B0008BD
:10BA00000900010012000200014800F03BBF00BF26
:10BA10004C0D0024014800F037BF00BF4C0D00243E
:10BA200038B5084B084D5B1B9C1007D0043B1D44E8
:10BA3000013C55F804399847002CF9D1BDE838404D
:10BA400003F006B888F2000884F20008F8B5244F25
:10BA50000C460646FBF7CAFCBA685568C4F57E6317
:10BA60000F3325F003052B4423F47F6323F00F03EA
:10BA7000A3F58054B4F5805F07DB00213046FBF767
:10BA800023FFBB682B44984204D03046FBF7B4FC3C
:10BA90000020F8BD61423046FBF716FF01300DD0A3
:10BAA000104ABB682D1B45F001055D6013683046E8
:10BAB0001B1B1360FBF7A0FC0120F8BD00213046E2
:10BAC000FBF702FFBA68831A0F2BDEDD43F0010398
:10BAD0005360054B03491B68C01A0860D5E700BFD7
:10BAE00050040024100D002458080024002961D0BF
:10BAF000F8B50C460646FBF779FC54F8042C7B4F4E
:10BB0000A4F1080522F0010105EB010CB868DCF88E
:10BB10000430604523F0030300F08B80D207CCF89B
:10BB2000043032D454F8082CAD1A1144AA6807F135
:10BB3000080082426AD00CEB0304D4F804E0EC68FD
:10BB4000D4601EF0010FA26000F0978041F0010365
:10BB50006B60CCF80010B1F5007F35D27A68CB0865
:10BB600048090121013381401143796007EBC30289
:10BB700057F83310083AC5E9021247F83350CD6040
:10BB80003046BDE8F840FBF737BC0CEB03025268C7
:10BB9000D00710D4194407F10800DCF808308342BC
:10BBA00073D0DCF80C20DA60936041F001036B6025
:10BBB0006950D0E7704741F00103B1F5007F44F8C8
:10BBC000043CCCF80010C9D3B1F5206F4FEA5123E3
:10BBD00048D28B0903F1390003F13802C300F81889
:10BBE000FB580838984259D05A6822F003028A421A
:10BBF00002D99B689842F7D1D868C5E902308560C0
:10BC0000DD603046BDE8F840FBF7F6BB0CEB030205
:10BC10005268D20763D40B44DCE90212CA60916017
:10BC200043F001026A603046EB50BDE8F840FBF794
:10BC3000E3BB0B44D10707D454F8082CAD1A1344C6
:10BC4000D5E90212CA60916043F001026A60284A95
:10BC5000BD6012689A4293D8264B30461968FFF7A8
:10BC6000F5FE8DE7142B0AD9542B1FD80B0B03F1CB
:10BC70006F0003F16E02C300B1E719448DE703F1D1
:10BC80005C0003F15B02C300A9E741F00103C7E9CF
:10BC90000455C5E902006B60695071E7796892103C
:10BCA000012404FA02F20A437A60A6E7B3F5AA7FF8
:10BCB00006D8CB0B03F1780003F17702C3008EE7BF
:10BCC00040F25452934206D88B0C03F17D0003F1ED
:10BCD0007C02C30083E74FF47E737E227FE741F04E
:10BCE00001036B60CCF800104AE700BF5004002449
:10BCF0005C080024400D00249368002B00F0818034
:10BD00002DE9F04FB1F90C300C461907804683B08D
:10BD1000174698B223D523690BB310F002033D6890
:10BD20002BD04FF0000ADFF8B4B256465E453346DA
:10BD3000524628BF5B464046002E4FD0E169D4F8FA
:10BD400024C0E047002852DDBB681B1A8244361A23
:10BD5000BB60002BEAD1002003B0BDE8F08F214684
:10BD60004046FEF787FC002840F03481B4F90C30DF
:10BD70003D6898B210F00203D3D110F0010942D10E
:10BD80004E463EB38205D4F808B040F18180B345F9
:10BD90005A4600F2B18010F4906F40F0BE802068E7
:10BDA0000192494600F03EFEA3682168019AA3EB88
:10BDB0000B030A44B246A36022600026B868A0EBD9
:10BDC0000A00D144B8600028C5D0B4F90C0080B294
:10BDD000002ED7D1D5E900960835D2E7D5E900A6DF
:10BDE0000835A3E721464046FFF754FD80B3B4F978
:10BDF0000C3043F040034FF0FF30A38103B0BDE8A7
:10BE0000F08F002070471E46AA46994618461D46E8
:10BE100056B388B34A46D4E904132068B24228BF17
:10BE20003246884205D9A16803EB010B5A4500F35D
:10BE3000A780934264DCE169D4F824C02A464046D6
:10BE4000E047B0F1000BD2DDB9EB0B09CAD00120FD
:10BE5000BB68A3EB0B035D44A6EB0B06BB60002B9A
:10BE60003FF479AF002ED4D10AF1080353E902560A
:10BE70009A460833002EF9D032460A212846F5F7B3
:10BE80004FFB002800F09D800130A0EB0509C1E7C1
:10BE900020682369984217D86369B34214D86FF0B9
:10BEA0000042B24228BF3246E16992FBF3F2D4F875
:10BEB00024C002FB03F340464A46E047B0F1000AC3
:10BEC00095DDA6EB0A0679E7B345DA4628BFB24608
:10BED0005246494600F0A6FDA3682268A3EB0A0378
:10BEE0005244A3602260002BEBD121464046FFF76D
:10BEF000D1FC0028E5D07AE72068B34632464FE708
:10BF00002946019200F08EFD019AA3689B1AA36056
:10BF1000236813442360934696E723682169A3EBC3
:10BF2000010B636903EB430A0AEBDA7A0BF10103B5
:10BF30004FEA6A0A33445345524684BF9A465246F2
:10BF400043052CD511464046FAF74EFF00283BD05A
:10BF50005A4621690190F5F755F8A289019B22F410
:10BF6000906242F08002A28103EB0B002361AAEBF6
:10BF70000B03C4F814A0A3602060B34632460FE759
:10BF800029465A4600F04EFD23685B442360214653
:10BF90004046FFF77FFC00283FF456AF27E74046B6
:10BFA000FBF7A6FA03460028DED121694046FFF7D9
:10BFB0009DFDB4F90C300C2223F08003C8F800205A
:10BFC00017E7721C914626E70C22B4F90C30C8F82A
:10BFD00000200EE74FF0FF30BEE600BF00FCFF7F01
:10BFE0002DE9F8430746884600F538764FF00009FA
:10BFF000D6E90154013D11D4A389012B05F1FF3588
:10C0000008D9B4F90E300133214603D03846C04771
:10C0100049EA00096B1C04F16804EDD13668002E72
:10C02000E6D14846BDE8F8832DE9F0410469B4EB58
:10C03000611F2FDD00F1140E4E1111F01F0C0EEBDD
:10C0400084050EEB86032BD05EF8262004339D4238
:10C0500022FA0CF1CCF1200818D977461A6802FAB6
:10C0600008F20A4347F8042B53F8041B9D4221FAB7
:10C070000CF1F3D8A41BA300053B9B0801330EEB86
:10C0800083044EF82310C9B1043417E041617446AB
:10C090000029F9D10023036100234361BDE8F08149
:10C0A0009D4288BF00F11002F4D953F8041B42F8F6
:10C0B000041F9D42F9D8A41B0EEB8404A4EB0E03CD
:10C0C0009B1074450361E7D0BDE8F0812DE9F04F86
:10C0D000A84C8BB0246805902046894602920793AD
:10C0E0000394F5F7ADF921460144D9F8003011F871
:10C0F00001BC99783029024640F0DA816FF00100E6
:10C10000C01A033300EB030A1C4613F8011B302945
:10C11000F8D0DFF8648218F80130002B00F0F080CE
:10C120002378002718F803303D4626462BB116F831
:10C13000013F18F80330002BF9D1039901923046E2
:10C14000FBF7F2FC019A0090002800F09180002D8E
:10C1500040F091803378009503F0DF03502B354693
:10C1600000F09380C9F80060002F40F0AB802B1BDB
:10C17000013B072B394604DD5B10072B01F1010160
:10C18000FADC0598049200F0C9FC049A019000289A
:10C1900000F06782019BAC4203F11406069680F022
:10C1A000DC810027C2F10103B946049310E0202F7F
:10C1B00000F091803946043715F8013C18F8033037
:10C1C000554603F00F038B40A54249EA030916D9EF
:10C1D00015F8013C5B4505F1FF3AE8D1049B534457
:10C1E000A342E4D31846039909920893FBF79CFCF9
:10C1F000DDE908320028DAD11D46A542E8D846F824
:10C20000049B069BF61A019BB6101E61484600F07F
:10C210005FFD029B76011C68301AA04200F3AE80DD
:10C22000C0F226810027029B009A9B689342C0F2CD
:10C2300089810299009A4B6893427EDD9D1AAC4237
:10C2400000F3BC80CA68022A00F0BC81032A00F017
:10C25000B481012A00F098810598019900F084FCCE
:10C260005025149A0023284613600BB0BDE8F08FC8
:10C27000002D00F00B81AD1BAB000093337803F071
:10C28000DF03502B35467FF46DAF6B782B2B00F01E
:10C29000ED802D2B6AD06E1C002018F803104B1E69
:10C2A000182B61D8737818F803301039013623BB86
:10C2B00000B14942009BC9F800600B440093002F75
:10C2C0003FF455AFBAF1000F14BF002506252846EC
:10C2D0000BB0BDE8F08F002146F8049B0427894687
:10C2E0006AE701EB810103EB4103A3F1100116F8AA
:10C2F000013F18F80330002BDAD0192BF1DDD7E716
:10C30000039900922046FBF70FFC009A002873D196
:10C31000A15C18F80130A518002B6FD030292C46ED
:10C3200005D114F8013F302BFBD018F80330B3FAD5
:10C3300083F77F094FF0010AF7E6012557B1029B09
:10C34000DB68022B62D0032B64D0012B00F08580C8
:10C3500045F01005149B019A1A60079B009A1A6019
:10C3600028460BB0BDE8F08F2E46FBE60120AB78E7
:10C37000AE1C92E77CF0000878EF0008019D061BD8
:10C380003146284601F0B4F8074678B1721E5311C1
:10C390000699012751F8231002F01F0307FA03F34F
:10C3A0000B4203D0BA4200F3E2800227009B0198BF
:10C3B000334431460093FFF737FE34E76E1E002FFB
:10C3C00040F0C980002E40F0CC807311069A01988D
:10C3D00052F8232006F01F06012303FA06F6164240
:10C3E000294618BF47F00207FFF71EFE029B5B6855
:10C3F0000093641B0225A1E72178254601F0DF01A7
:10C40000502900F0BD80C9F800505BE7159BC3F1CF
:10C4100001031593159B002B9AD0019BDDF8189012
:10C420001E6900214B464FEA860809EB860003E0AF
:10C43000984243F8041C3FD91F4653F8042BB2F12D
:10C44000FF3FF5D00132022D3A6000F0C08014F0B9
:10C450001F0440F0E08021257CE7BA077FF578AF24
:10C46000069B1B681F43FB07D7D471E700207EE7BC
:10C47000DDE90031221A9B1A0598009300F0B2FD05
:10C4800003461433019006930027CCE6B35C18F8FA
:10C490000310B018064600293FF45EAE16F8013FBF
:10C4A00018F803100029F9D1801B8100009153E690
:10C4B0009C1C4FF0000A2CE6019B9B689E4280F278
:10C4C0008D803346019901EB830201330B61022D0C
:10C4D0004FF0010151617AD09E42B8DA002B40F34F
:10C4E000A780019A09EB8303516902F11800834286
:10C4F0004FEA510140F2AF804C46026841EAC271F6
:10C5000044F8041B50F8041B83424FEA5101F4D84D
:10C51000019A9B1A193B9B08013349F8231009EB38
:10C520008303002940F09B800199A3EB090292103C
:10C530004B450A617FD0029B009A9B68013293426F
:10C54000009288DA0199059800F00EFB149A0023F6
:10C550001360A325BBE6012737E7069E4FF00009CD
:10C560004DE60198314600F0C3FF07462DE7B11EA6
:10C57000284600F0BDFF00283FF417AF032715E75A
:10C5800000230093012780E6AC427FF465AE012CC6
:10C5900008D00198611E00F0ABFF00283FF45CAEAC
:10C5A000029B5B6807990B60019B069901221A6147
:10C5B0000A60149A6225136089E6159A002A3FF4EE
:10C5C0004BAEEFE7159A002A7FF446AEEAE7029BEE
:10C5D0001B68013BA34232D02225BBE6019B059894
:10C5E0005968013100F09AFA074600283FD0DDF87B
:10C5F0000490D9F81030494602339A000C310C30BF
:10C60000F4F700FD4946059800F0AEFA07F1140969
:10C610003B69019756E7C844C4F1200458F8040C5C
:10C6200000F056FBA042BFF616AF019B1B6955E711
:10C63000019A00231361019A002353617BE7631180
:10C6400004F01F0459F823200123A34013420CBF18
:10C65000222521257EE6C9F800104B4669B1043336
:10C6600062E7074B0748019ADE2101F0A1FF044B66
:10C6700004483A46842101F09BFF019B1961DAE7E7
:10C680005CEE0008F0EE000810B4046809E014F84D
:10C69000013FA3F1410CBCF1190F98BF2033934225
:10C6A00008D111F8012B002AF1D1013404600120D6
:10C6B00010BC7047002010BC704700BF2DE9F04F40
:10C6C000096885B04B1111F01F01029002EB830342
:10C6D000039140F08E801D1F0193029B01991C68FD
:10C6E000002341F8043C61780134002900F0978070
:10C6F000DFF87091A846AC469A461E460EE0202907
:10C7000000F28B80B24506DAC44501D2072B5BDD0F
:10C71000624551D3082314F8011FA1B119F8010093
:10C720000028ECD00133082B06F101063ADCDCF8D6
:10C730000010090100F00F000843CCF8000014F8C5
:10C74000011F0029EAD1002E69D0E04501D9072B4D
:10C7500073DD624551D2111F634653F8040B41F853
:10C76000040F9D42F9D2A5EB0C0323F00303691CCF
:10C7700004330CF1010C614538BF0423134400213C
:10C7800043F8041B9D42FBD2019B53F8043C2BB998
:10C79000AA4248D055F8043D002BF9D0052005B039
:10C7A000BDE8F08F6245B6D200234CF8043C194630
:10C7B000ACF1040C0123BDE70023ACF104084CF8F4
:10C7C000043CB246C446A6E7C3F108018900DCF880
:10C7D0000030C1F1200E60468B46416801FA0EF729
:10C7E0003B43036021FA0BF340F8043F4045F4D388
:10C7F0008EE7191D01911D466FE7039B002BC3D0E7
:10C80000039B0198C3F120014FF0FF33CB4050F858
:10C81000041C0B4040F8043CB9E7292909D0042046
:10C8200005B0BDE8F08F012305202B6005B0BDE801
:10C83000F08F029901340C6085E7C3F108039B0077
:10C84000DCF80010C3F120076446666806FA07F0BA
:10C850000143216026FA03F144F8041FA045F4D8EF
:10C8600077E700BF78EF0008014B93F82801704785
:10C87000680800240048704758090024704700BF2A
:10C88000704700BF704700BF704700BF38B50C4607
:10C89000084D8446114620461A4600232B60644604
:10C8A000F6F722F9431C00D038BD2B68002BFBD0D3
:10C8B000236038BD540D00242DE9F0418B890C46CE
:10C8C000990796B008D504F143030122C4E9043264
:10C8D000236016B0BDE8F081B4F90E1000290646B9
:10C8E00027DB6A4601F0C2FF002821DB019D05F429
:10C8F0007045A5F50055B5FA85F54FF480686D09CA
:10C900004FF4006741463046FAF76EFAB4F90C303E
:10C91000F0B1204AF26343F08003C4F81480A3818D
:10C920002060206135BB3B43A38116B0BDE8F08198
:10C93000A38913F0800519D04FF0400841463046D6
:10C94000FAF752FA0025B4F90C302F460028E0D14E
:10C950009A05BED423F0030304F1430243F002031B
:10C960000121C4E90421A3812260B2E74FF4806869
:10C970002F46C7E7B4F90E10304601F08DFF10B90D
:10C98000B4F90C30CFE7A38923F0030343F001038C
:10C990001BB2C8E7F1B8000870B50C46B1F90E102B
:10C9A000002996B015461E4614DB6A4601F05EFF6C
:10C9B00000280FDB019A02F47042A2F50052B2FA8D
:10C9C00082F24FF4806352094FF4006032602B60B2
:10C9D00016B070BDB4F90C10002311F08000336064
:10C9E00004D0402218462A6016B070BD4FF4806310
:10C9F0002B6016B070BD00BF82B049B15AB16BB1A7
:10CA000013780B601278101E18BF012002B0704717
:10CA100001A9002AF3D1104602B070476FF001005F
:10CA2000F4E700BF88420DD98B1883420AD900EB86
:10CA3000020CBAB1624613F801CD02F801CD994259
:10CA4000F9D170470F2A0ED8034602F1FF3C4AB1D4
:10CA50000CF1010C013B8C4411F8012B03F8012F60
:10CA60006145F9D1704740EA01039B0750D1A2F11B
:10CA7000100370B501F1200C23F00F0501F1100E29
:10CA800000F11004AC441B095EF8105C44F8105C23
:10CA90005EF80C5C44F80C5C5EF8085C44F8085CDA
:10CAA0005EF8045C44F8045C0EF1100EE64504F1F7
:10CAB0001004E9D1013312F00C0F01EB031102F065
:10CAC0000F0400EB031327D0043C24F003064FEAC5
:10CAD000940C1E441C1F8E465EF8045B44F8045FF1
:10CAE000B442F9D10CF1010402F0030203EB840318
:10CAF00001EB840102F1FF3C4AB10CF1010C013B56
:10CB00008C4411F8012B03F8012F6145F9D170BD58
:10CB100002F1FF3C03469BE72246EBE7C36C70B58E
:10CB200005460C464BB153F8240080B1026843F827
:10CB300024200023C0E9033370BD2122042101F029
:10CB400057FD0346E8640028EDD1002070BD0121A7
:10CB500001FA04F6721D9200284601F049FD0028F2
:10CB6000F3D0C0E90146E4E731B1C36C4A6853F839
:10CB70002200086043F82210704700BF2DE9F04101
:10CB80000D6907460E461C4601F1140E0020DEF822
:10CB900000108BB202FB03434FEA134C090C02FB5B
:10CBA00001CC01309BB203EB0C4385424EF8043BB1
:10CBB0004FEA1C44EBDC3CB1B368AB4207DD06EB4B
:10CBC000850301355C6135613046BDE8F0817168EF
:10CBD00038460131FFF7A2FF8046A8B13269023220
:10CBE00006F10C0192000C30F4F70CFAFB6C726841
:10CBF00053F82210316043F82260464606EB850365
:10CC000001355C613561DFE7024B03484246B521DF
:10CC100001F0CEFC5CEE000894F000082DE9F8432A
:10CC20000C4628491E46174603F1080281FB0231D3
:10CC3000092E4FEAE2730546C3EB610339DD4FF07D
:10CC4000010C00214FEA4C0C634501F10101F9DCB4
:10CC50002846FFF763FF014668B3089B4361092F2D
:10CC60004FF00103036112DC0A340927BE420BDDD9
:10CC7000F61B264414F8013B0A22303B2846FFF7F6
:10CC80007DFFA6420146F5D10846BDE8F88304F1D0
:10CC90000909C8463C4418F8013B0A22303B2846A3
:10CCA000FFF76CFFA0450146F5D1A7F108044C44FD
:10CCB000DCE70021CCE70A46034B0448CE2101F013
:10CCC00077FC00BF398EE3385CEE000894F0000872
:10CCD000020C12040346CAB90304102013F07F4F5C
:10CCE00004BF1B02083013F0704F04BF1B01043057
:10CCF00013F0404F04BF9B000230002B05DB13F004
:10CD0000804F00F1010008BF202070470020E5E7B8
:10CD10000368024613F0070007D0D9071DD498070F
:10CD20001FD55B0813600120704799B209B91B0C2D
:10CD30001020D9B209B908301B0A190704BF1B0912
:10CD40000430990704BF9B080230D90703D45B085D
:10CD500000F1010003D013607047002070472020CD
:10CD600070479B0813600220704700BF38B5C36C42
:10CD700004460D464BB15868B0B102685A600022B3
:10CD80000123C0E90435C26038BD2122042101F02D
:10CD90002FFC0346E0640028EDD1094B094800222E
:10CDA0004FF4A07101F004FC1C220121204601F087
:10CDB0001FFC0028F1D001220223C0E90123DEE795
:10CDC0005CEE000894F000082DE9F04F0E6915693B
:10CDD000AE4285B08846144605DB2A4623463546D2
:10CDE0000C4616469846A3686168AF19BB42B8BFA7
:10CDF0000131FFF793FE0190002800F08780019B2E
:10CE000003F1140909EB870AD14505D24B460022EC
:10CE100043F8042B9A45FBD808F1140808EB860B5D
:10CE200004F11403D8451A4603EB85055FD22B1B8A
:10CE3000153B23F0030304331534A54238BF042304
:10CE4000CDE902A7AC461F46924605E0000C29D169
:10CE5000C34509F1040948D958F8040B85B2002DDF
:10CE6000F4D056464C46002356F8040B216882B293
:10CE70001FFA81FE05FB02EE000C0A0C734405FB51
:10CE8000002202EB13429BB243EA0243B44544F84A
:10CE9000043B4FEA1243E7D849F8073058F8040C2E
:10CEA000000CD5D0D9F80030544619464D46002222
:10CEB0002688090C00FB06110A449BB243EA024390
:10CEC00045F8043B54F8046B2968360C8BB200FB20
:10CED000063303EB1243A4454FEA1342E8D8C34597
:10CEE00049F8073009F10409B6D8DDE902A7002F97
:10CEF00002DC05E0013F03D05AF8043D002BF9D0D5
:10CF0000019B18461F6105B0BDE8F08F034B044834
:10CF1000019A40F25D1101F04BFB00BF5CEE00088E
:10CF200094F0000812F003032DE9F0411446064680
:10CF300032D10D46A41020D0D6F84880B8F1000FA9
:10CF400033D0E3074FF0000707D4641015D0D8F8AA
:10CF50000000A8B18046E307F7D54246294630468F
:10CF6000FFF732FFB5B16968F36C641053F8212004
:10CF70002A6043F821500546E9D12846BDE8F081F2
:10CF8000424641463046FFF71FFFC8F800000760E1
:10CF90008046E0E70546D8E7013B0F4A52F82320D8
:10CFA0000023FFF7EBFD0546C4E701213046FFF7FC
:10CFB000B5FD804640B1012340F27122C0E9043240
:10CFC0000023B0640360BCE7044B054842464FF4BD
:10CFD000A07101F0EDFA00BF08F200085CEE000855
:10CFE00094F000082DE9F0470C4690462669A368A6
:10CFF000496806EB6216751C9D4207464FEA6219A6
:10D0000004DD5B009D4201F10101FADC3846FFF7C7
:10D0100085FD8446002851D0B9F1000F00F11400BD
:10D020000EDD09F105024FEA820E03460CEB820287
:10D03000002143F8041B9342FBD1AEF114031844C2
:10D04000216904F1140318F01F0803EB81012DD0AE
:10D05000C8F1200986464FF0000A1A6802FA08F261
:10D0600042EA0A024EF8042B53F8042B994222FAA2
:10D0700009FAF2D80B1B153B23F00303043304F128
:10D080001502914238BF0423BAF1000F18BF2E4693
:10D0900040F803A0FB6C6268CCF8106053F82210D3
:10D0A0002160604643F82240BDE8F087043853F819
:10D0B000042B40F8042F9942F9D8EBE7034B0448BE
:10D0C000624640F2D91101F073FA00BF5CEE00082D
:10D0D00094F000080B6984460069C01A15D10CF160
:10D0E000140C14310CEB830210B401EB830301E048
:10D0F000944508D252F8044D53F8041D8C42F7D0E1
:10D1000004D24FF0FF3010BC70477047012010BCB4
:10D11000704700BF2DE9F84F0F691369FF1A002F00
:10D120000E4690467AD101F11405143202EB8302C7
:10D1300005EB830301E09D4273D253F8041D52F8BE
:10D14000044DA142F7D064D37168FFF7E7FC814634
:10D15000002872D03569D8F81020C76008F1140E85
:10D1600006F1140009F1140A06F1100C0EEB82020C
:10D1700000EB8507564600215EF8044B5CF804BFBF
:10D18000A3B211FA8BF1CB1A210CC1EB1B4101EBBD
:10D1900023419BB243EA0143724546F8043B4FEA00
:10D1A0002141E9D8A2EB0804153C08F115084245D5
:10D1B00024F0030606F1040638BF0426304424F0A8
:10D1C000030238BF002287425244B24416D9564661
:10D1D000044654F8043B11FA83F10A1402EB13429B
:10D1E00089B241EA0243A74246F8043B4FEA224192
:10D1F000EFD87A1E101A20F00302524423B952F8D5
:10D20000043D013D002BFAD0C9F810504846BDE856
:10D21000F88F334601274646984695E7F9DB002705
:10D2200092E70021FFF77AFC814668B101220023D2
:10D23000C9E904234846BDE8F88F074B07484A462A
:10D240004FF4107101F0B4F9034B04484A4640F220
:10D25000322101F0ADF900BF5CEE000894F0000847
:10D260000F4B0B40A3F15073002B02DD0020194639
:10D2700070475B42B3F1A07F4FEA235205DA4FF4C7
:10D280000023002043FA02F17047143A1E2ADABF45
:10D290004FF0004323FA02F20122002110467047AA
:10D2A0000000F07F2DE9F843066900F1140808EB4F
:10D2B0008606A6F1040956F8047C3846FFF708FDF7
:10D2C000C0F120030A280B6036DDC8451ED2B0F13C
:10D2D0000B0356F8082C26D0C3F1200C22FA0CF1CF
:10D2E0009F400F43A6F1080147F07F55884545F45C
:10D2F00040153AD202FA03F056F80C3C23FA0CF32C
:10D3000003431C4620462946BDE8F883B0F10B03D1
:10D3100008D007FA03F343F07F55002345F4401586
:10D320001C46EFE71A4647F07F5545F44015144672
:10D3300020462946BDE8F883C0F10B0327FA03F223
:10D34000C84542F07F553CBF56F8082CDA4000F142
:10D35000150328BF002207FA03F345F4401543EAFA
:10D36000020420462946BDE8F88302FA03F31C466E
:10D37000C8E700BF70B5012182B016461D46FFF711
:10D38000CDFB044600284BD02B46C5F30A55C3F30A
:10D3900013030DB143F48013002E019322D068468D
:10D3A0000096FFF7B5FC002836D0019B0099C0F12C
:10D3B000200203FA02F20A43C34001936261002B88
:10D3C00014BF02210121A3612161ADB1069AA5F22A
:10D3D000334303441360079BC0F1350018602046B7
:10D3E00002B070BD01A8FFF793FC019B0121C4E9C5
:10D3F00004132030002DE9D104EB8102A0F2324366
:10D400001069069A1360FFF763FC079BC0EB41119C
:10D410002046196002B070BDDDE900236261CEE7ED
:10D42000034B0448224640F20A3101F0C1F800BF24
:10D430005CEE000894F000082DE9F04383B00F463D
:10D4400069468046FFF72EFF04460D46384601A97F
:10D45000FFF728FFD8F810303A690F469A1ADDE92D
:10D460000013CB1A03EB4213002B06460BDD05EB32
:10D4700003594D4632463B4620462946F4F7CAF941
:10D4800003B0BDE8F083C3EB033307EB03510F4652
:10D49000F0E700BF0139491101F1010C116902F1F6
:10D4A000140303EB81018B4200EB8C0C16D210B5F8
:10D4B000A0F1040E53F8044B4EF8044F9942F9D8EA
:10D4C0008B1A153B23F0030304331844844504D915
:10D4D000002340F8043B8445FBD810BD844505D9A2
:10D4E000002340F8043B8445FBD87047704700BFD9
:10D4F00003694A11934200F1140009DA00EB830337
:10D5000002E053F8042DC2B98342FAD800207047D4
:10D5100010DD11F01F010DD010B450F8224000EBC7
:10D52000820324FA01F202FA01F18C420BD00120AD
:10D5300010BC704700EB8203E6E70120704753F808
:10D54000042D002AF3D18342F9D8002010BC704783
:10D5500038B50C46084D8446114620461A4600232D
:10D560002B606446F5F7C8FA431C00D038BD2B6821
:10D57000002BFBD0236038BD540D0024DFF860C0C1
:10D58000F8B521F000430027634504460D461646D2
:10D59000176022DC844653EA0C0C1ED0DFF844C02E
:10D5A00001EA0C0C0A46BCF1000F09D10E4B002217
:10D5B000F4F706F86FF0350704460A4621F00043F9
:10D5C00022F0FF421B1522F4E002A3F2FE3342F0E8
:10D5D0007F553B4445F40015336020462946F8BD8D
:10D5E000FFFFEF7F0000F07F000050430149002063
:10D5F000704700BF0000F87F30B540EA0104A30780
:10D6000001D1032A0FD8844601F1FF3E07E01EF83E
:10D61000011F03F8011B541EC1B19C4622466346FC
:10D62000002AF4D130BD0B468446194653F8045BFA
:10D63000A5F1013424EA050414F0803FE4D1043A52
:10D64000032A4CF8045B1946EFD8DDE76244002C4E
:10D65000E8D003F8011B9342FBD130BD2DE9F84F10
:10D660004B6E9C0490462DD59368126843B38B464D
:10D67000064602F1080959E9025A5FEA9A0715D0ED
:10D68000043D002401E0A7420ED055F8041F5A467D
:10D69000304601F0B7F8431C04F10104F3D1002334
:10D6A000C8E90133BDE8F88FD8F808302AF0030A3A
:10D6B000A3EB0A03C8F8083009F10809002BDAD1F6
:10D6C0000020ECE7FEF718FB0023C8E90133BDE8B2
:10D6D000F88F00BF10B4946814B110BCFFF7BEBF40
:10D6E0002046546010BC70472DE9F04FBDB0CDE925
:10D6F00004301C460191174618B1836B002B00F0D3
:10D700008682019A536EDE0740F18F81B2F90C10C8
:10D710008AB2900408D441F4005201994B6E8A8178
:10D7200023F4005392B24B66110740F1F780019B3E
:10D730001B69002B00F0F28002F01A030A2B00F0A4
:10D74000FB8013AB10930023CDE91133CDE90A33ED
:10D7500008930DF14C09099303933B78002B00F0DB
:10D7600051813C4604E014F8013F002B00F02C816D
:10D77000252BF8D1E51B40F029812378002B00F000
:10D7800041814FF0000300258DF83B30671C637822
:10D7900002954FF0FF3B2B240137A3F120025A2AB8
:10D7A00000F25281DFE812F0980250015001940219
:10D7B0005001500150016A005001500136026B02C5
:10D7C00050014102A6025001A2025B005B005B0017
:10D7D0005B005B005B005B005B005B005001500185
:10D7E00050015001500150015001500150012302DD
:10D7F000840050015001500150015001500150016E
:10D80000500150015001DD0050015001500107024C
:10D8100050015902500150011E05500150015001A4
:10D82000500150015001500150015001500123029C
:10D8300086005001500150014F02860080005001C7
:10D84000450250018102DF006F0280005001070293
:10D850007E003E0550015001400550017E00A3F1BD
:10D860003002002117F8013B01EB810102EB41017D
:10D87000A3F13002092AF5D902918EE7DDF8148070
:10D880004046FEF7F7FF43680A931846F3F7D8FDC2
:10D890000B9006464046FEF7EDFF83680993002E85
:10D8A00040F07B843B7877E73B7845F0200573E7D1
:10D8B00045F01005AC06049E40F16F81073626F056
:10D8C00007063246736852F8086B04929846002B9C
:10D8D000C0F22D84BBF1FF3F00F0108556EA08032B
:10D8E00025F0800A00F008840A2E78F1000380F009
:10D8F000BD84303601238DF8EF60554600930DF15D
:10D90000EF04DDF800809DF83B30D845B8BFD8461D
:10D91000002B00F0A88008F10108A4E0019D059803
:10D920002946FCF7A7FE002840F08885AA8902F066
:10D930001A030A2B7FF405AF0199B1F90E30002BC1
:10D94000FFF6FFAE4B6EDE0702D4950540F156851B
:10D950000199059823463A463DB0BDE8F04F00F0E6
:10D9600093BD45F0100515F0200800F00781049ED6
:10D97000073626F007063346D6F8048053F8086BBE
:10D98000049325F4806A00234FF000028DF83B20B9
:10D99000BBF1FF3F00F0C88156EA08022AF080057B
:10D9A00040F0C181BBF1000F40F0AB84002B40F090
:10D9B000A8831AF00103009300F0D68330238DF87A
:10D9C000EF300DF1EF049CE7E51B1BD0119B129A81
:10D9D00001332A44072BC9E900751292119305DC23
:10D9E00009F10809039B2B440393C6E6002A00F0C3
:10D9F0007F830199059810AAFFF730FE40B90DF119
:10DA00004C09EFE7129B002B40F00985002311938E
:10DA1000019A536ED90740F1A68093895B0600F105
:10DA2000198503983DB0BDE8F08F019BB3F90C1048
:10DA30008D058AB23FF56DAE1D46986DFEF722FF4B
:10DA4000B5F90C108AB264E6002BDBD08DF88C306F
:10DA50004FF001084FF000038DF83B30CDF8008007
:10DA600023AC4FF0000B15F00203069318BF08F12A
:10DA7000020815F08403079305D1029BA3EB080667
:10DA8000002E00F36C82DDE91121501C9DF83B60F3
:10DA90008EB10DF13B020131C9F8002007284FF08B
:10DAA0000102CDE91101C9F8042000F33B820246CE
:10DAB00009F108090130069BDBB10FAB0231C9F84F
:10DAC000003007284FF00203CDE91101C9F80430F6
:10DAD00040F34082002900F006830199059810AABE
:10DAE000FFF7BCFD002893D1DDE911210DF14C09B0
:10DAF000501C079B802B00F05881009BABEB03066A
:10DB0000002E00F3B681009BC9F800401944072895
:10DB1000CDE91101C9F8043040F34481002900F037
:10DB200072820199059810AAFFF798FD00287FF4EA
:10DB30006FAF12990DF14C09680705D5029BA3EB55
:10DB40000804002C00F36982DDE902234245ACBFE2
:10DB50009B1843440393002940F0D581002311937F
:10DB60000DF14C09F9E5019B9B899A053FF556AFEC
:10DB7000019CA06DFEF788FEA3894FE715F0100306
:10DB800040F0238315F0400200F0EB83049A52F832
:10DB9000046B04929846B6B2F3E656F8043B04963A
:10DBA000E80600F1ED82690640F1E78243F3C038F0
:10DBB0001EB243468BE6049E56F8044B4FF000031A
:10DBC0008DF83B30002C00F0B183BBF1FF3F00F03B
:10DBD0002E835A4600212046F3F7A2FC002800F0CD
:10DBE0001284031B009304964FF0000B89E6049EF9
:10DBF0004FF000038DF83B304FF0010856F8043B1E
:10DC00008DF88C300496CDF8008023AC29E7FDF721
:10DC100075FE76E5049B53F8042B0292002A80F2ED
:10DC20009F82029A0493524202923B7845F0040587
:10DC3000B2E53B786C2B03BF7B7845F020050137BC
:10DC400045F01005A8E53B78682B03BF7B7845F4C9
:10DC50000075013745F040059EE545F0100A1AF0C1
:10DC6000200800F05582049E073626F0070633464A
:10DC7000D6F8048053F8086B0493012384E63B78BC
:10DC80008DF83B4088E5049B53F8046B04933023E4
:10DC90008DF83C3078238DF83D30B94B089345F032
:10DCA000020A4FF0000802236EE6AE0600F18382FE
:10DCB000EC0600F13383680600F19283A90540F178
:10DCC0002D83049E039A56F8043B04961A7044E58B
:10DCD0003B7845F001055FE59DF83B30002B7FF474
:10DCE000E1AD20238DF83B303B7855E53B7845F09E
:10DCF000800551E5394611F8013B2A2B00F0B3832A
:10DD0000A3F13002092A0F464FF0000B3FF645AD54
:10DD100017F8013B0BEB8B0B02EB4B0BA3F1300223
:10DD2000092AF5D939E5AA46012B3FF4DDAD022BCE
:10DD30003CAC12D1089A06F00F033609D35C04F804
:10DD4000013D46EA08764FEA181856EA0803F2D170
:10DD50003CAB1B1B55460093D3E506F00703F608C2
:10DD600046EA48764FEAD808303356EA0801224698
:10DD700004F8013DF1D11AF0010FE9D0302BE7D0C2
:10DD80003023023A04F8013C3CAB9B1A5546009301
:10DD90001446B6E50099139401231491129111933E
:10DDA0000DF14C0909F10809C6E6029BA3EB080630
:10DDB000002E7FF7A2AE102E40F35183DFF8C4A1EE
:10DDC0005346CDE906B4BA46DDF814B0019C2F469F
:10DDD0001D4607E002F1020C09F108090246103E57
:10DDE000102E1EDD501C103110230728CDE9110123
:10DDF000C9F80050C9F80430ECDD10AA002900F081
:10DE00008B80214658460DF14C09FFF727FC00286E
:10DE10007FF4FEADDDE91121103E102E02F1010C60
:10DE2000E0DCDDE906B42B463D4657469A463144D0
:10DE3000BCF1070FCDE911C1C9F800A0C9F8046011
:10DE400040F39581002900F0BB820199059810AA42
:10DE5000FFF704FC00287FF4DBAD009BDDE9112116
:10DE6000ABEB0306002E02F101000DF14C097FF728
:10DE70004AAE102EDFF80CA131DD5346CDE9064540
:10DE8000BA46059C019D4FF0100B1F4607E002F1BA
:10DE9000020C09F108090246103E102E19DD501C33
:10DEA00010310728C9E9007BCDE91101EFDD10AA87
:10DEB00019B3294620460DF14C09FFF7CFFB002886
:10DEC0007FF4A6ADDDE91121103E102E02F1010C08
:10DED000E5DCDDE906453B46604657469A46314457
:10DEE0000728CDE91101C9F800A0C9F8046000F3C2
:10DEF000E68009F10809013005E64FF0010C0A46F9
:10DF00000DF14C09C8E70199059810AAFFF7A6FB87
:10DF100000283FF423AE7BE54FF0010C0A460DF1DB
:10DF20004C095CE7002900F0DB800199059810AAF4
:10DF3000FFF794FB00287FF46BADDDE911210DF1B3
:10DF40004C09501CB7E502210FAB1491139301202B
:10DF50000DF14C09024609F10809501CC9E5102EC3
:10DF600040F35782DDE911C1DFF81CA0CDE90CB404
:10DF700010235446DDF804B0DDF814A062460DE02D
:10DF8000F8ED000824F2000814F2000802F1020C77
:10DF900009F108090246103E102E1BDD501C1031FD
:10DFA0000728C9E90043CDE91101EFDD10AA21B32B
:10DFB000594650460DF14C09FFF750FB00287FF4FD
:10DFC00027ADDDE91121103E102E02F1010C4FF0BA
:10DFD0001003E3DCA246DDF830B00D9C624631440C
:10DFE000072ACDE91121C9F800A0C9F8046000F39F
:10DFF000A78009F10809501C48E50A464FF0010CBA
:10E000000DF14C09C7E76C07119150D5029BA3EBAA
:10E010000804002C4BDD0DF14C09102C40F3098253
:10E02000DFF8ECA2119A059EDDF804B053461025E6
:10E03000BA461F4606E0901C09F108091A46103C32
:10E04000102C19DD531C1031072BC9E90075CDE9DF
:10E050001131F0DD10AA29B359463046FFF7FEFA18
:10E0600000287FF4D5ACDDE91121103C102C02F121
:10E0700001000DF14C09E5DC3B4657469A46214428
:10E080000728C9E900A4CDE911017FF75DAD71B1A1
:10E090000199059810AAFFF7E1FA00287FF4B8ACBF
:10E0A000129951E501200A460DF14C09C7E7DDE957
:10E0B00002234245ACBF9B18434403934EE500291D
:10E0C0003FF468AE0199059810AAFFF7C7FA002837
:10E0D0007FF49EAC1198129901300DF14C0912E5B4
:10E0E000069B002B77D101200A460DF14C0900E573
:10E0F00011920DF14C0975E4BBF1000F7FF4F9ABFF
:10E1000055464FF0000BCDF800B03CACFFF7F9BB23
:10E110001AF010033AD11AF0400200F01381049A69
:10E1200052F8046B04929846B6B201232CE42D23D6
:10E1300076428DF83B3068EB4808AA46012327E475
:10E1400000297DD00199059810AAFFF787FA0028C9
:10E150007FF45EACDDE911210DF14C09501C95E412
:10E1600004933B78FFF718BB3CACFFF7CABB09F13F
:10E1700008090CF101006246BFE4AA0500F13881EC
:10E180004FEAE3781E464346FFF7A1BB049B53F8D2
:10E19000046B04930123FFF7F7BB099B002B3FF4AB
:10E1A00081AB099B1B78002B3FF47CAB3B7845F49B
:10E1B0008065FFF7F1BADDE9031656F8042B0496E3
:10E1C000CB17C2E90013FFF7C8BA049B53F8046BDE
:10E1D0000493FFF7D6BB02210FAB149113930DF1FB
:10E1E0004C09B8E64B4A089215F0200836D0049E38
:10E1F000073626F007063246D6F8048052F8086B38
:10E200000492EA0709D556EA080206D08DF83D3097
:10E21000302345F002058DF83C3025F4806A022356
:10E22000FFF7B2BBAA461AE53B4A0892DCE7204654
:10E230000496F3F705F94FF0000B0090FFF761BB70
:10E240009DF83B20002A00F0C18001200DF13B0227
:10E25000149013920DF14C09014628E415F01002B8
:10E2600042D0049A52F8046B0492CAE70AF480631D
:10E27000CDF800B0CDF81890BB46DDF8249000250D
:10E280003CAC1F4609E030464146F2F739FD0A2E04
:10E2900078F100031BD306468846304641460A22E1
:10E2A0000023F2F72DFD1146303104F8011C0A223B
:10E2B0000023013C0135002FE5D099F80010A94258
:10E2C000E1D1FF2DDFD00A2E78F1000364D23CAB00
:10E2D0001B1BCDF824905F46DDF81890DDF800B0E8
:10E2E00000935546FFF70DBB15F0400147D0049948
:10E2F00051F8046B04919046B6B282E7AA46FFF744
:10E30000F3BA012BAA467FF412ADFFF7F2BA00BFB1
:10E3100014F200080CEE0008F8ED0008049E039AC1
:10E3200056F8043B1A600496FFF717BABBF1060FC4
:10E33000D84628BF4FF00608504CCDF80080049610
:10E34000FFF78FBB049B1AF4007814BF53F8046BDB
:10E3500053F8046B04931CBF9046F6B20123FFF7F9
:10E3600013BB049B15F4007814BF53F8046B53F8E7
:10E37000046B04931CBF9046F6B2FFF702BB049AED
:10E3800015F4007814BF52F8046B52F8046B049231
:10E390001CBF8846F6B234E70B9B0A99E41A1A466A
:10E3A0002046FFF729F999F801300BB109F101096D
:10E3B000304641460A2200230025F2F7A1FC6AE715
:10E3C00001200A460DF14C09FFF797BB069B002B75
:10E3D0007FF4B9AD0A4601200DF14C09FFF78DBB62
:10E3E000049E039A56F8043B04961A80FFF7B5B9C9
:10E3F00043F3C0185EB24346FFF769BA886DFEF773
:10E4000043FAFFF7A5BACDF800B004968346FFF7AC
:10E4100078BA119A1299DFF868A00132DFE5019904
:10E42000059810AAFFF71AF900283FF4EFAAFFF7A2
:10E43000EFBA1198DFF848A0013020E6019B5B6E2F
:10E44000DB0707D4019B9B899F0503D4019B986D33
:10E45000FEF71AFA4FF0FF330393FFF7E2BADFF843
:10E4600024A08446E3E4049A7B780F4652F8041B08
:10E47000049241EAE17BFFF78FB900BF20EE00086C
:10E4800014F2000824F20008F0B51F468B89ADF2A3
:10E490006C4D23F00203ADF80C304B6E1993CB8911
:10E4A000ADF80E30CB6907934B6A09931AAB009312
:10E4B00004934FF48063154606460293059316A80D
:10E4C00000230C460693FEF7D9F92A463B466946D7
:10E4D0003046FFF709F9051E07DB69463046FDF7B0
:10E4E000D9F9002818BF4FF0FF35BDF80C305B0696
:10E4F00003D5A38943F04003A3811698FEF7C0F922
:10E5000028460DF26C4DF0BD49B1FF2A02D80A70C1
:10E51000012070478A2303604FF0FF3070470846A0
:10E52000704700BF2DE9F047DFF87CA00646DAF817
:10E53000000098460F469146FEF7A4F91B4B1B6856
:10E54000D3F8484124B365681F2D26DC5EB96B1CE7
:10E550000235DAF80000636044F82570FEF794F99C
:10E560000020BDE8F08704EB85010123C1F8889005
:10E57000D4F88821AB401A43022EC4F88821C1F890
:10E580000881E4D1D4F88C211343C4F88C31DEE740
:10E5900003F5A674C3F84841D5E7DAF80000FEF7A2
:10E5A00073F94FF0FF30DCE76008002484ED0008C9
:10E5B00000B50B4C25681446EE681A4685B0034634
:10E5C0000D464CB107490095CDE901143046064986
:10E5D00000F0B0F800F0E8F904490C46F3E700BF9A
:10E5E0002000002434F2000844F2000888EB000800
:10E5F00038B5A1FB02148CBBF8F7F6FB0546E0B179
:10E6000050F8042C22F00302043A242A17D8132AC3
:10E610001AD91B2AC0E900441DD9242A14BF00F1CD
:10E62000100200F118024FF00003C0E9024404BFD9
:10E6300004614461C2E900339360284638BD214635
:10E64000F8F782FE284638BD02460023C2E90033AF
:10E650009360284638BD00F10802F6E7F8F78AFB18
:10E660000C2300250360E8E770B500294BD006466F
:10E670000C4610B1836B002B48D0636ED80734D59D
:10E68000B4F90C30002B3ED021463046FDF772F82D
:10E69000E36A054633B1E169304698470028B8BFC0
:10E6A0004FF0FF35A3891A063BD4216B41B104F129
:10E6B0004003994202D03046FDF718FA0023236345
:10E6C000616C21B13046FDF711FA00236364FDF758
:10E6D0009BF9636E0022DB07A28127D5A06DFEF7B0
:10E6E000CFF8FDF797F9284670BDA3899905CBD4DB
:10E6F000A06DFEF7C7F8B4F90C30002BC4D1656EDD
:10E7000015F0010508D00025284670BDFDF7F6F884
:10E71000636ED807B4D4E8E7A06DFEF7B5F82846D5
:10E7200070BD21693046FDF7E1F9BEE7A06DFEF747
:10E73000ABF8D3E70EB410B583B005AB064C53F875
:10E74000042B019301462068FEF7CEFF03B0BDE81D
:10E75000104003B0704700BF200000242DE9F043B3
:10E7600083B0074688461446FEF77EF8012803D199
:10E7700008F1FF33FE2B37D9424604F15C0301A9AF
:10E78000384600F0F3F8421C064633D038B39DF803
:10E7900004C00DF10509002509E023685A1C226018
:10E7A00083F800C00135B54219D219F801CBA3682E
:10E7B000013B002BA360F0DAD4F818E07345614602
:10E7C0002246384602DBBCF10A0FE6D100F076F8AB
:10E7D000431CE7D10646304603B0BDE8F083464609
:10E7E000304603B0BDE8F0835FFA88FC8DF804C0C2
:10E7F0000646CEE7A389304643F04003A38103B029
:10E80000BDE8F08330B5536E13F0010FB2F90C3050
:10E81000144683B005469AB201D198051CD59004E0
:10E8200006D4626E43F4005342F40052A381626640
:10E8300022462846FFF792FF636EDA07054602D4A8
:10E84000A3899B0502D5284603B030BDA06DFEF715
:10E850001BF8284603B030BDA06D0191FEF712F8F9
:10E86000B4F90C3001999AB2D9E700BF70B50C46E3
:10E87000084D03460026204611461C462E60F4F73C
:10E8800053F9431C00D070BD2B68002BFBD02360D4
:10E8900070BD00BF540D002438B5074D002204465A
:10E8A00008462A60F4F7EEF8431C00D038BD2B6808
:10E8B000002BFBD0236038BD540D0024F8B50D4665
:10E8C0001446064610B1836B002B43D0B4F90C20DC
:10E8D000A369A360170790B21BD52369CBB1EDB232
:10E8E00081042F4622D522686169D31A994229DD15
:10E8F0000133A1680139A160511C21601570626962
:10E900009A422AD0A389DB0701D50A2D25D03846A3
:10E91000F8BD21463046FBF7ADFE20BBB4F90C2014
:10E92000236990B2EDB281042F46DCD442F4005248
:10E93000A281626E616922F4005262662268D31A73
:10E940009942D5DC21463046FCF7A4FF58B922682D
:10E950000123CEE7FCF7D2FFB8E721463046FCF7AB
:10E9600099FF0028D3D04FF0FF37D0E770B50546A8
:10E9700084B01C4639B10B4ED6F8E060B047431C5A
:10E9800009D004B070BD0A460649D1F8E06001A97B
:10E99000B047431CF5D100228A2322602B6004B0CB
:10E9A00070BD00BF6808002408B5062000F004F818
:10E9B0000120F4F7FFF800BF38B5154B1F281D687C
:10E9C00020D8D5F8DC22044662B152F820304BB191
:10E9D000012B15D0591C0FD0002542F82050984724
:10E9E000284638BD284600F02BF822460146284626
:10E9F000BDE8384000F00EB816232B60012038BD6A
:10EA0000002038BD16232B604FF0FF3038BD00BF0B
:10EA10002000002470B50C46084D03460026204611
:10EA200011461C462E60F4F7BDF8431C00D070BDA3
:10EA30002B68002BFBD0236070BD00BF540D002459
:10EA4000F4F7AEB8F8B500BFF8BC08BC9E467047F6
:0CEA5000F8B500BFF8BC08BC9E4670473B
:10EA60005374203D2025640A0000000054656D7039
:10EA7000657261747572653A252E31660D0A000063
:10EA8000BDD3CAD5B5BDB5C44A534F4EC3FCC1EEC4
:10EA90003A200000C7D0B8EED6AEBAF3A3BA20250C
:10EAA000730D0A00495249535F5A48555F3031008F
:10EAB00053656E736F725F31000000003230323484
:10EAC00030313331000000004972697300000000EA
:10EAD000EFBBBF006E756C6C000000002564000089
:10EAE00025312E3135670000256C670025312E3128
:10EAF0003767000066616C736500000074727565AD
:10EB0000000000004A534F4E20737472696E673ADA
:10EB10002025730D0A00000074656D7065726174C4
:10EB200075726500706E0000736E000070726F6425
:10EB3000756374696F6E5F64617465006D616E7595
:10EB400066616374757265720000000064657669C1
:10EB500063655F706978656C5F6C656E677468008B
:10EB60007365745F696E746567726174696F6E5FF7
:10EB700074696D650000000054656D7065726174A4
:10EB80007572653A2025640A00000000506E3A252F
:10EB9000640A0000536E3A25640A000050726F64E4
:10EBA000756374696F6E5F646174653A25640A0009
:10EBB0004D616E7566616374757265723A25640A9B
:10EBC000000000004465766963655F506978656C94
:10EBD0005F4C656E6774683A25640A005365745F1C
:10EBE000496E746567726174696F6E5F54696D65B3
:10EBF0003A25640A000000004A534F4E20706172AB
:10EC000073696E67206572726F72204A534F4E208F
:10EC100070617273696E67206572726F72204A53F9
:10EC20004F4E2070617273696E67206572726F72E9
:10EC3000204A534F4E2070617273696E672065726F
:10EC4000726F722E00000000000000000102030439
:10EC5000010203040607080901000200040006007F
:10EC600008000A000C001000200040008000000195
:10EC70000804020408010101010101030701000069
:10EC8000002020202020202020202828282828207C
:10EC90002020202020202020202020202020202074
:10ECA00020881010101010101010101010101010DC
:10ECB00010040404040404040404041010101010CC
:10ECC0001010414141414141010101010101010196
:10ECD00001010101010101010101010110101010E8
:10ECE0001010424242424242020202020202020268
:10ECF00002020202020202020202020210101010BC
:10ED000020000000000000000000000000000000E3
:10ED100000000000000000000000000000000000F3
:10ED200000000000000000000000000000000000E3
:10ED300000000000000000000000000000000000D3
:10ED400000000000000000000000000000000000C3
:10ED500000000000000000000000000000000000B3
:10ED600000000000000000000000000000000000A3
:10ED70000000000000000000000000000000000093
:10ED800000000000280000246E660000696E6974AF
:10ED900079000000616E000035000000CEFBFFFF2F
:10EDA000CB03000001000000000000003400000060
:10EDB000CEFBFFFFCB0300000100000000000000BD
:10EDC000BC89D897B2D29C3C33A7A8D523F6493941
:10EDD0003DA7F444FD0FA5329D978CCF08BA5B2563
:10EDE000436FAC6428066811494E4600696E6600A0
:10EDF0004E414E006E616E0030313233343536375D
:10EE00003839616263646566000000003031323376
:10EE10003435363738394142434445460000000016
:10EE2000286E756C6C290000300000002020202026
:10EE30002020202020202020202020203030303092
:10EE40003030303030303030303030304E614E0085
:10EE5000496E66696E6974790000000042616C6CED
:10EE60006F6320737563636565646564000000000B
:10EE70002F6D6E742F776F726B73706163652F7770
:10EE80006F726B73706163652F4743432D31302D73
:10EE9000706970656C696E652F6A656E6B696E73FB
:10EEA0002D4743432D31302D706970656C696E6557
:10EEB0002D3333385F32303231313031385F3136D3
:10EEC00033343531363230332F7372632F6E6577BA
:10EED0006C69622F6E65776C69622F6C6962632F53
:10EEE0007374646C69622F64746F612E6300000038
:10EEF0002F6D6E742F776F726B73706163652F77F0
:10EF00006F726B73706163652F4743432D31302DF2
:10EF1000706970656C696E652F6A656E6B696E737A
:10EF20002D4743432D31302D706970656C696E65D6
:10EF30002D3333385F32303231313031385F313652
:10EF400033343531363230332F7372632F6E657739
:10EF50006C69622F6E65776C69622F6C6962632FD2
:10EF60007374646C69622F6764746F612D67657474
:10EF70006865782E630000000000000000000000BB
:10EF80000000000000000000000000000000000081
:10EF90000000000000000000000000000000000071
:10EFA00000000000000000001011121314151617C5
:10EFB0001819000000000000001A1B1C1D1E1F0075
:10EFC0000000000000000000000000000000000041
:10EFD0000000000000000000001A1B1C1D1E1F0086
:10EFE0000000000000000000000000000000000021
:10EFF0000000000000000000000000000000000011
:10F000000000000000000000000000000000000000
:10F0100000000000000000000000000000000000F0
:10F0200000000000000000000000000000000000E0
:10F0300000000000000000000000000000000000D0
:10F0400000000000000000000000000000000000C0
:10F0500000000000000000000000000000000000B0
:10F0600000000000000000000000000000000000A0
:10F0700000000000000000002E00000078F00008F2
:10F0800088EB00086408002443000000504F5349F7
:10F09000580000002F6D6E742F776F726B73706164
:10F0A00063652F776F726B73706163652F4743439E
:10F0B0002D31302D706970656C696E652F6A656ED3
:10F0C0006B696E732D4743432D31302D7069706528
:10F0D0006C696E652D3333385F3230323131303107
:10F0E000385F313633343531363230332F73726313
:10F0F0002F6E65776C69622F6E65776C69622F6C15
:10F100006962632F7374646C69622F6D70726563DA
:10F110002E630000000000000080E03779C3414307
:10F12000176E05B5B5B89346F5F93FE9034F384D6D
:10F13000321D30F94877825A3CBF737FDD4F157519
:10F14000000000000000F03F00000000000024402C
:10F1500000000000000059400000000000408F4007
:10F16000000000000088C34000000000006AF84072
:10F170000000000080842E4100000000D012634196
:10F180000000000084D797410000000065CDCD410C
:10F19000000000205FA00242000000E876483742ED
:10F1A000000000A2941A6D42000040E59C30A2428B
:10F1B0000000901EC4BCD64200003426F56B0C4300
:10F1C0000080E03779C3414300A0D88557347643A7
:10F1D00000C84E676DC1AB43003D9160E458E14308
:10F1E000408CB5781DAF154450EFE2D6E41A4B447D
:10F1F00092D54D06CFF08044F64AE1C7022DB544C2
:10F20000B49DD9794378EA44050000001900000054
:10F210007D000000202020202020202020202020F1
:10F22000202020203030303030303030303030301E
:10F23000303030302C2066756E6374696F6E3A2002
:10F2400000000000617373657274696F6E2022257F
:10F250007322206661696C65643A2066696C65207A
:10F26000222573222C206C696E6520256425732568
:04F27000730A00001D
:08F27400BC1AFF7F010000003D
:08F27C0049A70008E5020008A3
:04F28400C1020008BB
:10F28800C96D0008D96D0008D97400080100000094
:10F298000090D0030090D00301000000100000008F
:10F2A80028000024000000000000000014030024CF
:10F2B8007C030024E4030024000000000000000098
:10F2C8000000000000000000000000000000000036
:10F2D8000000000000000000000000000000000026
:10F2E8000000000000000000000000000000000016
:10F2F8000000000000000000000000000000000006
:10F3080000000000000000000000000000000000F5
:10F3180000000000000000000000000000000000E5
:10F3280000000000000000000000000000000000D5
:10F3380000000000000000000000000000000000C5
:10F3480000000000000000000000000000000000B5
:10F3580001000000000000000E33CDAB34126DE652
:10F36800ECDE05000B0000000000000000000000BB
:10F378000000000000000000000000000000000085
:10F388000000000000000000000000000000000075
:10F398000000000000000000000000000000000065
:10F3A8000000000000000000000000000000000055
:10F6D8000000000000000000500400245004002432
:10F6E8005804002458040024600400246004002402
:10F6F80068040024680400247004002470040024B2
:10F708007804002478040024800400248004002461
:10F718008804002488040024900400249004002411
:10F728009804002498040024A0040024A0040024C1
:10F73800A8040024A8040024B0040024B004002471
:10F74800B8040024B8040024C0040024C004002421
:10F75800C8040024C8040024D0040024D0040024D1
:10F76800D8040024D8040024E0040024E004002481
:10F77800E8040024E8040024F0040024F004002431
:10F78800F8040024F80400240005002400050024DF
:10F79800080500240805002410050024100500248D
:10F7A800180500241805002420050024200500243D
:10F7B80028050024280500243005002430050024ED
:10F7C800380500243805002440050024400500249D
:10F7D800480500244805002450050024500500244D
:10F7E80058050024580500246005002460050024FD
:10F7F80068050024680500247005002470050024AD
:10F80800780500247805002480050024800500245C
:10F81800880500248805002490050024900500240C
:10F828009805002498050024A0050024A0050024BC
:10F83800A8050024A8050024B0050024B00500246C
:10F84800B8050024B8050024C0050024C00500241C
:10F85800C8050024C8050024D0050024D0050024CC
:10F86800D8050024D8050024E0050024E00500247C
:10F87800E8050024E8050024F0050024F00500242C
:10F88800F8050024F80500240006002400060024DA
:10F898000806002408060024100600241006002488
:10F8A8001806002418060024200600242006002438
:10F8B80028060024280600243006002430060024E8
:10F8C8003806002438060024400600244006002498
:10F8D8004806002448060024500600245006002448
:10F8E80058060024580600246006002460060024F8
:10F8F80068060024680600247006002470060024A8
:10F908007806002478060024800600248006002457
:10F918008806002488060024900600249006002407
:10F928009806002498060024A0060024A0060024B7
:10F93800A8060024A8060024B0060024B006002467
:10F94800B8060024B8060024C0060024C006002417
:10F95800C8060024C8060024D0060024D0060024C7
:10F96800D8060024D8060024E0060024E006002477
:10F97800E8060024E8060024F0060024F006002427
:10F98800F8060024F80600240007002400070024D5
:10F998000807002408070024100700241007002483
:10F9A8001807002418070024200700242007002433
:10F9B80028070024280700243007002430070024E3
:10F9C8003807002438070024400700244007002493
:10F9D8004807002448070024500700245007002443
:10F9E80058070024580700246007002460070024F3
:10F9F80068070024680700247007002470070024A3
:10FA08007807002478070024800700248007002452
:10FA18008807002488070024900700249007002402
:10FA28009807002498070024A0070024A0070024B2
:10FA3800A8070024A8070024B0070024B007002462
:10FA4800B8070024B8070024C0070024C007002412
:10FA5800C8070024C8070024D0070024D0070024C2
:10FA6800D8070024D8070024E0070024E007002472
:10FA7800E8070024E8070024F0070024F007002422
:10FA8800F8070024F80700240008002400080024D0
:10FA9800080800240808002410080024100800247E
:10FAA800180800241808002420080024200800242E
:10FAB80028080024280800243008002430080024DE
:10FAC800380800243808002440080024400800248E
:10FAD8004808002448080024FFFFFFFF0000020038
:10FAE800440D0024FF000000430000000000000057
:10FAF80000000000000000000000000000000000FE
:10FB080000000000000000004300000000000000AA
:10FB180000000000000000000000000000000000DD
:10FB2800000000000000000043000000000000008A
:10FB380000000000000000000000000000000000BD
:10FB4800000000000000000043000000000000006A
:10FB5800000000000000000000000000000000009D
:10FB6800000000000000000043000000000000004A
:10FB7800000000000000000000000000000000007D
:10FB8800000000000000000043000000000000002A
:10FB9800000000000000000000000000000000005D
:10FBA800000000000000000043000000000000000A
:10FBB800000000000000000000000000000000003D
:10FBC800000000000000000009E50008F9C900086D
:10FBD8000000000080EC000878F0000888EB0008BE
:10FBE80088EB000888EB000888EB000888EB000821
:10FBF80088EB000888EB000888EB000888EB000811
:10FC0800FFFFFFFFFFFFFFFFFFFFFFFFFFFF0000FA
:10FC18000100415343494900000000000000000072
:10FC280000000000000000000000000000000000CC
:10FC38000000415343494900000000000000000053
:10FC480000000000000000000000000000000000AC
:04FC580000000000A8
:0400000508002F6957
:00000001FF
